:020000040000FA
:1000000090F40720190200001D0200001F020000EA
:10001000210200002302000025020000B2FEF7DFEB
:1000200000000000000000000000000027020000A7
:1000300029020000000000002B0200002D02000039
:100040002F020000350200002F0200002F020000E6
:100050002F0200002F0200002F0200002F020000DC
:100060002F0200002F0200002F0200002F020000CC
:100070002F0200002F0200002F0200002F020000BC
:100080002F0200002F0200002F0200002F020000AC
:100090002F0200002F0200002F0200002F0200009C
:1000A0005B2A00002F0200002F0200002F02000038
:1000B0002F0200002F0200002F0200002F0200007C
:1000C0002F0200002F0200002F020000DFF80CD0EA
:1000D00005F038FC00480047DB0F000090F40720D3
:1000E000D0F800D0D0F804F02A4810B500780028E5
:1000F0000CD12949294800F0E0FC80232649BDE8BD
:1001000010401A461031254800F091BC10BD70B562
:100110000C4605462049214800F0CFFC22462946DE
:10012000BDE870404FF480731C4800F003BD70B50B
:100130001A4C41F2210340346088984215D00021C6
:100140004FF6FF7505EA01205FF0000210F4004F42
:1001500005EA400000D05840521C082AF6DB24F87B
:100160001100491C89B2FF29ECD970BD70B50B4D47
:10017000002340350AE0CE5C04885B1C86EA142626
:100180009BB235F8166086EA04240480521E92B2AF
:10019000F1D270BD00C00720DC5A000054C2072015
:1001A000EFF3108010F0010F72B64FF080404FF067
:1001B000000202704FF0AA0303724FF0550404725C
:1001C00002614FF0FF0242604FF0030202700372BF
:1001D000047200D162B6FEE770B50025102400203D
:1001E00000F0B2F8C0F30B100544641EF7D12909E2
:1001F0004FF47A70B1FBF0F06422B1FBF2F100072A
:100200000A22B1FBF2F302FB131141EA106001492B
:10021000086070BDD0C0072005480047FEE7FEE734
:10022000FEE7FEE7FEE7FEE7FEE7FEE7FEE7FEE7A6
:10023000CD00000010B54FF040210120086001F012
:1002400085FF01F0B9FF10BD4FF04020002101678C
:1002500002224260C1600321416144F25061816128
:100260000B4B182183F8001401215B1EC3F80021F9
:10027000416000207047074802214160002101676A
:1002800041611122C260C1630121416000207047B9
:1002900001E000E000000940FEE7FEE7FEE7FEE7C0
:1002A00012498220086012490220086078461149EC
:1002B00008608220704704F0BABD04F0E4BD30B499
:1002C00020F070430C4C000F54F820401846A44610
:1002D00030BC604730B420F07043074C000F40340E
:1002E00054F820401846A44630BC604784C007201C
:1002F00088C007208CC00720205E0000214365874E
:100300001849174808601849886842F210728B68CB
:100310001B1A9342FBD30020704712490A6822F04F
:1003200080720A600A68012322F0FF0283401A43A8
:1003300042F08070086048680028FCDA0A6822F001
:1003400080720A6080B2704710B5EFF3108101F03F
:10035000010472B6FFF7E1FF002C00D162B610BDB8
:100360000001200000400340000009401948062118
:100370000161072101600021416141620221416068
:10038000C168C906FCD400E08168C1684907FBD494
:10039000002070470F498860C868C006FCD4886890
:1003A000704700B50B46024604E000BF12F8010B8F
:1003B000FFF7F0FF5B1EF9D200BD00B50B46024609
:1003C00004E00020FFF7E6FF02F8010B5B1EF8D205
:1003D00000BD00000080084010B50B4604461146E1
:1003E000184605F09BFAC4E9000110BD02E008C8F8
:1003F000121F08C1002AFAD17047704700000000A0
:1004000000000000A92040EA01039B0703D009E097
:1004100008C9121F08C0042AFAD203E011F8013BF0
:1004200000F8013B521EF9D27047000000000000A6
:100430000000000002000000FFB5BCA60446E1CEAB
:100440008DE8E100022902DA002004B0F0BD601856
:10045000002100F8011D6946B3FBF2F502FB1535DA
:10046000B3FBF2F34D5D00F8015DA042F4D8ECE778
:1004700010B504F0B9FC04F0A3FCB0494FF40052ED
:10048000C1E90020A0F5F420886010BD70B50346D6
:1004900008468D18A949002449688D4200D9881A58
:1004A000194604F01BFD204670BDF8B51446A34E56
:1004B0000A460B19716800258B4200D90A1B0346B6
:1004C0000094306804F035FD2846F8BD10B50B46A1
:1004D00001460024184604F0AAFC204610BD2DE970
:1004E000FC410746002090460E46ADF80000044649
:1004F0000EE0351B402D00D9402539192A46904879
:10050000FFF7E4FFAAB28E496846FFF72FFE2C449E
:10051000B442EED33919424601A8FFF7D7FFBDF820
:100520000000BDF80410884202D10120BDE8FC8122
:100530000020FBE70021425C12B9491C1829FAD3BC
:10054000182901D000207047012070472DE9F04F95
:100550007A4C074606460C348BB00020A070E07041
:1005600088462071FFF7C0FDDFF8D8A1DFF8D891E9
:100570004FF4807B0125192231466846FFF7A6FF1C
:10058000022216213046FFF7AAFF00287DD0DDF8B1
:100590000E10022206F11900FFF7A1FF002874D007
:1005A0009DF8000006282CD2DFE800F02B03032B77
:1005B0002B1CDAF87420DDF80A30521C93421FD24B
:1005C000DAF87410DDF80A30C91ADDF80E30491C6B
:1005D000994215D3DDF80A10DDF80E301944914226
:1005E0000ED80EE0DDF80E10B1F5F42F00D9A5708D
:1005F000DDF81210C1F30B41A1F58072113A00D061
:10060000A570012803D0022801D0052845D19DF806
:1006100008005A46400706F2194107D54B48FFF734
:1006200055FF49494948FFF772FD02E04648FFF788
:100630004DFF00200990B9F80410ADF82410099A74
:10064000019992B24846914200D0A57000210991CB
:10065000017B8DF82410099ABDF80110D2B29142A5
:1006600000D0A5709DF80010022916D1016B0991E8
:10067000DDF81210099A914200D0A570002109916D
:1006800099F834008DF8240000E032E009999DF8D3
:100690000300C9B2884200D0A5709DF81800401E22
:1006A000FE2800D2A570BDF80100A0F57F41FF39FA
:1006B00001D0562802D19DF8030060B96846FFF7C3
:1006C00039FF40B9BDF80100502803D19DF8000062
:1006D000052800D0A570DDF80E001B3606446846DC
:1006E000FFF728FF30B1E07880B1217988420DD042
:1006F00012E0A5709DF8180010B92079401C2071F7
:10070000E078401CC0B2E0700C2801D3A57003E073
:10071000A07800283FF42FAFB8F1000F02D0F11BF2
:10072000C8F80010A0780BB0BDE8F08F303132333C
:1007300034353637383941424344454604C00720F2
:1007400094C40720D45B000094C6072094C50720FA
:1007500030B590B000236A4651F8234042F8234058
:100760005B1C102BF8DB0823049D009C2C44009498
:10077000009D0C9C6C404FEA34440C940C9D089CEA
:100780002C440894089D049C6C404FEA3454049413
:10079000049D009C2C440094009D0C9C6C404FEAEE
:1007A00034640C940C9D089C2C440894089D049C73
:1007B0006C404FEA74640494059D019C2C440194A0
:1007C000019D0D9C6C404FEA34440D940D9D099C95
:1007D0002C440994099D059C6C404FEA34540594BF
:1007E000059D019C2C440194019D0D9C6C404FEA99
:1007F00034640D940D9D099C2C440994099D059C1D
:100800006C404FEA74640594069D029C2C4402944B
:10081000029D0E9C6C404FEA34440E940E9D0A9C3F
:100820002C440A940A9D069C6C404FEA345406946A
:10083000069D029C2C440294029D0E9C6C404FEA43
:1008400034640E940E9D0A9C2C440A940A9D069CC6
:100850006C404FEA74640694079D039C2C440394F7
:10086000039D0F9C6C404FEA34440F940F9D0B9CEA
:100870002C440B940B9D079C6C404FEA3454079416
:10088000079D039C2C440394039D0F9C6C404FEAEE
:1008900034640F940F9D0B9C2C440B940B9D079C70
:1008A0006C404FEA74640794059D009C2C440094AE
:1008B000009D0F9C6C404FEA34440F940F9D0A9C9E
:1008C0002C440A940A9D059C6C404FEA34540594CC
:1008D000059D009C2C440094009D0F9C6C404FEAA9
:1008E00034640F940F9D0A9C2C440A940A9D059C25
:1008F0006C404FEA74640594069D019C2C4401945D
:10090000019D0C9C6C404FEA34440C94DDE90B458E
:100910002C440B940B9D069C6C404FEA3454069477
:10092000069D019C2C440194019D0C9C6C404FEA57
:1009300034640C94DDE90B452C440B940B9D069C10
:100940006C404FEA74640694079D029C2C44029408
:10095000029D0D9C6C404FEA34440D940D9D089C03
:100960009B1E2C440894DDE907456C404FEA345443
:100970000794079D029C2C440294029D0D9C6C40A0
:100980004FEA34640D940D9D089C2C440894DDE9D5
:1009900007456C404FEA74640794DDE903452C4435
:1009A0000394039D0E9C6C404FEA34440E940E9DBC
:1009B000099C2C440994099D049C6C404FEA3454D2
:1009C0000494DDE903452C440394039D0E9C6C4084
:1009D0004FEA34640E940E9D099C2C440994099DA1
:1009E000049C6C404FEA74640494002B3FF7BCAE47
:1009F0005FF0000352F8234051F823502C4442F892
:100A000023405B1C102BF5DB5FF0000100EB810342
:100A100052F8214000F82140250A5D70250C240E73
:100A20009D70491CDC701029F0DB10B030BD10B592
:100A3000CC780B68B2F5807F64F31F630361CC79D7
:100A40004B6864F31F634361CC7A8B6864F31F6364
:100A50008361CC7BCB6864F31F63C36129D0364AC2
:100A6000CC780B6864F31F630362CC794B6864F342
:100A70001F634362CC7A8B6864F31F638362CB7B12
:100A8000C96863F31F61C162D378116863F31F61A2
:100A90000160D379516863F31F614160D37A916833
:100AA00063F31F618160D37BD16863F31F61C16011
:100AB00010BD214A103A1031D2E70022026342638E
:100AC000CB780A6863F31F628263CA79496862F36C
:100AD0001F61C16370472DE9F04190B01C001646BC
:100AE0000F46054618D0E84629466846FFF730FE0F
:100AF000286B401C286302D1686B401C6863402C43
:100B00004FF00000414605D909E03A5C0B5C5A40C1
:100B10003254401CA042F8D310B0BDE8F0813A5CDA
:100B20000B5C5A403254401C4028F8DB403C4036B5
:100B30004037D9E7CFE700000C5B00002DE9F0411A
:100B4000092000F09FFFF84800264FF47A770670DE
:100B5000C821384601F0DAFAF44CA06842F2107568
:100B6000A168091AA942FBD3C821384601F0CEFA80
:100B7000A068A168091AA942FBD3C821384601F030
:100B8000C5FAEB48022186708171C670BDE8F0811C
:100B90008EB04FF0000ACDF828A046208DF8140042
:100BA0008DF817A038208DF8150036208DF8160026
:100BB000E048CDF824A0D34602684FF6FF031A4060
:100BC000DD4B42F480721A430260DC486FF47051CE
:100BD000DD4AC0F800A0DA4800680144D9489142D3
:100BE000016000D902600068D84900F5E050D94D95
:100BF0000860D749400A0860F8202870FF20687014
:100C0000A87001F01BFACA4CD349002094F90520C2
:100C100051F82220291801F58051135C401C81F8FD
:100C200000386028F6D34FF4E175294640F24910A8
:100C300001F06CFA294640F29F1001F067FA4FF478
:100C400000594D46207808B101F088FFA07938B1ED
:100C500001281ED003287CD0207800287AD0A6E175
:100C60000A2000F00FFF00214E464846FFF76EFCB9
:100C700018B100BFFFF762FFE4E70120A07135461D
:100C800084F803B0062000F0FDFE0A2000F0FAFE12
:100C9000D8E719222946B148FFF718FCAF48007E73
:100CA00000287BD0AD480078062878D2DFE800F035
:100CB000E003318F8F9240F23440A84E077840F223
:100CC000044000880C90307A400713D541F2194057
:100CD00029184FF48072A248FFF7F8FB06F11901BA
:100CE0009F48FFF714FA06F1190090F834008DF8C8
:100CF000100006E041F24D402918012204A8FFF738
:100D0000E5FB70680C99884249D09DF81000B84204
:100D100045D3924F3878022808D100F041FE28B11F
:100D200046F23440F9780078814238D3787A4FF02F
:100D3000010A012833D1D7F80A0018B98948806917
:100D4000C7F80A004FF480780026072000F09AFECA
:100D500001E012E124E1D7F80E00B0422AD9801B4D
:100D6000FF2800D88046FF22511C7D4804F0C4FDB6
:100D7000A91942467A481931FFF7A8FB387A40078B
:100D80000ED5764976481931FFF7C1F9D7F80A0030
:100D9000724930444FF48072193107E088E015E061
:100DA000D7F80A004FF4807230446D4900F0BEFD60
:100DB0004644CAE7387801285AD14FF0E0210006AE
:100DC000C1F88001D7F80A0000F0E3FD50E04FF0D1
:100DD000010A50E061484FF0010A417A03294AD1E3
:100DE0005749614A4FF000060B681360027A5207B8
:100DF00020D54FF48077804617E0072000F042FEB0
:100E0000A9193A4656481931FFF760FB534954482F
:100E10001931FFF77CF94A483A46006881194F4872
:100E20001930FFF742FB06F58076D8F80E00B04285
:100E3000E3D81DE0804616E0072000F023FED7F837
:100E40000E00871B402F00D94027A9193A46444875
:100E50001931FFF73BFB3A483A4600688119404890
:100E6000FFF723FB3E44D8F80E004746B042E3D8D4
:100E70003A48007EE0B1394E307AC00613D53A497F
:100E800001220CA8C1F8009005F11801CDF830B08E
:100E9000FFF7FCFA307820B1C8214FF47A7001F0E6
:100EA00035F9307E20B1307A800701D5FFF778F927
:100EB0002A481B35D0F80E0005442848FFF73AFBB6
:100EC00048B302201849A0714D4681F800B00B20AC
:100ED00000F0D8FDBAF1000F1DD014484FF0000A01
:100EE000816842F2107283685B1A9342FBD34FF41D
:100EF0002F714FF47A7001F009F91C48416DC90453
:100F000005D5406D400502D500200B9001E00B98FF
:100F100008B9FFF745F9E078401CC0B2E0700C2832
:100F200026D30120A070A5E680C00720000009405C
:100F300010C007200CED00E00000FA05C4C0072037
:100F40000CC00720B4C0072000D03900ACC0072077
:100F5000B0C00720ADC8072078C0072094C707207D
:100F600094C407205C5B000004C0072000C0092077
:100F7000A07800283FF480AE7CE6434881680A9858
:100F8000091A099800EB4002C2EBC010B1EBC00F88
:100F9000FFF472AE00200A90099084F806B051E682
:100FA0000120207001F072FC012001F030FC374874
:100FB00000780028F3D0002105A800F0FCFB0028F1
:100FC000EDD00320A071304884F803B04D4680680E
:100FD0000A904FF47A70099034E62D4C0025FF20DA
:100FE0002560A580A5716071FFF7A1F8FFF77CF877
:100FF00000F008FE62B600F0B3FEFFF73CF9FFF721
:1010000023F900F005FD002000F03CFDFFF778F922
:10101000FFF7E2F8FFF7AAF904F0EFF901F0F7F8AB
:1010200001F0BAF842280FD01A48406DC0040BD422
:10103000042000F027FD1449886842F210728B6882
:101040001B1A9342FBD36571FFF712FA00214FF48C
:101050000050FFF77BFA80B100F0A2FC68B10220DB
:1010600000F010FD94F90500401C03D10A48806986
:1010700000F08FFC0120607004E0022000F002FD0F
:1010800065706571FFF784FD0000094080C007208E
:1010900010C0072000C009205C5B00002DE9F0476C
:1010A000FE4A00234FF40077156A4FF4FF79C5F329
:1010B0000724DFF8ECA34FF4E05CDFF8E883FA4E96
:1010C00025E0B84216D213280CD014280CD048457D
:1010D0000CD0A0F58072FF3A0AD03E2813D81AF837
:1010E000002011E0EAB20FE022460DE055220BE0AD
:1010F000AA2209E0604506D208EB0002A2F5805260
:1011000092F8002E00E00022F254401C5B1C8B423F
:10111000D7D3BDE8F08770B5E04D2C6B402C00D9DB
:101120004024E86AE96902198A4202D90C1A0421AA
:1011300069702146FFF7B2FF2246DB49822001F0A9
:1011400062FCE86A2044E862286B011BD7482963E7
:101150008268A2EB0402826005D06978022901D07E
:101160000021017370BD03216970F9E7CF4910B503
:10117000CF4808600D22822001F045FCC7490520B8
:10118000487010BD70B50D46CA494A6DD20402D5EB
:10119000496D490521D4B0F5007F1ED3C64BBF4C25
:1011A000B0F5E05F1AD29968A269891AC34A9142E0
:1011B00004D39968A161002161606161BB4A00218B
:1011C0005F3AB84B07E044181C44565CA4F58054C1
:1011D000491C84F8006EA942F5D370BD616921B93C
:1011E0009968A16199686161A060B5494979002950
:1011F000F3D199686269891AB24A91421CD2B24A03
:10120000012111709968A16199686161A168401A12
:101210006168884203D9616A884200D26060062012
:1012200000F030FC61682A46BDE870409F4801F537
:1012300000515F38FFF739B9BDE870400C2000F06D
:1012400021BC10B5954CA178E06A4218E1698A4248
:1012500006D9081AA07005206070022001F08EFBEC
:10126000A178E06AFFF78EFFA178E06A0844E062A7
:10127000206B421A8D4822638368A3EB01018160D1
:1012800002D06178052904D100210173BDE8104026
:101290006CE710BD2DE9F041804CA178E06A42185E
:1012A000E1698A4206D9081AA07005206070022000
:1012B00001F064FB7D4D0021A0787B4B5F3DE26A2D
:1012C00008E056186F5C9E5DBE4202D00021A1620C
:1012D00002E0491C8142F4D31118E162216B0A1A21
:1012E000724922638B68A3EB0000886002D06078AB
:1012F000052808D1A06A20B100200873BDE8F0419C
:1013000034E70120F9E7BDE8F081684810B51F38DF
:10131000D0F81110027D09BA21F0FF0111435F4A94
:101320004902D162C18A49BA490211638068884280
:101330000CD0822001F022FB022001F01FFB5B4950
:1013400002200873FFF712FF002010BD012010BD1E
:1013500070B55648554D1F380224816829B1007B6D
:10136000000607D4022001F009FB2C73FFF7FEFEF4
:10137000002070BD012070BD10B54C48474C1F388F
:101380008068A178884200D2A0704849A2785F396D
:10139000822001F038FB032060704448A278816805
:1013A000891A81600021017310BD404810B51F38B3
:1013B000816839B1007B000601D5822000E002205F
:1013C00001F0DCFA394900200873BDE81040CDE691
:1013D00010B5FFF7BDFF00281FD0344870215F38DB
:1013E00002220170002141708270C170017141714F
:1013F00081710A22C271017241728172C1723022FE
:101400000273012242738173C173017441742349D1
:1014100012208870BDE81040AEE710BD1CB5FFF784
:1014200097FF00286AD029480A22062103886846C7
:10143000FFF702F81D4800225F38802302704370D6
:1014400082700121C1702021017143718271C271CA
:1014500041220272542242724F2282724C22C27284
:10146000017341738173C173462202745023437424
:10147000722383746923C3746E23037574234375C5
:101480008175C2756C220276612242767322827661
:101490006822C27601774177817719E090C00720F2
:1014A0001C5B0000ADC8072094C407200CE3072094
:1014B0005553425300C0092000000940A086010096
:1014C00010C0072020A1070080C0072004040000EE
:1014D000C1779DF8011080F820109DF8021080F867
:1014E00021109DF8031080F822109DF8041080F858
:1014F0002310DF4924208870FFF73EFF1CBD10B584
:10150000FFF726FF00280CD0DA48032101700021E4
:1015100041708170C170D64904208870BDE81040C8
:101520002AE710BD10B5FFF713FF002810D0D148EF
:1015300000210622017042708170C17001714171F9
:101540008171C171CA4908208870BDE8104013E755
:1015500010BD10B5FFF7FCFE002815D0C44AC548E1
:10156000116A491E0B0E03700B0C43700B0A83703B
:10157000C17000210171417102238371C171082082
:101580009070BDE81040F7E610BD10B5FFF7E0FE23
:10159000002819D0B7480021B54B01704170817007
:1015A0000822C2701A6A140E0471140C4471140AD1
:1015B0008471C2710222027241728272C1720C2065
:1015C0009870BDE81040D7E610BD2DE9F041A84D58
:1015D000A84C0021A8784034A64A02E0535C63542A
:1015E000491C03468142F9D31F2B72D12068A249BE
:1015F00088426ED19F4E60685F364FF00108706080
:10160000A068B060607B18B9A07B08B1102802D92F
:1016100086F80C8059E0E07B1E28F9D00FDC1228F8
:101620002ED005DC48B30328F2D1BDE8F041CFE667
:101630001528EDD01A28EBD1BDE8F0415FE702276D
:101640002A2828D010DC23281DD025281ED02828A1
:10165000DED1FFF75AFE002826D0207B000618D5E1
:101660006F70BDE8F04156E52F281ED05528CFD029
:101670005A28CDD1BDE8F04154E7BDE8F04194E6E9
:10168000BDE8F041CAE6BDE8F0417EE7BDE8F041C3
:101690005FE7022016E0FFF738FE002804D0207B29
:1016A00000060ED485F801802DE6FFF72EFE0028F7
:1016B000FAD0207B000604D485F80180C5F8288084
:1016C00021E6822001F05AF93773BDE8F0414DE57B
:1016D000FFE7822001F052F9022001F04FF90620C5
:1016E000687010E6624810B54178022908D00329D5
:1016F0000ED004290FD0052901D10021417010BD61
:101700005C484030C07B2828F9D1BDE8104002E594
:10171000BDE810402AE5822001F030F9F8E710B565
:101720005449022001F03EF951498870487858B177
:1017300001280CD0022001F021F94E4902205F312E
:101740000873BDE8104011E5BDE810403DE7494889
:101750004030C07B2A2804D02F2805D1BDE8104096
:1017600098E5BDE810406CE510BDFFB502460020CD
:1017700002EB420501464FF440566C4603AA6B1833
:1017800044F82130B34202DD002004B0F0BD3B4FED
:1017900007EB6307DB073F78575401D03B095354ED
:1017A000535C8F0003F00F035354BB40491C184493
:1017B0000329E4DBE9E7F0B50646002003460246CC
:1017C0002E4C4FF4007700E05B1CF55C45B102EB5A
:1017D000030CA4440CF5805C9CF800C8AC45F3D025
:1017E000032B40D302F5C0502044037F457FC67FC2
:1017F00003EB0523857F2D0405EB06652B4451EA99
:1018000003052CD021B91A49496840318B4226D8AA
:10181000184B00216C335518254405F5805595F873
:1018200000585D54491C0C29F5D3817EC27E01EB22
:101830000221027D407D120402EB00600C1820465C
:10184000FFF793FF40F6F57502E000BFFFF78DFF4D
:10185000C11EA942FAD3A0F57061FF3901D0002062
:10186000F0BD2046F0BD2032BA42AED3F0BD00003C
:1018700090C00720ADE2072055534243ADC8072072
:101880005C4A10475C4A34231360C2E901015B489B
:101890004FF47A710068B0FBF1F0D06002F11401EE
:1018A0001046EDE7544A32231360C2E90101534860
:1018B0004FF47A710068B0FBF1F0D06002F11401CE
:1018C0001046DDE710B572B633244B4B10C307C387
:1018D0004A484FF47A710068B0FBF1F01860191DA6
:1018E0004548FFF7CDFF62B610BD10B572B60624AD
:1018F000434900BF51F82420824212D94049783927
:1019000051F82410814207D121460846FFF7CAFF4B
:1019100021460846FFF7B6FF21460846FFF7C2FFFB
:1019200002E0641C1D2CE5D962B610BD2DE9F04122
:10193000344C236803B920602F4D0020283563689C
:1019400003E00F5C1E18401CAF559042F9D3981865
:101950004FF480766060B04218D12068FFF7C5FF71
:10196000254D1435286810B100F028F9FCE722490C
:10197000324628312068FFF7A5FF286818B100BF5C
:1019800000F01CF9FCE70020606020600020BDE84A
:10199000F08172B61C491D4A01401160FEF7A0BBE0
:1019A00010B546F204410023098846F23840A1F5FB
:1019B0001942993A1BD001684FF4F420814200D8B3
:1019C00001B901464FF4C042541E1046214401E0C3
:1019D00010C823448842FBD94BB100204FF40021AA
:1019E00008CA8A421844FBD308B1002010BD012068
:1019F00010BD0000F11FFF1F28E30720F4C00720DF
:101A0000D45B0000C8C0072080FFFF1F08ED00E086
:101A1000002070477649C20702D04FF480028A61E5
:101A2000800702D54FF4001088610020704770498C
:101A3000C20702D04FF48002CA61800702D54FF47A
:101A40000010C8610020704701460020684ACB079B
:101A500003D053695B0200D50120890704D5516981
:101A6000890201D540F00200704710B50446FFF727
:101A7000EBFF0346FFF7DBFF24EA0300FFF7CAFF93
:101A8000002010BD70B55B4B50B15968042403258C
:101A90000226052907D2DFE801F0072B4A718E00E4
:101AA00000205860986070BD042807D0052809D030
:101AB000012402287AD0012808D00FE00320FFF784
:101AC000B6FF46E0BDE870400120B0E70320FFF715
:101AD000AEFF0BE0FFF79EFF5C6070BD0E28FCD1EF
:101AE0000320FFF7A4FF0220FFF794FF0120F1E796
:101AF00006280AD0032810D00A2813D0092811D0AC
:101B00000D280FD00C28D9D070BD0320FFF78FFF10
:101B10000220FFF77FFF5E6070BD0320FFF787FFA5
:101B2000012027E00320FFF782FF022012E00628B1
:101B300013D00A281AD00928C8D00C28BED00D28E6
:101B4000F0D00F28E8D10320FFF771FF0220FFF744
:101B500061FF0120BDE870405CE7986810F01F0F3E
:101B600000F101009860D7D102201BE00320FFF7AD
:101B70005EFF0220FFF74EFF5D6070BD072806D0B4
:101B80000A289BD00B2811D009289FD070BD0220B5
:101B9000FFF74DFF986810F03F0F00F101009860CB
:101BA000F4D10120BDE870405FE7FFE70320FFF7B5
:101BB0003EFF02208EE70628A7D08FE770B50E4EB5
:101BC0000E4D00240120FFF750FFA868A968091AEC
:101BD000B142FBD3641CE4B20A2CF3D30120FFF71B
:101BE00019FFA8680649AA68121A8A42FBD370BD79
:101BF00000C00920E8C00720A086010000000940BD
:101C000040420F004E4810B52021C0F8A01100BF7F
:101C1000D0F8A0114906FBD50321C0F80411494AA8
:101C2000C0F8A8214FF48062C0F8AC210122C0F8AE
:101C30000C210B23C0F88430C0F88020AA22C0F801
:101C40008C205523C0F88C30D0F888406401FBD537
:101C5000C0F88010C0F88C20C0F88C300521C0F886
:101C600008113949C0F8C4100021C0F8C811D0F8D3
:101C700088106FEA11618A073449D0F80C2102F00C
:101C8000030207D07AB3012A44D0022A47D0032A9C
:101C90004ED13AE02AB1012A13D0022A24D0032AD5
:101CA00046D1D0F88820D0F80431C2F30742DBB225
:101CB000521C5B1C5A43D0F88830254CC3F30E03EA
:101CC0000EE0D0F88820D0F80431C2F30742DBB22E
:101CD000521C5B1C5A43D0F888301E4CC3F30E03D1
:101CE0005B1C634321E010E0D0F88820D0F8043179
:101CF000C2F30742DBB2521C5B1C5A43D0F8883057
:101D00004FF47A44C3F30E03EAE7D0F80421124BF0
:101D1000D2B209E0D0F80421104BD2B204E0D0F8DE
:101D200004214FF4FA43D2B2521CB3FBF2F20A6020
:101D3000016821F4704141F44051016010BD000080
:101D400000C00F4040101103DE97E8A7F4C0072041
:101D500000127A0000366E0100093D00001BB7003A
:101D6000B44810B500218162816821F003018160CF
:101D7000816C41F003018164AF490122CA630B6A9F
:101D800043F001030B62836823F440238360836C78
:101D900023F4402343F4002383644315CB630B6A8D
:101DA00043F400730B62836823F440338360836CD5
:101DB00043F44033836483158B630B6A43F480736D
:101DC0000B62036923F440030361036D23F44003B2
:101DD0000365C314CB650B6C23F400630B64436889
:101DE00023F440534360436C23F4405343F40053C3
:101DF00043649305CB610C6844F480040C60446830
:101E000024F440644460446C24F4406444F400646A
:101E1000446454058C610C6844F400140C604468FC
:101E200024F0406444F080644460446C24F04064D6
:101E300044F000644464446824F0405444F0805406
:101E40004460446C24F0405444F000544464C4683A
:101E500024F0405444F00054C460C46C44F0405436
:101E6000C464C46924F44024C461C46D24F44024CF
:101E700044F40024C4655406CC670C6E44F000742E
:101E80000C66C46844F44034C460C46C24F4403428
:101E900044F40034C464C46844F44044C460C46C72
:101EA00024F4404444F40044C464C46844F44074DA
:101EB000C460C46C24F4407444F40074C464C46802
:101EC00024F03004C460C46C24F03004C46494046E
:101ED0008C630C6A44F480240C62C46824F440547B
:101EE000C460C46C24F44054C4648B630B6A43F430
:101EF00080030B62036923F440130361036D23F431
:101F0000401303650315CB650B6C23F480630B64EE
:101F1000036923F040730361036D23F0407303658D
:101F20008314CB650B6C23F480530B64036923F09B
:101F300040630361036D23F0406343F00063036576
:101F40005303CB650B6C43F400530B64C36823F05D
:101F50000303C360C36C23F003039B1CC36413041B
:101F6000CB630B6A43F480330B62C36823F0C00376
:101F7000C360C36C23F0C00343F08003C364D30485
:101F8000CB630B6A43F400230B62C36823F00C039A
:101F9000C360C36C23F00C0343F00803C364530411
:101FA000CB630B6A43F400330B62436823F4404372
:101FB00043F480434360436C23F4404343F40043C1
:101FC0004364C36843F44023C360C36C23F44023D9
:101FD00043F40023C364036923F00C030361036D1E
:101FE00023F00C0343F0080303650223CB650B6C5D
:101FF00043F002030B64036923F030030361036DB4
:1020000023F0300343F0200303650423CB650B6CFE
:1020100043F004030B64036923F003030361036DBE
:1020200043F003030365CA65086C40F001000864CF
:1020300010BD000000C0024000C009204F49002030
:102040000867C86010224A618861C022CA634C498F
:102050008A684C49C1E900204B4908604B49086037
:1020600078464B490860002070472DE9F04341F263
:1020700088320023444C454D454E904208D8642890
:1020800000D228B942F21072914201D8052907D234
:10209000862020602B60784630608620BDE8F08383
:1020A000DFF8DC90D9F80820DFF8D880D8F8007085
:1020B000D21BD8F8047007EB470CCCEBC717B2EB78
:1020C000C70F06D2052020602B60784630600520BF
:1020D000E4E72A4A02275760D2F83CC00CF0FD0C16
:1020E000C2F83CC040B1DFF8ACC0BCFBF0F040101F
:1020F000D061576001205060D9F80800C8E900019C
:1021000023602B60784630600020C7E770B51D4C17
:1021100000250E466560FFF7A8FF1B49000601D5A4
:10212000086870BD164B06EB46022068C2EBC6126B
:102130009E68361AB6EBC20FFAD3104802224260EC
:10214000C26B02F0FD02C2636560E9E70C4880687B
:102150000C490A68801A4A6802EB4203C3EBC212B8
:10216000B0EBC20F08D3054802224260C26B02F0F6
:10217000FD02C263002048607047000000800040FC
:1021800000000940F8C0072084C0072088C007204D
:102190008CC0072080A8120108B501226946274893
:1021A000FEF78DF89DF8000008BD01B501226946D3
:1021B0002248FEF78FF808BD21484FF4FA634188A2
:1021C000994201D2491C41801E49496D0A054FF0D0
:1021D00000010BD48180027812B94278521C4270FF
:1021E0004278022A00D1417001210EE082889A4291
:1021F00001D2521C82804288B2F5FA7F03D88288CD
:10220000B2F5E17F00D1417041800170704710B597
:10221000FFF7C2FF0B49422808D0502809D05228A6
:102220000BD0486D000508D4422003E0486D00053E
:1022300003D54420BDE81040B7E710BD28000020BA
:1022400000C1072000C00920FA4800214FF0011208
:10225000818001704170C0E902217047F5491C314D
:10226000002000F09FBB10B5F24C1434A288402A25
:1022700000D940228020216800F0C5FB216801447C
:102280002160A188081AA08010BD10B5E94C00207B
:102290001434216800F086FB216801442160A18884
:1022A000081AA08010BD00221146802000F0ABBBB0
:1022B000E149002000F076BB70B5DE48DD4D1C30F2
:1022C00005F11405007810F01F040AD0D949DA4B43
:1022D00001F11C004A780079012C06D0022C26D18D
:1022E00009E0D448001D28601DE002B389788842C7
:1022F0001DD2002015E000F08F04200605D504F063
:102300000F064FF48030B04001E00120A0400AB930
:1023100022070CD18A68024209D0C9680142E8D07C
:10232000012018802B60FFF79EFF012070BD002068
:1023300070BD024670B5BF48BE4C1C30017811F02C
:102340001F030146498804D0012B29D0022B27D135
:1023500011E0012924D132B1012000F0BDFAA0889A
:1023600040F0020005E0002000F0B6FAA08820F05E
:102370000200A08021E0007900F08F00030605D55F
:1023800000F00F034FF480359D4001E001258540AA
:1023900063782BB1030703D0A3682B4200D009B1A7
:1023A000002070BD22B100F0E9FAE068284303E0A4
:1023B00000F0EEFAE068A843E060012070BD9D489F
:1023C00010B51C30007810F01F0F9A4800F11C0067
:1023D000C0782AD197491431012807D001F10802A9
:1023E0000228937806D003281FD112E09348086092
:1023F000122012E09248002204E004780CB14488D4
:102400002044521C9342F8D1027872B1086040888F
:1024100003E08C481844086000788A88824200D91A
:102420008880FFF720FF012010BD002010BD2DE99E
:10243000F84F804F00201C370090B8787D4E4FF049
:1024400000094FF0010A4FF4803B00286BD07C4C10
:1024500065E06078022804D0042841D005285CD1CA
:1024600041E06179B878814238D170702079B070DC
:102470007049002011F1100101F80090401C04285F
:10248000FAD301254FEA06080AFA05F0D8F8081031
:10249000084202D0284600F05DFAD8F808100BFA7E
:1024A00005F0084203D045F0800000F053FA6D1C9F
:1024B000102DE9D34FF00110C8E90209012000F006
:1024C0000CFAE0794006B8F8040002D540F00100AB
:1024D00001E020F00100A8F804001EE060881DE083
:1024E000E078009019E00098B8B9A07800F08F0566
:1024F000280604D505F00F010BFA01F001E00AFAF5
:1025000005F0B16801432046B16000F0FCF92846AF
:1025100000F016FA284600F027FA207804442078C4
:10252000002896D11FE086F8019001245546D84630
:10253000B16805FA04F0084202D0204600F00AFA19
:10254000B16808FA04F0084203D044F0800000F0BB
:1025500001FA641C102CEBD34FF00110C6E90209FC
:10256000002000F0BAF9B8787178884202D10120D1
:10257000BDE8F88F0020FBE72DE9FC5F2D4D00271B
:102580003E466878BB46B846002871D0BA462C4C07
:1025900005F11C0968E06078022804D0042808D0FE
:1025A00005285FD119E06079697888425AD060883F
:1025B00059E0A77899F80410E6784FF00008B9427E
:1025C00050D199F80200B0424CD11A484FF0010A9C
:1025D000103010F807B0C65544E099F80410B9421D
:1025E00040D1A17801F08F010191090605D501992B
:1025F00001F00F024FF4803101E0019A0121914076
:10260000009199F80200B0421ED1A8680843A86062
:10261000E968009881432046E96000F074F9019868
:1026200000F08EF9019800F09FF9009948EA01083E
:1026300018E0000008C1072050E407204C5C0000AF
:102640005E5C00007F5C00005E450BD118EA010F64
:1026500008D1A8688843A860E8688843E8600198C2
:1026600000F078F9207804442078002893D150466F
:10267000BDE8FC9F2DE9F041494C0027A4F1080674
:102680002178A4F11C05082863D2DFE800F0620479
:10269000647262628381FFF7E1FD2078C00900F077
:1026A0004EF9E088B0802078C0F34111F1BB617829
:1026B0000C294AD2DFE801F00609490B49101A1D1E
:1026C0001F253142FFF7F8FD4DE0002000E001201A
:1026D000FFF72FFE50B306E010F01F0F35D1A078A2
:1026E00040F080002870BDE8F041DCE5FFF767FEB0
:1026F00039E000202AE010F01F0F26D128481B38AF
:102700001AE010F01F0F20D1FFF791FE70B1FFF714
:10271000CAFDBDE8F04100F072BA00F01F000128C8
:1027200013D1687810B12079A97800E00DE08842D3
:102730000BD21B490C39084430601CE000F01F002C
:10274000012802D1FFF718FFC4E7802000F016F936
:10275000B780BDE8F081080608D4B0880028F8D01A
:10276000FFF793FDB0880028EFD0F2E7BDE8F04115
:102770009EE5080602D5BDE8F04174E5287801061B
:10278000E7D500F07F002870BDE8F04100F054B8B4
:10279000802000E00020BDE8F04100F0F9B8000022
:1027A00024C1072001460007C00E090600D5401CC1
:1027B0007047DA491022C1F80822C1F8100200BFA0
:1027C000D1F80002C006FBD57047D44A1023C2F8E6
:1027D0000832C2F8100200BFD2F80002C006FBD5D2
:1027E000C2F80832C2F81012D2F80002C006FBD5B7
:1027F0007047CA493022C1F80822C1F8100200BF50
:10280000D1F800028006FBD5D1F81402704710B54C
:10281000040001D0012000E000204FF4807141EA63
:102820000041BF48FFF7D1FFBE494FF000700CB127
:10283000886710BDC86710BD30B5BB49BB4D41EAC4
:10284000004421462846FFF7C0FF21462846BDE840
:102850003040BAE7B1480021C0F848124021C0F822
:102860004C120122C0F84822C0F84C12D0F80012D5
:10287000C905FBD54FF0FF31C0F83812C0F834124B
:10288000C0F808120C21C0F804127047A84800B51F
:10289000C16821F0405141F00051C160C16C41F06C
:1028A0004051C164A3491A200860091D0A6830EA32
:1028B0000202FBD14FF0E0214FF08070C1F880029E
:1028C0009D4B202283F80024C1F80001FFF7C2FFCE
:1028D00000205DF804EBAFE7704710B500B10120B0
:1028E0004FF4807444EA00419448FFF76EFF8B4830
:1028F0000321C0F8441200BFD0F80012C905FBD56F
:10290000C0F8084210BD10B502468078FFF74AFFB4
:102910008249D1F84432012484402343C1F844322F
:10292000C1F848029088C1F84C0200BFD1F80002FB
:10293000C005FBD54FF48070C1F8080210BD704788
:1029400000B5FFF72FFF7E495DF804EB41EA004038
:1029500089133AE700B5FFF725FF79495DF804EBE5
:1029600041EA0040774930E700B5FFF71BFF7449A3
:102970005DF804EB41EA0040891326E700B5FFF754
:1029800011FF6F495DF804EB41EA00406E491CE716
:1029900000B5FFF707FF6A495DF804EB41EA004024
:1029A000891312E700F00F02012370B503EB8203D5
:1029B0005A4AC2F8283200BFD2F820321C05FBD593
:1029C000C3F309030024DD1C05E000BFD2F8186240
:1029D00041F8046B641CB4EB950FF7D30021C2F8E7
:1029E000281241F24821C140C9070AD1FFF7DAFE97
:1029F0004FF4A06141EA0040FFF7DBFE5348FFF7C8
:102A0000D8FE184670BD70B513460546434C00F01D
:102A10000F00022202EB8000C4F82802C4F824321E
:102A20000020DA1C05E000BF51F8046BC4F81C62FA
:102A3000401CB0EB920FF7D30020C4F828022846C0
:102A4000FFF7B0FE4FF4A06141EA0040FFF7B1FE8E
:102A50003F48FFF7AEFE184670BD2DE9F0412F4DFF
:102A6000D5F80032C5F80832180721D52C48FFF7F1
:102A7000A0FE3848FFF7BDFEC10605D5FFF7EAFE08
:102A8000BDE8F04100F0ACB8810705D5BDE8F041E4
:102A900000F0010000F09EB8010709D5400703D5FA
:102AA000BDE8F04100F0A3B8BDE8F04100F0A6B8E1
:102AB000294E58074FF001071CD4BDE8F0810024CF
:102AC000D5F8302207FA04F10A4210D06008C5F8A0
:102AD000381200BFD5F800128906FBD5D5F81412BC
:102AE000E2070CD056F8201009B103208847641C77
:102AF000202CE5D3D5F830020028E0D1DDE73CB941
:102B0000490705D5316819B1012088470124D7E765
:102B100056F820100029EAD00220E7E700C0005054
:102B20000005FE0000C00920000180000005D00063
:102B300000C00240F4CF005018E000E00005D800CB
:102B40000005400000012000000101000005F20026
:102B50000005FA000002FE00F05C00002DE9F041E3
:102B60002C4C00250127A07850B32B4E012811D002
:102B700002280DD1B0686168401A2849884216D3EE
:102B80002748406B400012D50120FFF740FEA5709A
:102B9000BDE8F081B0686168401A22498842F7D3E5
:102BA0000020FFF734FEB06860600220A07025703E
:102BB00060780028ECD10C20FEF764FF6770E7E72F
:102BC00020780028E4D165702770BDE8F0410D2021
:102BD000FEF758BF002802D10E49012088707047C7
:102BE00010B5FFF731FB0B490020887010BD094874
:102BF00001218170084989684160704770477047BA
:102C0000022803D0032803D1FEF76CBDFEF787BD71
:102C1000704700002CC1072000000940A086010079
:102C200000C0092040420F002DE9F047FC4E8046CD
:102C30004FF080773068BC11FA4DB84249D100BFDF
:102C400000BF00BF00BF00BF00BF00BF00BF00BF8C
:102C500000BF00BF00BF00BF00BF00BF00BF00BF7C
:102C600000BF00BF00BF00BF00BF00BF00BF00BF6C
:102C700000BF00BF00BF00BF00BF00BF00BFEC63CC
:102C80001520FDF787FB0020FDF784FB00F0FF090E
:102C9000AC6300BF00BF00BF00BF00BF00BF00BFEC
:102CA00000BF00BF00BF00BF00BF00BF00BF00BF2C
:102CB00000BF00BF00BF00BF00BF00BF00BF00BF1C
:102CC00000BF00BF00BF00BF00BF00BF00BF00BF0C
:102CD00000BF00BF00BF00BF00BF00BF00BF00BFFC
:102CE00000BF00BF00BF00BF00BF00BF00BF00BFEC
:102CF00000BF00BF00BF00BF00BF00BF00BF00BFDC
:102D000000BF00BF00BF00BF00BF00BF00BF00BFCB
:102D100000BFEC630620FDF73DFBAC6300BF00BFC6
:102D200000BF00BF00BF00BF00BF00BF00BF00BFAB
:102D300000BF00BF00BF00BF00BF00BF00BF00BF9B
:102D400000BF00BF00BF00BF00BF00BF00BF00BF8B
:102D500000BF00BF00BF00BF00BF00BF00BF00BF7B
:102D600000BF00BF00BF00BF00BF00BF00BF00BF6B
:102D700000BF00BF00BF00BF00BF00BF00BF00BF5B
:102D800000BF00BF00BF00BF00BF00BF00BF00BF4B
:102D900000BF00BF00BF00BF00BF00BFEC63012049
:102DA000FDF7F8FA4FEA8800FDF7F4FA3068B84208
:102DB00002D14846FDF7EEFAAC6300BF00BF00BF8A
:102DC00000BF00BF00BF00BF00BF00BF00BF00BF0B
:102DD00000BF00BF00BF00BF00BF00BF00BF00BFFB
:102DE00000BF00BF00BF00BF00BF00BF00BF00BFEB
:102DF00000BF00BF00BF00BF00BFBDE8F0872DE9E6
:102E0000FC5F8846044601A9874800F078FB874D9F
:102E1000874E884FF0BB03208DF8000020098DF805
:102E2000010020018DF802004FF000098DF8039099
:102E300000BF00BF00BF00BF00BF00BF00BF00BF9A
:102E400000BF00BF00BF00BF00BF00BF00BF00BF8A
:102E500000BF00BF00BF00BF00BF00BF00BF00BF7A
:102E600000BF00BF00BF00BF00BF00BF00BF00BF6A
:102E7000DFF8B0B14FF4802ACBF83CA004216846BB
:102E8000FDF78FFA00240020FDF784FAC0B28DF818
:102E9000040000E003E018F80410884208D0822003
:102EA000286022203060784638608220BDE8FC9F90
:102EB000641CB4F5805FE6D3CBF838A000BF00BF38
:102EC00000BF00BF00BF00BF00BF00BF00BF00BF0A
:102ED00000BF00BF00BF00BF00BF00BF00BF00BFFA
:102EE00000BF00BF00BF00BF00BF00BF00BF00BFEA
:102EF00000BF00BF00BF00BF00BF00BFC5F800900B
:102F0000C6F80090784638600020CFE72DE9F047FA
:102F10004FF0000900BF00BF00BF00BF00BF00BFEF
:102F200000BF00BF00BF00BF00BF00BF00BF00BFA9
:102F300000BF00BF00BF00BF00BF00BF00BF00BF99
:102F400000BF00BF00BF00BF00BF00BF00BF00BF89
:102F500000BF00BF334F4FF48026FE639F20FDF774
:102F600019FA0020FDF716FAC4B20020FDF712FA94
:102F7000C5B20020FDF70EFAC1B2BE6300BF00BFAC
:102F800000BF00BF00BF00BF00BF00BF00BF00BF49
:102F900000BF00BF00BF00BF00BF00BF00BF00BF39
:102FA00000BF00BF00BF00BF00BF00BF00BF00BF29
:102FB00000BF00BF00BF00BF00BF00BF1B4E1C4FC3
:102FC000DFF87080C22C08D0C82C09D01F2C0AD082
:102FD0001C2C0BD09D2C0CD00DE0202D14D00AE021
:102FE000402D11D007E0322D0ED004E0702D0BD013
:102FF00001E0602D08D082203060212038607946C1
:10300000C8F800108220F8E605481439052920D2B6
:10301000DFE801F0031216191C004FF480110DE0D7
:1030200034C1072000C00920E093040084C00720B9
:1030300088C007208CC007204FF4001101600AE00F
:103040004FF48001FAE74FF40001F7E74FF0807189
:10305000F4E7C0F800900020FFF7E6FDC6F8009006
:10306000C7F800907946C8F800100020C5E62DE9A1
:10307000F34FC3B0804600244FF0820AFE4DFF4E4E
:10308000FF4F4FF0210BA14641A9FE4800F037FA4F
:1030900000286CD100F0A0FA02208DF800004FEA61
:1030A00018108DF8010004EB08108DF80200449808
:1030B0008DF8039000EB04214FF4807201A8FDF716
:1030C000A2F900BF00BF00BF00BF00BF00BF00BF2C
:1030D00000BF00BF00BF00BF00BF00BF00BF00BFF8
:1030E00000BF00BF00BF00BF00BF00BF00BF00BFE8
:1030F00000BF00BF00BF00BF00BF00BF00BF00BFD8
:1031000000BFE1494FF48020C8634FF482716846E4
:10311000FDF747F9DC494FF48020886300BF00BF0A
:1031200000BF00BF00BF00BF00BF00BF00BF00BFA7
:1031300000BF00BF00BF00BF00BF00BF00BF00BF97
:1031400000BF00BF00BF00BF00BF00BF00BF00BF87
:1031500000BF00BF00BF00BF00BF00BF641CE4B2DF
:10316000102C91D341A9C74800F0C9F948B1C5F85E
:1031700000A0C6F800B078463860822045B0BDE8AF
:10318000F08F00F073FAC5F80090C6F8009078460A
:1031900038600020F2E72DE9F04F89B0DFF8D882DF
:1031A0005FEA020B4FF0000607910FD04FF48055F5
:1031B00001462A466846FDF70FF9DDE90047284633
:1031C00002F034FC5FEA00090CD016E08621C8F852
:1031D0000010AA48092101607946A94801608620AB
:1031E00009B0CCE78221C8F80010A4482221016070
:1031F0007946A34801608220F2E7ABEB0605C7F5EC
:1032000080504FF0000AA84200D20546B5F5805F15
:1032100004D02046494600F0A7FCD8B907982A46B2
:10322000811907EB0900FDF7EEF8204600F021FCBC
:1032300080B920464946FFF71AFF58B9204649464B
:10324000FFF7DDFD78B10AF1010000F0FF0ABAF1E5
:10325000030F05D3484602F0BBFBD8F80000BFE7D8
:10326000BAF1000FE1D12E440027641C5E45C4D39F
:10327000484602F0ADFB0020C8F800007F49086016
:1032800079467F4801600020AAE72DE9FF4F8DB005
:103290000D46DDF868900026774C07935FEA090138
:1032A0003FD04FF4805701463A466846FDF794F800
:1032B000DDE900B10C913A46691C6846FDF78CF8CF
:1032C000DDE90010CDE904013A4668460F99FDF7A3
:1032D00083F8DDE9008500BFA9EB0607C5F580503E
:1032E000B84200D2074625B1D8457CD10C9885421A
:1032F00079D14FF4805002F099FB5FEA000A1BD0AD
:10330000D8454FD10C9885424CD12A464FEA083017
:10331000514600F002FB000618D5504602F058FB5B
:1033200079E086202060554809210160784654499B
:103330000860862011B022E7822020604F482221B9
:10334000016079464E4801608220F3E70598804588
:1033500009D1049901EB0030C1F58052514400F0CD
:10336000DCFA0006D9D4404600F083FB0006D4D432
:1033700007983A46811905EB0A00FDF744F8EA1967
:103380004FEA0830514601F0E0F90006C5D405992E
:10339000884533D1049800EB01300499C1F580527F
:1033A000514427E0059988450AD1049800EB013083
:1033B0000499C1F58052514600F0AFFA0006ACD432
:1033C000404600F056FB0006A7D407983A468119FC
:1033D0000F98304401F0B9F900069ED4059988454C
:1033E0000CD1049800E00DE000EB01300499C1F528
:1033F0008052514601F0A9F900068ED4504602F0E1
:10340000E7FA0AE007983A4681190F98304401F02C
:103410009CF9000601D520688CE73E44002508F1A0
:1034200001084E45FFF458AF0020206013490860A2
:1034300078461349086000207CE71448006870470C
:103440004FF4805070474FF4805070472DE9F04F93
:10345000DFF82480DFF824B089B00F0004464FF075
:10346000000633D04FF4805501462A466846FCF7E3
:10347000B3FFDDE900A10BE084C0072088C007206E
:103480008CC00720E093040000C0092034C107204D
:1034900005912A46214606A8FCF79EFFDDE9064075
:1034A0004FF00009BD1BC0F58051A94200D20D4666
:1034B00020B1544515D10599884212D1204600F01B
:1034C000D8FA00060DD5D8F8000089E68621C8F89C
:1034D00000100921CBF8001079463C480160862095
:1034E0007EE62E44641C4846BE42DBD3C8F800008A
:1034F000CBF80000794635480160002070E62DE9E0
:10350000F041334C0F460646A56806E0A068401B14
:10351000B04202D30120BDE8F081384600F003F844
:103520000028F3D1F7E770B5044600BF00BF00BF25
:1035300000BF00BF00BF00BF00BF00BF00BF00BF93
:1035400000BF00BF00BF00BF00BF00BF00BF00BF83
:1035500000BF00BF00BF00BF00BF00BF00BF00BF73
:1035600000BF00BF00BF00BF00BF1A4E4FF4802550
:10357000F5630520FCF70EFF0020FCF70BFF207021
:10358000B56300BF00BF00BF00BF00BF00BF00BFEA
:1035900000BF00BF00BF00BF00BF00BF00BF00BF33
:1035A00000BF00BF00BF00BF00BF00BF00BF00BF23
:1035B00000BF00BF00BF00BF00BF00BF00BF00BF13
:1035C00000BF207800F0010070BD00008CC0072013
:1035D0000000094000C0092070B500BF00BF00BF57
:1035E00000BF00BF00BF00BF00BF00BF00BF00BFE3
:1035F00000BF00BF00BF00BF00BF00BF00BF00BFD3
:1036000000BF00BF00BF00BF00BF00BF00BF00BFC2
:1036100000BF00BF00BF00BF00BFFE4C4FF48025BD
:10362000E5630620FCF7B6FEA56300BF00BF00BF40
:1036300000BF00BF00BF00BF00BF00BF00BF00BF92
:1036400000BF00BF00BF00BF00BF00BF00BF00BF82
:1036500000BF00BF00BF00BF00BF00BF00BF00BF72
:1036600000BF00BF00BF00BF00BF70BD70B500BF8E
:1036700000BF00BF00BF00BF00BF00BF00BF00BF52
:1036800000BF00BF00BF00BF00BF00BF00BF00BF42
:1036900000BF00BF00BF00BF00BF00BF00BF00BF32
:1036A00000BF00BF00BF00BF00BF00BF00BFD94CBC
:1036B0004FF48025E5630420FCF76CFEA56300BF92
:1036C00000BF00BF00BF00BF00BF00BF00BF00BF02
:1036D00000BF00BF00BF00BF00BF00BF00BF00BFF2
:1036E00000BF00BF00BF00BF00BF00BF00BF00BFE2
:1036F00000BF00BF00BF00BF00BF00BF00BF70BD64
:1037000070B5064600BF00BF00BF00BF00BF00BFCE
:1037100000BF00BF00BF00BF00BF00BF00BF00BFB1
:1037200000BF00BF00BF00BF00BF00BF00BF00BFA1
:1037300000BF00BF00BF00BF00BF00BF00BF00BF91
:1037400000BF00BFB34D4FF48024EC635020FCF762
:1037500021FEAC6300BF00BF00BF00BF00BF00BFC1
:1037600000BF00BF00BF00BF00BF00BF00BF00BF61
:1037700000BF00BF00BF00BF00BF00BF00BF00BF51
:1037800000BF00BF00BF00BF00BF00BF00BF00BF41
:1037900000BF00BF00BF00BF00BF00BF00BF00BF31
:1037A00000BF00BF00BF00BF00BF00BF00BF00BF21
:1037B00000BF00BF00BF00BF00BF00BF00BF00BF11
:1037C00000BF00BF00BF00BF00BF00BF00BF00BF01
:1037D00000BF00BFEC630120FCF7DCFDB000FCF78C
:1037E000D9FDAC6300BF00BF00BF00BF00BF00BF7A
:1037F00000BF00BF00BF00BF00BF00BF00BF00BFD1
:1038000000BF00BF00BF00BF00BF00BF00BF00BFC0
:1038100000BF00BF00BF00BF00BF00BF00BF00BFB0
:1038200000BF00BF70BD2DE9FE430F46044602A94C
:10383000794800F0BCFD794D794EDFF8E88148B158
:1038400082202860222030607946C8F8001082204B
:10385000BDE8FE839DF80800800701D4FFF7BCFE99
:1038600002208DF80000200C8DF80100200A8DF850
:1038700002008DF803408DF8047000BF00BF00BF48
:1038800000BF00BF00BF00BF00BF00BF00BF00BF40
:1038900000BF00BF00BF00BF00BF00BF00BF00BF30
:1038A00000BF00BF00BF00BF00BF00BF00BF00BF20
:1038B00000BF00BF00BF00BF00BF564F4FF48024C1
:1038C000FC6305216846FCF76CFDBC6300BF00BFCC
:1038D00000BF00BF00BF00BF00BF00BF00BF00BFF0
:1038E00000BF00BF00BF00BF00BF00BF00BF00BFE0
:1038F00000BF00BF00BF00BF00BF00BF00BF00BFD0
:1039000000BF00BF00BF00BF00BF00BF0020286095
:1039100030607946C8F800109AE72DE9FC5F3F4D0A
:103920003F4E404F5FEA020A8B4604464FF00008C4
:103930000DD001A9384800F03AFD80B182202860FE
:1039400021203060784638608220BDE8FC9FC5F8B1
:103950000080C6F80080784638600020F5E7032034
:103960008DF80000200C8DF80100200A8DF802006F
:103970008DF8034000BF00BF00BF00BF00BF00BF05
:1039800000BF00BF00BF00BF00BF00BF00BF00BF3F
:1039900000BF00BF00BF00BF00BF00BF00BF00BF2F
:1039A00000BF00BF00BF00BF00BF00BF00BF00BF1F
:1039B00000BF00BF174C4FF48029C4F83C9004218D
:1039C0006846FCF7EEFC51465846FCF7F6FCC4F896
:1039D000389000BF00BF00BF00BF00BF00BF00BFE6
:1039E00000BF00BF00BF00BF00BF00BF00BF00BFDF
:1039F00000BF00BF00BF00BF00BF00BF00BF00BFCF
:103A000000BF00BF00BF00BF00BF00BF00BF00BFBE
:103A100000BF9CE700C00920E093040084C0072099
:103A200088C007208CC007202DE9F05FFF4EDFF82B
:103A30000094DFF800A4150083460F464FF00008FD
:103A40000ED000240AE0395D0BEB0400FFF7EBFE1B
:103A5000000602D53068BDE8F09F641CAC42F2D38A
:103A6000C6F80080C9F800807946CAF80010002026
:103A7000F1E72DE9FC47044601A9EF4800F097FC67
:103A8000EA4DEB4EDFF8AC9348B18220286022204B
:103A900030607946C9F800108220BDE8FC879DF8A7
:103AA0000400800701D4FFF797FD20208DF8000067
:103AB00020098DF8010020018DF8020000248DF806
:103AC000034000BF00BF00BF00BF00BF00BF00BF7A
:103AD00000BF00BF00BF00BF00BF00BF00BF00BFEE
:103AE00000BF00BF00BF00BF00BF00BF00BF00BFDE
:103AF00000BF00BF00BF00BF00BF00BF00BF00BFCE
:103B000000BFDFF838834FF48027C8F83C700421E9
:103B10006846FCF746FCC8F8387000BF00BF00BF1D
:103B200000BF00BF00BF00BF00BF00BF00BF00BF9D
:103B300000BF00BF00BF00BF00BF00BF00BF00BF8D
:103B400000BF00BF00BF00BF00BF00BF00BF00BF7D
:103B500000BF00BF00BF00BF00BF2C6034607946CB
:103B6000C9F80010002098E72DE9FC478A46044672
:103B700001A9B14800F01BFCAC4DAD4EDFF8B4928A
:103B800040B182202860222030607946C9F80010B8
:103B9000822082E703208DF8000020098DF80100C3
:103BA00020018DF8020000248DF8034000BF00BF03
:103BB00000BF00BF00BF00BF00BF00BF00BF00BF0D
:103BC00000BF00BF00BF00BF00BF00BF00BF00BFFD
:103BD00000BF00BF00BF00BF00BF00BF00BF00BFED
:103BE00000BF00BF00BF00BF00BF00BFDFF84C82B6
:103BF0004FF48027C8F83C7004216846FCF7D1FBDD
:103C0000B9115046FCF7D9FBC8F8387000BF00BFA7
:103C100000BF00BF00BF00BF00BF00BF00BF00BFAC
:103C200000BF00BF00BF00BF00BF00BF00BF00BF9C
:103C300000BF00BF00BF00BF00BF00BF00BF00BF8C
:103C400000BF00BF00BF00BF00BF00BF2C603460DA
:103C50007946C9F8001000201FE72DE9F34F83B023
:103C6000044601A9744800F0A2FB704D704E714FDC
:103C70004FF0820820B100BFC5F8008021206CE021
:103C80009DF80400800701D4FFF7A6FCAD208DF855
:103C9000000020098DF8010020018DF802004FF08E
:103CA000000B8DF803B000BF00BF00BF00BF00BF16
:103CB00000BF00BF00BF00BF00BF00BF00BF00BF0C
:103CC00000BF00BF00BF00BF00BF00BF00BF00BFFC
:103CD00000BF00BF00BF00BF00BF00BF00BF00BFEC
:103CE00000BF00BF00BFDFF854914FF4802A544654
:103CF000C9F83CA004216846FCF753FB0221049854
:103D0000FCF74FFBC9F8384000BF00BF00BF00BF41
:103D100000BF00BF00BF00BF00BF00BF00BF00BFAB
:103D200000BF00BF00BF00BF00BF00BF00BF00BF9B
:103D300000BF00BF00BF00BF00BF00BF00BF00BF8B
:103D400000BF00BF00BF00BF022401A93A4800F035
:103D50002EFB48B1C5F800802220306078463860DC
:103D6000822005B0BDE8F08F00BF00BF00BF00BFDC
:103D700000BF00BF00BF00BF00BF00BF00BF00BF4B
:103D800000BF00BF00BF00BF00BF00BF00BF00BF3B
:103D900000BF00BF00BF00BF00BF00BF00BF00BF2B
:103DA00000BF00BF00BF00BFC9F83CA0AD20FCF7BA
:103DB000F1FA049802212044FCF7F3FAC9F838A07C
:103DC00000BF00BF00BF00BF00BF00BF00BF00BFFB
:103DD00000BF00BF00BF00BF00BF00BF00BF00BFEB
:103DE00000BF00BF00BF00BF00BF00BF00BF00BFDB
:103DF00000BF00BF00BF00BF00BF00BF00BF00BFCB
:103E0000A41CA4B2B4F5805F9FD301A90A4800F0B6
:103E1000CEFA00287FF430AFFFF728FCC5F800B0D9
:103E2000C6F800B07846386000209AE784C00720C2
:103E300088C007208CC00720E093040000C0092040
:103E400070B5FD4DFD4EFE4C2AB1FFF766FD000634
:103E500009D5206870BD862020600920286078463A
:103E60003060862070BD0020206028607846306079
:103E7000002070BD2DE9F04F89B0DFF8C483DFF872
:103E8000B8B35FEA02094FF0000607910FD04FF474
:103E9000805501462A466846FCF79EFADDE9004750
:103EA000284601F0C3FD5FEA000A0CD016E0862127
:103EB000C8F800100921CBF800107946DF480160EE
:103EC000862009B04EE78221C8F800102221CBF8E5
:103ED00000107946D94801608220F2E7A9EB060577
:103EE000C7F58050A84200D20546B5F5805F04D0E2
:103EF00020465146FFF738FE80B92046FFF7B9FD4E
:103F000060B907982A46811907EB0A00FCF77BFA8B
:103F10002E4420465146FFF7A0FE28B1504601F03E
:103F200057FDD8F80000CCE70027641C4E45D5D3D8
:103F3000504601F04DFD0020C8F80000CBF800000D
:103F40007946BE4801600020BBE72DE9FF4F8DB0E8
:103F50000D46DDF868900026B94C07935FEA090129
:103F60003FD04FF4805701463A466846FCF734FA92
:103F7000DDE900B10C913A46691C6846FCF72CFA61
:103F8000DDE90010CDE904013A4668460F99FCF7D7
:103F900023FADDE9008500BFA9EB0607C5F58050CF
:103FA000B84200D2074625B1D8457CD10C9885424D
:103FB00079D14FF4805001F039FD5FEA000A1BD03F
:103FC000D8454FD10C9885424CD12A464FEA08304B
:103FD0005146FFF7A2FC000618D5504601F0F8FC48
:103FE00079E0862020609448092101607846934951
:103FF0000860862011B0B5E6822020608E4822211C
:10400000016079468D4801608220F3E7059880457C
:1040100009D1049901EB0030C1F580525144FFF7FA
:104020007CFC0006D9D44046FFF723FD0006D4D41B
:1040300007983A46811905EB0A00FCF7E4F9EA19FA
:104040004FEA08305146FFF7EFFC0006C5D405994A
:10405000884533D1049800EB01300499C1F58052B2
:10406000514427E0059988450AD1049800EB0130B6
:104070000499C1F580525146FFF74FFC0006ACD4BD
:104080004046FFF7F6FC0006A7D407983A46811988
:104090000F983044FFF7C8FC00069ED40599884568
:1040A0000CD1049800E00DE000EB01300499C1F55B
:1040B00080525146FFF7B8FC00068ED4504601F0FE
:1040C00087FC0AE007983A4681190F983044FFF7B9
:1040D000ABFC000601D520688CE73E44002508F1C2
:1040E00001084E45FFF458AF002020605249086097
:1040F00078465249086000207CE72DE9F0474FF0F0
:10410000000900BF00BF00BF00BF00BF00BF00BF6D
:1041100000BF00BF00BF00BF00BF00BF00BF00BFA7
:1041200000BF00BF00BF00BF00BF00BF00BF00BF97
:1041300000BF00BF00BF00BF00BF00BF00BF00BF87
:1041400000BF404E4FF48025F5639F20FCF722F915
:104150000020FCF71FF900F0FF080020FCF71AF917
:10416000C4B20020FCF716F9C1B2B56300BF00BFAE
:1041700000BF00BF00BF00BF00BF00BF00BF00BF47
:1041800000BF00BF00BF00BF00BF00BF00BF00BF37
:1041900000BF00BF00BF00BF00BF00BF00BF00BF27
:1041A00000BF00BF00BF00BF00BF00BF244D224EB4
:1041B000224FB8F1BF0F03D1252C0AD0262C08D0EE
:1041C0008220286021203060784638608220BDE857
:1041D000F0871D48412912D04FF48002422912D0A5
:1041E0004A2910D0C0F800900020FFF789FAC5F8DE
:1041F0000090C6F80090784638600020E7E74FF45A
:1042000000110160F0E70260EEE72DE9F84F694622
:104210000E4800F0CCF88227094C074D074E4FF0AE
:10422000220A002862D19DF80000800701D4FFF720
:10423000D3F900BF00BF0BE088C007208CC0072067
:1042400084C0072000C0092038C10720E093040083
:1042500000BF00BF00BF00BF00BF00BF00BF00BF66
:1042600000BF00BF00BF00BF00BF00BF00BF00BF56
:1042700000BF00BF00BF00BF00BF00BF00BF00BF46
:1042800000BF00BF00BF00BF00BF00BFDFF8EC9160
:104290004FF48028C9F83C806020FCF77BF8C9F80F
:1042A000388000BF00BF00BF00BF00BF00BF00BF1D
:1042B00000BF00BF00BF00BF00BF00BF00BF00BF06
:1042C00000BF00BF00BF00BF00BF00BF00BF00BFF6
:1042D00000BF00BF00BF00BF00BF00BF00BF00BFE6
:1042E00000BF6946664800F062F838B12760C5F83B
:1042F00000A0784630608220BDE8F88F0020206062
:104300002860784630600020F6E75E480068704715
:104310004FF4805070472DE9F04FDFF86C81DFF8E3
:104320006CB189B00F0004464FF0000626D04FF460
:10433000805501462A466846FCF74EF8DDE900A1A3
:1043400005912A46214606A8FCF746F8DDE9064015
:104350004FF00009BD1BC0F58051A94200D20D46A7
:1043600020B1544515D10599884212D12046FFF756
:1043700080FB00060DD5D8F80000A2E58621C8F81C
:1043800000100921CBF800107946414801608620D1
:1043900097E52E44641C4846BE42DBD3C8F80000B3
:1043A000CBF8000079463A480160002089E52DE904
:1043B000F041384C0F460646A56806E0A068401B51
:1043C000B04202D30120BDE8F081384600F003F886
:1043D0000028F3D1F7E770B5044600BF00BF00BF67
:1043E00000BF00BF00BF00BF00BF00BF00BF00BFD5
:1043F00000BF00BF00BF00BF00BF00BF00BF00BFC5
:1044000000BF00BF00BF00BF00BF00BF00BF00BFB4
:1044100000BF00BF00BF00BF00BF184E4FF4802593
:10442000F5630520FBF7B6FF0020FBF7B3FF207014
:10443000B56300BF00BF00BF00BF00BF00BF00BF2B
:1044400000BF00BF00BF00BF00BF00BF00BF00BF74
:1044500000BF00BF00BF00BF00BF00BF00BF00BF64
:1044600000BF00BF00BF00BF00BF00BF00BF00BF54
:1044700000BF207800F0010070BD000000C00920DE
:1044800080C3C90138C1072084C0072088C0072025
:104490008CC00720000009402DE9FF4703A9FE4812
:1044A00000F063FBFD4DFE4EDFF8F89350B1822023
:1044B0002860212030607946C9F80010822004B0BD
:1044C000BDE8F0879DF80C00800701D4FFF784F861
:1044D00042208DF800000024CDF80140CDF80540C1
:1044E000ADF8094000BF00BF00BF00BF00BF00BF64
:1044F00000BF00BF00BF00BF00BF00BF00BF00BFC4
:1045000000BF00BF00BF00BF00BF00BF00BF00BFB3
:1045100000BF00BF00BF00BF00BF00BF00BF00BFA3
:1045200000BF00BFDFF880834FF48027C8F83C70DD
:104530000B216846FBF735FFC8F8387000BF00BF95
:1045400000BF00BF00BF00BF00BF00BF00BF00BF73
:1045500000BF00BF00BF00BF00BF00BF00BF00BF63
:1045600000BF00BF00BF00BF00BF00BF00BF00BF53
:1045700000BF00BF00BF00BF00BF00BF2C603460A1
:104580007946C9F80010002099E72DE9F34F85B06E
:10459000044603A9C04800F0E8FAC04DC04EC14F20
:1045A0004FF0820B18B1C5F800B0212060E0FFF792
:1045B00013F842208DF800004FF0000ACDF801A05A
:1045C000CDF805A0ADF809A000BF00BF00BF00BF37
:1045D00000BF00BF00BF00BF00BF00BF00BF00BFE3
:1045E00000BF00BF00BF00BF00BF00BF00BF00BFD3
:1045F00000BF00BF00BF00BF00BF00BF00BF00BFC3
:1046000000BF00BF00BF00BFDFF89C924FF48028BE
:10461000C9F83C800B216846FBF7C3FEC9F8388017
:1046200000BF00BF00BF00BF00BF00BF00BF00BF92
:1046300000BF00BF00BF00BF00BF00BF00BF00BF82
:1046400000BF00BF00BF00BF00BF00BF00BF00BF72
:1046500000BF00BF00BF00BF00BF00BF00BF00BF62
:1046600003A98D4800F081FA48B1C5F800B02220B6
:10467000306078463860822007B0BDE8F08F9DF842
:104680000C00800701D4FEF7A7FF02208DF8000080
:10469000200C8DF80100200A8DF8020006988DF894
:1046A00003408DF8040000BF00BF00BF00BF00BF83
:1046B00000BF00BF00BF00BF00BF00BF00BF00BF02
:1046C00000BF00BF00BF00BF00BF00BF00BF00BFF2
:1046D00000BF00BF00BF00BF00BF00BF00BF00BFE2
:1046E00000BF00BF00BF4446C846C9F83C40052192
:1046F0006846FBF756FEC8F8384000BF00BF00BF51
:1047000000BF00BF00BF00BF00BF00BF00BF00BFB1
:1047100000BF00BF00BF00BF00BF00BF00BF00BFA1
:1047200000BF00BF00BF00BF00BF00BF00BF00BF91
:1047300000BF00BF00BF00BF00BFC5F800A0C6F8A3
:1047400000A078463860002096E72DE9F05F534ED0
:10475000DFF84C91DFF84CA1150083460F464FF06F
:1047600000080ED000240AE0395D0BEB0400FFF7CF
:104770000CFF000602D53068BDE8F09F641CAC4217
:10478000F2D3C6F80080C9F800807946CAF8001054
:104790000020F1E72DE9F34F0024404D404E414FFA
:1047A000C3B080464FF0820A4FF0210BA14641A9C9
:1047B000394800F0DAF900287CD19DF8040180071F
:1047C00001D4FEF709FF02208DF800004FEA18100F
:1047D0008DF8010004EB08108DF8020044988DF864
:1047E000039000EB04214FF4807201A8FBF70BFE4D
:1047F00000BF00BF00BF00BF00BF00BF00BF00BFC1
:1048000000BF00BF00BF00BF00BF00BF00BF00BFB0
:1048100000BF00BF00BF00BF00BF00BF00BF00BFA0
:1048200000BF00BF00BF00BF00BF00BF00BF00BF90
:104830001D494FF48020C8634FF482716846FBF72E
:10484000B0FD19494FF48020886300BF00BF00BF4E
:1048500000BF00BF00BF00BF00BF00BF00BF00BF60
:1048600000BF00BF00BF00BF00BF00BF00BF00BF50
:1048700000BF00BF00BF00BF00BF00BF00BF00BF40
:1048800000BF00BF00BF00BF00BF641CE4B2102C1B
:104890008DD341A900480AE0E093040084C00720BA
:1048A00088C007208CC0072000C0092002E000F06B
:1048B0005CF940B1C5F800A0C6F800B07846386091
:1048C000822045B0D9E6FEF7D1FEC5F80090C6F8C3
:1048D0000090784638600020F3E72DE9F04F89B06A
:1048E000DFF85483DFF854B35FEA02094FF00006A3
:1048F00007910FD04FF4805501462A466846FBF7D2
:104900006BFDDDE90047284601F090F85FEA000AF8
:104910000CD016E08621C8F800100921CBF8001051
:104920007946C7480160862009B0A6E68221C8F80A
:1049300000102221CBF800107946C1480160822086
:10494000F2E7A9EB0605C7F58050A84200D205465C
:10495000B5F5805F04D020465146FFF705F980B9D0
:104960002046FFF786F860B907982A46811907EBB9
:104970000A00FBF748FD2E4420465146FFF70AFF88
:1049800028B1504601F024F8D8F80000CCE7002701
:10499000641C4E45D5D3504601F01AF80020C8F8E3
:1049A0000000CBF800007946A54801600020BBE775
:1049B0002DE9FF4F8DB00D46DDF8689000269E4C26
:1049C00007935FEA09013ED04FF4805701463A460B
:1049D0006846FBF701FDDDE900B10C913A46691C20
:1049E0006846FBF7F9FCDDE90010CDE904013A4621
:1049F00068460F99FBF7F0FCDDE90085A9EB060797
:104A0000C5F58050B84200D2074625B1D8457CD1C3
:104A10000C98854279D14FF4805001F007F85FEA95
:104A2000000A1BD0D8454FD10C9885424CD12A465C
:104A30004FEA08305146FEF770FF000618D5504681
:104A400000F0C6FF79E0862020607C4809210160E3
:104A500078467B490860862011B00EE682202060EF
:104A60007648222101607946754801608220F3E78B
:104A70000598804509D1049901EB0030C1F58052B9
:104A80005144FEF74AFF0006D9D44046FEF7F1FF35
:104A90000006D4D407983A46811905EB0A00FBF7C3
:104AA000B2FCEA194FEA08305146FFF74EFE000605
:104AB000C5D40599884533D1049800EB0130049999
:104AC000C1F58052514427E0059988450AD10498E0
:104AD00000EB01300499C1F580525146FEF71DFFED
:104AE0000006ACD44046FEF7C4FF0006A7D40798E2
:104AF0003A4681190F983044FFF727FE00069ED4EE
:104B0000059988450CD1049800E00DE000EB0130D8
:104B10000499C1F580525146FFF717FE00068ED466
:104B2000504600F055FF0AE007983A4681190F9861
:104B30003044FFF70AFE000601D520688CE73E44AA
:104B4000002508F101084E45FFF458AF0020206011
:104B50003A49086078463A49086000207CE74FF4FB
:104B6000800070474FF4805070472DE9F041354C7C
:104B70000F460646A56806E0A068401BB04202D377
:104B80000120BDE8F081384600F003F80028F3D199
:104B9000F7E770B5044600BF00BF00BF00BF00BF0D
:104BA00000BF00BF00BF00BF00BF00BF00BF00BF0D
:104BB00000BF00BF00BF00BF00BF00BF00BF00BFFD
:104BC00000BF00BF00BF00BF00BF00BF00BF00BFED
:104BD00000BF00BF00BF1C4E4FF48025F5630520C9
:104BE000FBF7D8FB0020FBF7D5FB2070B56300BFB7
:104BF00000BF00BF00BF00BF00BF00BF00BF00BFBD
:104C000000BF00BF00BF00BF00BF00BF00BF00BFAC
:104C100000BF00BF00BF00BF00BF00BF00BF00BF9C
:104C200000BF00BF00BF00BF00BF00BF00BF2078B3
:104C300000F0010070BD000084C0072088C007207C
:104C40008CC007200000094000C0092000207047E8
:104C5000D04982200860D049212008607846CF4999
:104C6000086082207047CB4982200860CA49222010
:104C700008607846C949086082207047C54982208B
:104C80000860C549222008607846C449086082202F
:104C9000704770B5002400BF00BF00BF00BF00BF59
:104CA00000BF00BF00BF00BF00BF00BF00BF00BF0C
:104CB00000BF00BF00BF00BF00BF00BF00BF00BFFC
:104CC00000BF00BF00BF00BF00BF00BF00BF00BFEC
:104CD00000BF00BF00BFB24E4FF48025F5639F2098
:104CE000FBF758FB0020FBF755FB60F3070400209F
:104CF000FBF750FB60F30F240020FBF74BFB60F346
:104D00001744B56300BF00BF00BF00BF00BF00BFB6
:104D100000BF00BF00BF00BF00BF00BF00BF00BF9B
:104D200000BF00BF00BF00BF00BF00BF00BF00BF8B
:104D300000BF00BF00BF00BF00BF00BF00BF00BF7B
:104D400000BF00BF9749601A8C4233D019DC964AE5
:104D50004FF48031A4EB020094422BD009DCA4F183
:104D6000C204B4F5A11425D08C4223D08F4820442E
:104D700013E000F65A70B0F540401BD0884216D1BF
:104D800018E08B4A811A90420FD008DCA0F56060D1
:104D9000A9380FD0A0F55F40FA3840B90AE085483D
:104DA000081809D08449C84201D1022400E0002437
:104DB000204670BD0324FBE70424FFF76DFBF7E7F3
:104DC0007E48007828B17E4900EB800051F8300021
:104DD00000477049822008606F49212008607846AA
:104DE0006E4908608220704770B5FFF752FF734923
:104DF000694D6A4E674C087050B1714900EB8000F4
:104E000001EBC000C0688047000609D5206870BD6E
:104E1000822020602120286078463060822070BD8A
:104E200000202060286078463060002070BD2DE9A9
:104E3000F041624B584D594E1B78564C63B19AB1B4
:104E40005F4F03EB830307EBC3035B6998470006DF
:104E500012D52068BDE8F0818220206021202860E2
:104E6000784630608220F5E786202060092028609F
:104E7000784630608620EDE7002020602860784684
:104E800030600020E6E72DE9F0414C4B424D434EA7
:104E90001B78404C5BB192B1494F03EB830307EBA6
:104EA000C3039B699847000611D52068D2E782208A
:104EB000206022202860784630608220CAE7862061
:104EC000206009202860784630608620C2E70020F4
:104ED00020602860784630600020BBE72DE9F04173
:104EE000364B2D4D2D4E1B782A4C5BB192B1344F71
:104EF00003EB830307EBC303DB699847000611D577
:104F00002068A7E782202060222028607846306051
:104F100082209FE786202060092028607846306044
:104F2000862097E7002020602860784630600020C7
:104F300090E7F8B5214C184D184E2778154CDDF840
:104F400018C087B1BCF1000F15D0CDF800C0DFF854
:104F500070C007EB87070CEBC7073F6AB84700062E
:104F600011D52068F8BD8220206022202860784674
:104F700030608220F8BD86202060092028607846B5
:104F800030608620F8BD00202060286078463060C0
:104F90000020F8BD84C0072088C007208CC00720EF
:104FA00000C009201F3217001C70150025C0FEFF2D
:104FB000A0F3290000FFFEFF0001F8FF3CC107201D
:104FC000305D00002DE9F84FFF4C07460026E068F1
:104FD00020F44040E060E06C40F44040E064FB4D71
:104FE0004FF4000BC5F83CB0286A20F4000028629A
:104FF00000BF00BF00BF00BF00BF00BF00BF00BFB9
:1050000000BF00BF00BF00BF00BF00BF00BF00BFA8
:1050100000BF00BF00BF00BF00BF00BF00BF00BF98
:1050200000BF00BF00BF00BF00BF00BF00BF00BF88
:105030004FF4800AC5F83CA00320FBF7ABF93046DB
:10504000FBF7A8F9686BC0F3C0593046FBF7A2F92B
:10505000686BC0F3C0583046FBF79CF9686B0121C0
:105060006846FBF7AAF9C5F838A000BF00BF00BF2B
:1050700000BF00BF00BF00BF00BF00BF00BF00BF38
:1050800000BF00BF00BF00BF00BF00BF00BF00BF28
:1050900000BF00BF00BF00BF00BF00BF00BF00BF18
:1050A00000BF00BF00BF00BF00BFC1456ED100BF41
:1050B00000BF00BF00BF00BF00BF00BF00BF00BFF8
:1050C00000BF00BF00BF00BF00BF00BF00BF00BFE8
:1050D00000BF00BF00BF00BF00BF00BF00BF00BFD8
:1050E00000BF00BF00BF00BF00BF00BF00BFC5F8CA
:1050F0003CA00320FBF74EF9E06820F44040E0605C
:10510000E06C20F44040E064C5F838B0286A40F410
:10511000000028623046FBF73DF9686BC0F3C059C8
:10512000286A20F4000028623046FBF733F9686BE8
:10513000C0F3C0583046FBF72DF9686B0121684673
:10514000FBF73BF9C5F838A000BF00BF00BF00BFA8
:1051500000BF00BF00BF00BF00BF00BF00BF00BF57
:1051600000BF00BF00BF00BF00BF00BF00BF00BF47
:1051700000BF00BF00BF00BF00BF00BF00BF00BF37
:1051800000BF00BF00BF00BFC14501D03E7007E0B7
:10519000B9F1000F18D0B8F1000F15D00120387008
:1051A000E06840F44040E060E06C20F4404040F4AF
:1051B0000040E06486480660864806607946864876
:1051C00001600020BDE8F88FE06840F44040E060F6
:1051D000E06C20F4404040F40040E0647C488221D0
:1051E00001607C480321016079467B480160822090
:1051F000E8E710B504467948007818B1C4F30740D1
:10520000FBF7C8F8C4F30720FBF7C4F8E0B2BDE829
:105210001040FBF7BFB870B5044600BF00BF00BF29
:1052200000BF00BF00BF00BF00BF00BF00BF00BF86
:1052300000BF00BF00BF00BF00BF00BF00BF00BF76
:1052400000BF00BF00BF00BF00BF00BF00BF00BF66
:1052500000BF00BF00BF00BF00BF5C4E4FF4800521
:10526000F5630520FBF796F80020FBF793F8207014
:10527000B56300BF00BF00BF00BF00BF00BF00BFDD
:1052800000BF00BF00BF00BF00BF00BF00BF00BF26
:1052900000BF00BF00BF00BF00BF00BF00BF00BF16
:1052A00000BF00BF00BF00BF00BF00BF00BF00BF06
:1052B00000BF207800F0010070BD70B5064600BF49
:1052C00000BF00BF00BF00BF00BF00BF00BF00BFE6
:1052D00000BF00BF00BF00BF00BF00BF00BF00BFD6
:1052E00000BF00BF00BF00BF00BF00BF00BF00BFC6
:1052F00000BF00BF00BF00BF00BF00BF00BF334DF5
:105300004FF48004EC630620FBF744F8AC6300BF65
:1053100000BF00BF00BF00BF00BF00BF00BF00BF95
:1053200000BF00BF00BF00BF00BF00BF00BF00BF85
:1053300000BF00BF00BF00BF00BF00BF00BF00BF75
:1053400000BF00BF00BF00BF00BF00BF00BF00BF65
:1053500000BF00BF00BF00BF00BF00BF00BF00BF55
:1053600000BF00BF00BF00BF00BF00BF00BF00BF45
:1053700000BF00BF00BF00BF00BF00BF00BF00BF35
:1053800000BF00BF00BF00BF00BF00BF00BFEC6395
:105390000120FAF7FFFF3046FAF7FCFFAC6300BFCD
:1053A00000BF00BF00BF00BF00BF00BF00BF00BF05
:1053B00000BF00BF00BF00BF00BF00BF00BF00BFF5
:1053C00000BF00BF00BF0BE000C0024000C00920CA
:1053D00084C0072088C007208CC0072040C1072058
:1053E00000BF00BF00BF00BF00BF00BF00BF00BFC5
:1053F00000BF00BF00BF00BF70BDF8B5FD4C6078B6
:10540000FD4EFE4FFE4D68BB012060706846FFF701
:1054100002FF9DF80000800811D00020FFF74DFF2B
:105420006846FFF7F8FE9DF80000800807D082204C
:10543000286003203060784638608220F8BDED484F
:10544000FFF7C0FD000601D52868F8BD207820B11F
:105450004FF400306060401203E04FF400406060A1
:105460004020A0600020286030607846386000202E
:10547000F8BDF8B54FF47A70E24DE34C4FF4800676
:10548000009000BF00BF00BF00BF00BF00BF00BF53
:1054900000BF00BF00BF00BF00BF00BF00BF00BF14
:1054A00000BF00BF00BF00BF00BF00BF00BF00BF04
:1054B00000BF00BF00BF00BF00BF00BF00BF00BFF4
:1054C00000BFEE630520FAF765FF0020FAF762FFE0
:1054D000AE6300BF00BF00BF00BF00BF00BF00BF82
:1054E00000BF00BF00BF00BF00BF00BF00BF00BFC4
:1054F00000BF00BF00BF00BF00BF00BF00BF00BFB4
:1055000000BF00BF00BF00BF00BF00BF00BF00BFA3
:1055100000BFC0070AD0009838B1401E0090A068B4
:10552000A168091A3229FBD3ABE70120F8BD2DE9A8
:10553000F041B14C15000F4680460AD0AD48032615
:10554000406810B1FFF795FF38B126608220BDE8B2
:10555000F081092020608620F9E700BF00BF00BF6E
:1055600000BF00BF00BF00BF00BF00BF00BF00BF43
:1055700000BF00BF00BF00BF00BF00BF00BF00BF33
:1055800000BF00BF00BF00BF00BF00BF00BF00BF23
:1055900000BF00BF00BF00BF00BF9A4E4FF48004A1
:1055A000F4630320FAF7F6FE4046FFF722FE294691
:1055B0003846FAF702FFB46300BF00BF00BF00BF68
:1055C00000BF00BF00BF00BF00BF00BF00BF00BFE3
:1055D00000BF00BF00BF00BF00BF00BF00BF00BFD3
:1055E00000BF00BF00BF00BF00BF00BF00BF00BFC3
:1055F00000BF00BF00BF00BF0020A8E72DE9F05F9B
:105600007D4F1500044688461AD07A480E464FF062
:105610000409416800297DD04FF4800B824660194F
:10562000401EDAF8081060404A1E904373D004EA26
:105630000200A1EB0008FFF71CFF00286AD104E07C
:10564000092038608620BDE8F09F00BF00BF00BF82
:1056500000BF00BF00BF00BF00BF00BF00BF00BF52
:1056600000BF00BF00BF00BF00BF00BF00BF00BF42
:1056700000BF00BF00BF00BF00BF00BF00BF00BF32
:1056800000BF00BF00BF00BF00BF5E49C1F83CB013
:105690000620FAF77FFE5B49C1F838B000BF00BFB3
:1056A00000BF00BF00BF00BF00BF00BF00BF00BF02
:1056B00000BF00BF00BF00BF00BF00BF00BF00BFF2
:1056C00000BF00BF00BF00BF00BF00BF00BF00BFE2
:1056D00000BF00BF00BF00BF00BF00BF00BF00BFD2
:1056E00000BF00BF00BF00BF00BF00BF00BF00BFC2
:1056F00000BF00BF00BF00BF00BF00BF00BF00BFB2
:1057000000BF00BF00BF00BF00BF00BF00BF00BFA1
:1057100000BF01E041E03DE000BF00BF00BF00BFAF
:1057200000BF3849C1F83CB00220FAF733FE2046EA
:10573000FFF75FFD41463046FAF733FE3149C1F8C5
:1057400038B000BF00BF00BF00BF00BF00BF00BF38
:1057500000BF00BF00BF00BF00BF00BF00BF00BF51
:1057600000BF00BF00BF00BF00BF00BF00BF00BF41
:1057700000BF00BF00BF00BF00BF00BF00BF00BF31
:1057800000BF46444444B5EB0805B0467FF447AF3C
:10579000002058E7FFF76DFE18B1C7F8009082208F
:1057A00051E700BF00BF00BF00BF00BF00BF00BF88
:1057B00000BF00BF00BF00BF00BF00BF00BF00BFF1
:1057C00000BF00BF00BF00BF00BF00BF00BF00BFE1
:1057D00000BF00BF00BF00BF00BF00BF00BF00BFD1
:1057E00000BF5E46074FC7F83CB00620FAF7D2FD6F
:1057F000BE630BE040C1072088C007208CC0072093
:1058000084C0072000C009200000094000BF00BF7D
:1058100000BF00BF00BF00BF00BF00BF00BF00BF90
:1058200000BF00BF00BF00BF00BF00BF00BF00BF80
:1058300000BF00BF00BF00BF00BF00BF00BF00BF70
:1058400000BF00BF00BF00BF00BF00BF00BF00BF60
:1058500000BF00BF00BF00BF00BF00BF00BF00BF50
:1058600000BF00BF00BF00BF00BF00BF00BF00BF40
:1058700000BF00BF00BF00BF00BF00BF00BF00BF30
:1058800000BF00BF00BF00BF00BF00BFFE6302201B
:10589000FAF780FD2046FFF7ACFC29464046FAF7B0
:1058A00080FDBE6300BF00BF00BF00BF00BF00BFE0
:1058B00000BF00BF00BF00BF00BF00BF00BF00BFF0
:1058C00000BF00BF00BF00BF00BF00BF00BF00BFE0
:1058D00000BF00BF00BF00BF00BF00BF00BF00BFD0
:1058E00000BF00BF54E70348406870470148806824
:1058F0007047000040C10720D2B201E000F8012B40
:10590000491EFBD270470022F6E710B513460A463F
:1059100004461946FFF7F0FF204610BD70B500247D
:105920002546002801DA01244042002901DA012538
:10593000494200F019F8AC4200D04042002C00D09F
:10594000494270BD064C074D06E0E06840F0010397
:1059500094E8070098471034AC42F6D3FAF7BAFB44
:10596000605F0000905F000030B50B4601460020EC
:105970002022012409E021FA02F59D4205D303FA11
:1059800002F5491B04FA02F52844151EA2F1010292
:10599000F1DC30BD30B58C1810F8012B12F00F037C
:1059A00001D110F8013B120906D110F8012B03E0D8
:1059B00010F8015B01F8015B5B1EF9D101E001F811
:1059C000013B521EFBD1A142E6D3002030BD0000B6
:1059D00030B528B1144C031F002021680A4605E0A9
:1059E000084630BD9A4203D810465268002AF9D1C1
:1059F000002800D041680BD00468A3EB0005A54245
:105A000004D11B681C440346046002E0436000E0CC
:105A100023603AB11C68D51AA54203D115682C44FD
:105A20001C6052685A6030BD4CC107202DE9F04718
:105A300082460F4C10480D4E0E4F001B4FF00008D1
:105A400020F007054FF0010900221146504600F0F2
:105A50001DF8002802D1306810B10020BDE8F087A1
:105A60003C60C4E90058C6F80090EDE750C107203B
:105A7000040000104CC1072000500010002001E07D
:105A800001C1121F002AFBD1704700002DE9F0412F
:105A90000B3020F00706104D19E02068B04215D3F6
:105AA000B0420AD9871B201DD4F80480FAF7ABFC5A
:105AB000A019C0E90078286004E060682860201D13
:105AC000FAF7A1FC201D2660BDE8F081251D2C6899
:105AD000002CE2D10020F7E74CC10720F0F1F2F3EF
:105AE000F0F1F2F3F0F1F2F3F0F1F2F3F0F1F2F39E
:105AF000F0F1F2F3F0F1F2F3F0F1F2F365787061A6
:105B00006E642033322D62797465206B6578706124
:105B10006E642031362D62797465206BEB3C904DBC
:105B200053444F53352E3000020201000110000093
:105B300004F80C000100010000000000000000005B
:105B4000000029EFBEADDE41544F4C204650726933
:105B50006E744641543132202020000000000000C5
:105B60000010000000200000003000000040000095
:105B70000050000000600000007000000080000085
:105B80000090000000A0000000B0000000C0000075
:105B900000D0000000E0000000F000000000010064
:105BA00000800100000002000080020000000300ED
:105BB00000800300000004000080040000000500D5
:105BC00000800500000006000080060000000700BD
:105BD00000800700FF0F0000FF1F0000FF2F0000E4
:105BE000FF3F0000FF4F0000FF5F0000FF6F00005D
:105BF000FF7F0000FF8F0000FF9F0000FFAF00004D
:105C0000FFBF0000FFCF0000FFDF0000FFEF00003C
:105C1000FFFF0000FF7F0100FFFF0100FF7F020088
:105C2000FFFF0200FF7F0300FFFF0300FF7F040070
:105C3000FFFF0400FF7F0500FFFF0500FF7F060058
:105C4000FFFF0600FF7F0700FFFF070012011001A2
:105C50000000004051C20313000104204801090262
:105C60002000010100803209040000020806506291
:105C70000705820240000007050202400000000400
:105C80000309041C03410054004F004C0020002075
:105C900000200020002000200020002000200028FC
:105CA0000346005000720069006E00740020004638
:105CB000006C0061007300680020002000200020BC
:105CC000002000200020001A034600690072006DC9
:105CD0000077006100720065003000300030003055
:105CE000000E034D0065006D006F0072007900002A
:105CF0007526000000000000012C000000000000DC
:105D00000000000000000000000000000000000093
:105D10000000000000000000000000000000000083
:105D20000000000000000000000000000000000073
:105D30004D4C00004D4C00004D4C0000514C0000FB
:105D4000674C0000514C0000674C0000674C00009D
:105D5000674C00007D4C00004D4C00004D4C000095
:105D60004D4C0000514C0000674C0000514C0000AD
:105D7000674C0000674C0000674C00007D4C000041
:105D80000B430000114300004D4C0000FB4000009D
:105D90000B420000413E0000753E0000293A000021
:105DA0004B3F0000174300003B340000413400002B
:105DB000473400000D2F00000B420000413E000060
:105DC000973100004B4700008B3200004D3400003B
:105DD0005F4B0000654B00004D4C0000FB40000095
:105DE0000B420000413E0000DB4800004B47000032
:105DF000B14900001743000000000000000000004F
:105E00000000000000000000000000000000000092
:105E10000000000000000000000000000000000082
:105E200099020000990200002F550000990200001D
:105E3000990200009902000099020000B7020000D8
:105E400099020000990200009902000099020000E6
:105E500099020000990200009902000099020000D6
:105E60009B0200009B020000FD5500009B02000009
:105E70009B0200009B0200009B020000BB0200008E
:105E80009B0200009B0200009B0200009B0200009E
:105E90009B0200009B0200009B0200009B0200008E
:105EA0009D0200009D020000E75800009D020000D6
:105EB0009D0200009D0200009D0200009D02000066
:105EC0009D0200009D0200009D0200009D02000056
:105ED0009D0200009D0200009D0200009D02000046
:105EE0009F0200009F020000ED5800009F0200008A
:105EF0009F0200009F0200009F0200009F0200001E
:105F00009F0200009F0200009F0200009F0200000D
:105F10009F0200009F0200009F0200009F020000FD
:105F2000A1020000A1020000A1020000A1020000E5
:105F3000A1020000A1020000A1020000A1020000D5
:105F4000A1020000A1020000A1020000A1020000C5
:105F5000A1020000A1020000A1020000A1020000B5
:105F6000905F000000C00720540100009459000019
:105F7000905F000000000010005000007C5A0000FC
:105F8000B05F000054C107203C3300007C5A000081
:105F90000118BD41544F4C20465072696E7428055B
:105FA00048D4284B3D057A17C00720035E093D0001
:105FB000B8729C9806F1D40FC7D197B43838A708A7
:105FC0004BC729114FCDFD6AAA6DAE2DBE580E24C8
:105FD0000D7B79624BE228D97D5C6EE5104175C975
:105FE000EC7DBEA600B928B12ADBA3CE10392D6303
:105FF00094CE6BEA0B0438B36D8EABDC4ECDBB9503
:10600000C8150820E160000089970200A142020043
:106010000D9702001D640000E91805001A9BEADFD5
:10602000000000000000000000000000EF60000021
:10603000F1600000000000003D330300F560000047
:10604000F760000065D20400F760000089D2040008
:10605000F9DA0400C1060500F76000003507050005
:10606000F7600000F7600000F7600000F7600000D4
:10607000F7600000F7600000F7600000F7600000C4
:10608000F7600000F7600000F7600000F7600000B4
:10609000F7600000F7600000F7600000F7600000A4
:1060A000A90F0500F7600000AD150100F7600000C2
:1060B000F7600000F7600000F7600000F760000084
:1060C000F7600000F7600000F7600000DFF80CD018
:1060D00000F0A6FC00480047B93D0500C81508209F
:1060E00005480047FEE7FEE7FEE7FEE7FEE7FEE7BE
:1060F000FEE7FEE7FEE7FEE7CD6000002DE9F05F7A
:106100000546002092469B46884606468146402426
:106110001BE0284641464746224600F02FF85346EA
:106120005A46C01A914110D311461846224600F033
:1061300016F82D1A67EB01084F4622460120002170
:1061400000F00DF817EB00094E41201EA4F10104E8
:10615000DFDC484631462A464346BDE8F09F202A08
:1061600004DB203A00FA02F1002070479140C2F1AE
:10617000200320FA03F3194390407047202A04DBE0
:10618000203A21FA02F00021704721FA02F3D040B0
:10619000C2F12002914008431946704700487047F9
:1061A000C05E06000649074A0868504343F23902B8
:1061B00010440860400870470149086070470000BB
:1061C000E00300106D4EC64110B50B460446114663
:1061D000184600F023FBC4E9000110BD10B5441AB5
:1061E0000346944209D28418114403E011F8013D9A
:1061F00004F8013D521EF9D210BD40EA0104A40783
:1062000003D009E010C9121F10C3042AFAD203E018
:1062100011F8014B03F8014B521EF9D210BDD2B256
:1062200001E000F8012B491EFBD270470022F6E77F
:1062300010B513460A4604461946FFF7F0FF2046FC
:1062400010BD421E12F8013F002BFBD111F8013B9B
:1062500002F8013B002BF9D1704730B505462A46BC
:106260000B4612F8010B13F8014B08B1A042F8D00D
:106270001CB1002802D06D1CF1E7284630BD10B5D6
:10628000044604E00B7800F8013B03B1491C521EA0
:10629000F8D2204610BDCAB2401E10F8011F8A4233
:1062A00002D00029F9D100207047421C10F8011BD0
:1062B0000029FBD1801A7047CBB203E001789942E4
:1062C00003D0401C521EF9D20020704730B504465E
:1062D0000020034600E05B1C934203D2E05CCD5CEF
:1062E000401BF8D030BD10B5044600E0401C0378D8
:1062F000002BFBD100E0401C521E04D311F8013BDF
:106300000370002BF7D100210170204610BD034619
:1063100011F8012B00F8012B002AF9D1184670471B
:1063200010B5484304464CF015F8002805D000216C
:10633000002C02D0641E0155FAE710BD2DE9F0478C
:1063400091460F4680460446002614F8015B2DB1A5
:10635000FFF724FF0068405DC007F6D12B2D02D067
:106360002D2D18D0641E4A463946204600F07CFA8E
:1063700027B13968A14201D1C7F8008071054FF0FB
:1063800002040BD54042002803DD4BF0B1FF04604E
:10639000A007BDE8F08746F48066E4E70028F8DA55
:1063A0004BF0A6FF04606FF00040F2E770B50646C0
:1063B0004BF09EFF046805460A2200213046FFF795
:1063C000BDFF2C6070BD0EB540F23341029100213B
:1063D000CDE900110A460B4600F0A4FA03B000BD57
:1063E0003A2800D2303820F02002412A01D3A2F10D
:1063F0003700884201D34FF0FF30704740BA7047F2
:106400005E663194C42070470100704756007047A3
:106410004F63742031382032303139004BF0F6FBB5
:1064200031353A33363A3132000070470100704757
:10643000000011010200704700A007002DE9F05F85
:1064400093460F468046044600264BF051FFD0F895
:106450000090824614F8015B2DB1FFF79FFE0068A3
:10646000405DC007F6D12B2D02D02D2D1AD0641E11
:106470000021CAF800105A463946204600F0F4F9C7
:10648000014627B13868A04201D1C7F80080DAF888
:106490000000022809D0CAF80090700505D54842CE
:1064A000BDE8F09F46F48066E2E70846F8E72DE98C
:1064B000FE4F804681EA0300C00F0C46009021F099
:1064C000004123F00045B8EB0200A94105D2404647
:1064D000214690461C460B46024623F000401043DE
:1064E00047D0270DC7F30A00C3F30A510290401AA0
:1064F000019040286BDAC3F3130040F4801B00982E
:10650000924620B10023D2EB030A63EB0B0B0198F8
:106510005946C0F140025046FFF721FE06460D469F
:1065200050465946019A00F08DF910EB0800614180
:10653000002487EA115284EAE7731A4340D0009A94
:1065400062B3019A012A4FEA075215DC001B61EB86
:1065500002014FF0004202EA0752CDE90042001C5E
:1065600041F5801132462B4600F0DCF903B0BDE85E
:10657000F08F40462146F9E7001B61EB0201001C49
:1065800041F5801300185B412018A2F5001747EB76
:10659000030140EAD570B6196D4111E06D084FEA6C
:1065A000360645EAC0754FEA0752001B61EB02014F
:1065B000001C41F5801149084FEA30000019514193
:1065C00032462B4603B0BDE8F04F00F09CB900986E
:1065D000012240000023D0EB020263EBE07300983D
:1065E00021464FEAE074B8EB000061EB0401E9E7F3
:1065F00083F000435BE781F0004158E72DE9FE4F4F
:1066000081EA030404F0004421F0004100944FF0BB
:10661000000B23F0004350EA01045ED052EA030469
:106620005BD0C3F30A54C1F30A552C44A4F2F334EB
:106630000194A0FB0254C1F3130141F48011C3F390
:10664000130343F4801301FB024400FB034E840A4E
:10665000970A44EA815447EA8357A4FB07680295E6
:106660008D0A05FB07854FEA932C04FB0C54270584
:10667000029D4FEA065847EA1637B5EB08056EEB60
:10668000070C870E920E47EA811742EA8312A7FB96
:106690000201B6EB0B0164EB00042B0D43EA0C3353
:1066A0005E1844EB1C50DA465146E7FB0201C5F385
:1066B00013044FEA0B3343EA14534FEA0432019CAC
:1066C00043EA0603A4F10C040294009CCDE900B453
:1066D00000F028F903B0BDE8F08F00200146F9E78B
:1066E0002DE9F04D81EA030404F0004B21F0004550
:1066F00014464FF0000A23F0004150EA050220D072
:1067000054EA01021DD0C5F30A570246C5F313032C
:10671000C1F31300C1F30A5640F4801543F480130B
:10672000A7EB0608101BD64608F2FD3873EB0500F0
:1067300002D308F1010801E092185B41B8F1000FA3
:1067400003DA00200146BDE8F08D00204FF48011EF
:10675000064684460EE0171B73EB050705D3121B94
:1067600063EB050306434CEA010C49084FEA30008D
:1067700092185B4150EA0107EDD152EA030012D0B2
:1067800082EA040083EA0501084305D0101BAB41EF
:1067900006D20122002306E000224FF0004302E06F
:1067A0006FF0010253101AEB06004CEB085110EB8E
:1067B0000A0041EB0B01BDE8F04D00F0A4B8C1F3B5
:1067C0000A5210B5C1F3130140F2FF3341F48011B6
:1067D0009A4201DA002010BD40F233439A42A2F2FD
:1067E000334203DC5242FFF7C9FC10BD904010BD9C
:1067F00030B50B46014600202022012409E021FA91
:1068000002F59D4205D303FA02F5491B04FA02F58D
:106810002844151EA2F10102F1DC30BD70B5002440
:106820002546002801DA01244042002901DA012529
:106830004942FFF7DDFFAC4200D04042002C00D0BF
:10684000494270BD202A06DBCB17203A41FA02F0FC
:1068500043EAE07306E041FA02F3D040C2F12002BD
:1068600091400843194670472DE9F05F8246007851
:10687000002715468B460AF10104B946302801D09D
:106880009DB113E014F8010B0127782803D0582894
:1068900001D045B10AE00DB1102D07D10027102518
:1068A00014F8010B02E0082500E00A250026B04696
:1068B0000EE005FB080005FB06F1012701EB104681
:1068C0001FFA80F8B6F5803F00D3B94614F8010BE3
:1068D0002946FFF785FD0028EBDABBF1000F05D054
:1068E0000FB1641E00E05446CBF80040B9F1000F30
:1068F00006D04BF0FDFC02210160C81EBDE8F09FF0
:1069000048EA0640FAE710B5141E73F1000408DAED
:10691000401C41F1000192185B411A4301D120F063
:10692000010010BD2DE9F04D92469B4611B1B1FA20
:1069300081F202E0B0FA80F220329046FFF70FFCBD
:1069400004460F4640EA0A0041EA0B0153465A4604
:10695000084313D0114653EA010019D0C8F1400290
:106960005046FFF70BFC05460E4650465946424638
:10697000FFF7F5FB084305D0012004E02046394627
:10698000BDE8F08D0020054346EAE0762C4337430E
:106990000A986305E40AA0EB08000022FD0A44EA15
:1069A00047540A3002D500200146E9E701051019D5
:1069B0006941DDE9084500196941BDE8F04DA2E7EC
:1069C000C1F30A52C1F3130140F2FF3341F48011C5
:1069D0009A4202DA00200146704740F233439A425D
:1069E000A2F2334202DC5242FFF7C8BBFFF7B7BB4B
:1069F00030B5041E71F1000404DB4FF00044404246
:106A000064EB0101141E73F1000405DB1C464FF01A
:106A10000043524263EB0403994208BF904230BDE9
:106A2000064C074D06E0E06840F0010394E80700DB
:106A300098471034AC42F6D3FFF74CFB00AB06008E
:106A400040AB060070B58C1810F8015B15F0070319
:106A500001D110F8013B2A1106D110F8012B03E0F7
:106A600010F8016B01F8016B5B1EF9D12B0705D4FF
:106A70000023521E0DD401F8013BFAE710F8013B48
:106A8000CB1A921C03E013F8015B01F8015B521E64
:106A9000F9D5A142D8D3002070BD00000B490A6887
:106AA00022F080720A600A68012322F0FF0283400C
:106AB0001A4342F08070086048680028FCDA0A68CF
:106AC00022F080720A6080B27047000000400340EC
:106AD00010B5EFF3108101F0010472B6FFF7DEFF8D
:106AE000002C00D162B610BD07490648086007496E
:106AF000886842F210728B681B1A9342FBD3002005
:106B000070470000000120000040034000000940E1
:106B10002DE9F05F59485A4D00260680B5F8223815
:106B2000B5F8201840F225145A1AC2F30A02A242FC
:106B300002DD701EBDE8F09F8146B0F800C04F48EE
:106B4000FE27801C4F4C0CF80070012702F07F0CD0
:106B500007F800C00227D2093A540322A9F80020FE
:106B600095F81D78B246A846474EFD43257086F835
:106B700000A04FF0310B25785FEA056C02D58BEA57
:106B8000450500E06D00257035786D1CEDB235705F
:106B9000082DF0D31754B9F800003C4F401CA9F859
:106BA000000038887A884546104007EB8000D846B8
:106BB000C38038887A88104007EB8000018178888C
:106BC000401C7880C1F30A002844491C007DA8714C
:106BD000A5F8201821784140217086F800A021787E
:106BE0000A0602D588EA410100E0490021703178A7
:106BF000491CC9B231700829F1D300BF45F094F99E
:106C0000B5F82208B5F82018401A40051CD0C1F389
:106C10000A002844491C007DA871A5F82018217895
:106C200042464140217086F800A021780B0602D52B
:106C300082EA410100E0490021703178491CC9B263
:106C400031700829F1D3D9E77888401E80B2788066
:106C50003988014007EB8100C188A5F82218008916
:106C6000A5F82008207845F05FF9B9F8001009F17F
:106C70000200BDE8F05F04F06DBD0000D6E1072022
:106C8000ACD5072029010010B0C2072004E307207B
:106C900070B5154C03460022A01CFE2111540121A1
:106CA0000A5402210A5403210B5404200F49208066
:106CB000D84308700E48312302700A78150602D5B1
:106CC00083EA420200E052000A700278521CD2B2FB
:106CD0000270082AF1D3087845F026F92188A01C13
:106CE000BDE8704004F036BDD6E107202901001050
:106CF000B0C207202DE9F047614C624D2046237851
:106D0000B0F80720604E614F80794FF000094FF6D0
:106D1000FF714FF031080A2B72D2DFE803F005AEA5
:106D2000091D2EAEAEAE528DFE2869D1022011E0B3
:106D3000FE22E270B4F81A28A4F82228A4F8202829
:106D4000020604D5FE285BD0A4F8071001E0A4F8E1
:106D50000700032020706BE08A420AD0030604D5A6
:106D6000FE284DD0A4F8071003E002EBC010A4F8F1
:106D70000700FF2028700420ECE784F81D08EF28A6
:106D800063D88A4261D084F8150808212170618A8D
:106D9000A4F81A18A4F8181829784840287086F81A
:106DA000009041462878020602D581EA400000E0C2
:106DB000400028703078401CC0B230700828F1D3F1
:106DC00036E01FF02FFC3860A32833D1B4F81A182E
:106DD000A079C1F30A0121440875B4F81A08401CCF
:106DE00081B2A4F81A18A0792A785040287086F841
:106DF000009042462878030603D582EA400001E06D
:106E00003BE0400028703078401CC0B23070082849
:106E1000F0D3B4F81808081AB4F80710C0F30A0041
:106E2000884212D802D14FF0090020702878607291
:106E30004FF0B700BDE8F0871FF0F4FB3860A328DF
:106E4000F8D1607AA179884201D0B520F2E7B4F890
:106E50001A08A4F82208A4F8200894F8150884F861
:106E60001D0804F61A0400F013F8E088A4F61A04CA
:106E7000C0F30A002044007DDCE7B620DAE700001A
:106E8000ACD5072028010010AFC207202401001054
:106E90001448B0F81818C1F30A020244491C127DC4
:106EA000A0F81818C13A052A0ED2DFE802F003094B
:106EB00005070B0000F0DAB900F08EBB00F014B843
:106EC00000F076B800F020B9B0F82228B521C2F35E
:106ED0000A0202441175B0F82218491CA0F82218C1
:106EE00070470000ACD5072070B52F4CB4F81A08D5
:106EF000B4F81818401A400501D0B5204CE0012123
:106F0000A2204DF001FD01B2481C3DD0B4F8240888
:106F1000084004EBC0022548B2F830580388468880
:106F2000334000EB8303DD80B2F82E3802884588B9
:106F30002A4000EB82021381428892B24280038889
:106F4000134000EB8300C288628200892082B4F87B
:106F50002228A220C2F30A0222441075B4F82208A3
:106F6000401CA4F82208B4F82428C0F30A000A4000
:106F700004EBC201204491F82C180175B4F82208E2
:106F8000401CA4F8220870BD002060822082A4F872
:106F90002808A4F82608A320B4F82218C1F30A018F
:106FA00021440875EAE70000ACD5072004E3072078
:106FB00070B5534CB4F81A08B4F81818401AC0F356
:106FC0000A032046012BB0F82228C2F30A02024429
:106FD00002D0B52010758DE0C1F30A002044491C91
:106FE000007DA071A4F81818EF280CD9B4201075F2
:106FF000B4F82208401CA4F82208C0F30A00204478
:107000000021017576E04DF0BBFC01B2481C0DD0AB
:10701000B4F82408084004EBC00090F82A08A3281C
:1070200006D0A42804D0A82857D101E0B3205BE003
:107030003448B4F82838028845882A4000EB820298
:10704000D38002884588B4F826382A4000EB8202B3
:1070500013814288521C428004EBC10292F82D3801
:1070600023F0010382F82D38A4F82818B4F8242856
:107070000A4004EBC20292F82A38A82B0ED129E06C
:1070800004EBC6025B1CA4F8263892F82D3802F6F1
:107090002A025D0702D423F00103D370B4F8242838
:1070A000B4F8283802EA0305B4F8263802EA0306E1
:1070B000AD1B1542E4D14288521E92B24280038831
:1070C000134000EB8300C288A4F828280089A4F8A4
:1070D000260802E0A32082F82A08B4F82408084011
:1070E00004EBC00090F82A08B4F82218C1F30A0192
:1070F00021440875B4F82208401CA4F8220870BD89
:10710000ACD5072004E307202DE9F041544CB4F836
:107110001A28B4F81808111AC1F30A052146062DD9
:10712000B1F82238C3F30A03194402D2B520087516
:1071300059E04C4D2B886E88334005EB8303B42611
:10714000DA802A886B881A4005EB820210816A88EF
:10715000521C93B2C0F30A0222446B80177D401C7C
:10716000A77182B2A4F81828EF2F07D90E75B4F8CA
:107170002208401CA4F82208002130E0C2F30A00D3
:107180002044521C007DA07192B2A4F81828C708B0
:1071900007D00E75B4F82208401CA4F8220801217B
:1071A0001DE094F817784FEA500C60F300076CF379
:1071B0004107800860F38207C2F30A00204484F884
:1071C0001778007D521CA071A4F81828EF2811D957
:1071D0000E75B4F82208401CA4F822080221C0F35E
:1071E0000A0020440175B4F82208401CA4F82208C3
:1071F000BDE8F0815B1E98B268802988014005EBEC
:107200008101401C0989A4F818186880491CA4F859
:107210001A18FFF7CDFEB4F82008C0F30A00204486
:10722000017D114801706888401E80B268802A88FC
:10723000024005EB8200A129C288A4F81A2800891F
:10724000A4F81808D4D0A229D2D0A529D0D0B32927
:10725000CED0401CA4F81808BDE8F04100F006B8F4
:10726000ACD5072004E30720AEC207202DE9F0418A
:10727000D84C2246B4F81A18B4F81808091AC1F301
:107280000A03B2F82218022BC1F30A01114401D2F9
:10729000B52098E0C0F30A022244401C157D83B259
:1072A000A571A4F81838E8084FF0B40207D00A75A1
:1072B000B4F82208401CA4F8220800217FE194F8C9
:1072C00017086E0865F3000066F34100AD0865F32A
:1072D000820084F81708450703D540F0010084F8C0
:1072E0001708C3F30A0020445B1C007DA071A4F8BA
:1072F0001838012684F81608EF280AD90A75B4F858
:107300002208401CA4F82208C0F30A002044067595
:1073100059E1B4F82428B4F82838B4F8267802EAF9
:1073200003051740EF1B17424FF0A8054FF0B108B7
:107330007DD05B1E1A4004EBC20292F82C78874283
:1073400037D1A448D2F82A38C0F81438D2F82E28F9
:10735000C0F8182894F814080875B4F82208401CDE
:10736000A4F8220894F81408A32819D0A42817D048
:10737000A5281CD114E000BFB4F82218C0F30A00FD
:107380002044C1F30A012144007D0875B4F81808AF
:10739000401CA4F81808B4F82208401CA4F82208DD
:1073A000B4F81A18B4F81808091A4905E4D1BDE868
:1073B000F0814DF0E5FA401C07D0B4F82218B22055
:1073C000C1F30A0121440875FDE094F8170840074D
:1073D0001ED50121A8204DF097FA411C18D084F841
:1073E0001458B4F82418014004EBC100794900F5A1
:1073F0000062D1F81438C0F82A38D1F81808C2F859
:107400002E00B4F82208C0F30A0020440575DAE023
:10741000B4F82408B4F82618B4F8282800EA0103C0
:1074200000EA0207BB423BD104EBC30300E04FE09C
:1074300093F82D385B0707D5491C0140521CA4F86E
:1074400026180240A4F82828B4F8261800EA0102F9
:1074500004EBC20292F82A38A22B07D092F82D280A
:10746000D70703D1A42B17D1920715D4B4F822184B
:10747000C1F30A01214481F81480B4F82208401CA9
:10748000A4F82208B4F82418B4F82628114004EB14
:10749000C10191F82C1892E0491C0140A4F826186B
:1074A0006078A8B1012824D0A52084F81408B4F885
:1074B0002218C1F30A0121440875B4F82208401CBF
:1074C000A4F82208C0F30A002044617901751DE088
:1074D000667094F81708400709D500BF84F814585F
:1074E000B4F82208C0F30A00204405750EE0A2207B
:1074F00004E094F817084007F0D4A12084F8140899
:10750000B4F82218C1F30A0121440875B4F822081E
:10751000401CA4F82208B4F82418B4F82808014044
:10752000401CA4F828082B4804EBC101D0F814280B
:10753000C1F82A28D0F81808C1F82E08E089618A15
:10754000228A01400240891A014202D1B4F8180887
:107550002082B4F81A08608206F0A2F9B4F8241860
:10756000B4F8260801EA0002B4F8280801EA00038A
:107570009A420BD0E289638A258A134015405B1B2F
:107580001340D21AB2F5967FBFF611AF401E0140EC
:1075900004EBC101B1F82E186182A4F82808A4F800
:1075A0002218A4F82018C1F30A01214481F814809C
:1075B000B4F82208401CA4F8220894F81618C0F366
:1075C0000A0020440175B4F82208401CA4F82208DF
:1075D000EDE60000ACD5072010B54A4CB4F81A0807
:1075E000B4F81818401AC0F30A032046012BB0F86B
:1075F0002228C2F30A02024402D0B520107558E0D6
:10760000C1F30A002044491C007DA071A4F8181899
:10761000EF2808D9B4201075B4F82208401CA4F84B
:107620002208002141E04DF0ABF900B2411C27D007
:10763000617802292CD004EBC0013248D1F82A2805
:10764000C0F81428D1F82E28C0F81828B4F8222839
:1076500094F81408C2F30A0222441075B4F8220800
:10766000401CA4F8220894F81408A12826D0A228C7
:1076700024D0A42823D0A52821D0A3281FD039E0C6
:10768000B4F82218B320C1F30A012144087510E0B0
:10769000B4F82218A520C1F30A0121440875B4F8F2
:1076A0002208401CA4F822086179C0F30A00204493
:1076B0000175B4F82208401CA4F8220810BD91F806
:1076C0002D0820F0010081F82D0813E0B4F82218ED
:1076D000C0F30A002044C1F30A012144007D08756B
:1076E000B4F81808401CA4F81808B4F82208401C84
:1076F000A4F82208B4F81A18B4F81808091A4905A9
:10770000E4D110BDACD507202DE9F0410021A22025
:107710004DF0FAF8354C0025C4F80A00401C0FD192
:107720000021A1204DF0F0F8C4F80A00411C34D02B
:10773000B4F82428A221104004EBC00080F82A18D5
:107740002B4A2C49062015600860D4F80A00B4F8CA
:107750002418DFF8A8C0084004EBC0002349D0F883
:107760002A38C1F81C38D0F82E08C1F82008224861
:10777000B4F8227801884388194000EB8101CF805A
:1077800001884688B4F82038314000EB81010B8134
:107790004188491C8EB2468011E065700020BDE82A
:1077A000F08100BFC1F30A032344491C93F814E09D
:1077B00013680CF803E0A4F820185B1C1360B4F8FD
:1077C00020187B1A5B05EDD1761EB1B2418002888C
:1077D0000A4000EB8200C188A4F822180089A4F8AE
:1077E0002008074805700120D9E70000ACD5072024
:1077F000E4000010D000001004E30720F0CD0720C3
:10780000CC00001070B5894CD4F80A00B4F82418E4
:10781000084004EBC0002146D0F82A28C1F81C28F3
:10782000D0F82E08C1F8200881480168002001B373
:10783000B4F82238B4F820288D1C9B1AC3F30A062A
:107840007C4BAE423DDBA4F82228C2F30A0222445C
:107850001075B4F82228521CA4F82228C2F30A0298
:1078600022441075B4F82208401CA4F82208002015
:1078700024E0B4F82028A4F82228C2F30A02224403
:107880001075B4F82228521CA4F82228C2F30A0268
:1078900022441075B4F82208401CA4F822083CE0E9
:1078A000B4F822581A5CC5F30A0525442A75B4F8C1
:1078B0002228521C401CA4F8222880B28842EFDB08
:1078C0002BE0228A521A921E2282A4F82028A4F8C1
:1078D0002228C2F30A0222441075B4F82228521C4E
:1078E000A4F82228C2F30A0222441075B4F8220830
:1078F000401CA4F8220800200DE0B4F822581A5CBD
:10790000C5F30A0525442A75B4F82228521C401CE8
:10791000A4F8222880B28842EFDB47480078E8B319
:10792000A42084F81C0894F81F08800704D40220BF
:10793000607094F81E0860714048B4F822380288DC
:1079400045882A4000EB8202D38003884588B4F83A
:1079500020282B4000EB83031A8143885B1C9BB2D9
:107960004380A4F8222894F81C58A32D2ED0A725D4
:10797000C2F30A0222441575B4F82228521CA4F856
:107980002228B4F8225894F81E28C5F30A05254485
:107990005B1E2A759AB24280038800E012E0134011
:1079A00000EB8300C288A4F822280089A4F82008EC
:1079B00094F81C08A42803D094F81F08C0071CD012
:1079C00031B10BE0A32084F81C08B5E7A625CFE76A
:1079D00094F81F0820F0010084F81F0894F81D583F
:1079E000F02084F81D08FFF793F894F81F0840076B
:1079F00001D539F045FB84F81D58B4F820080B4A2E
:107A0000801CA4F82008D4F80A00B4F82418D2F88E
:107A10001C38084004EBC00000F50061C0F82A38AB
:107A2000D2F82008C1F82E00012070BDACD5072087
:107A3000E8000010F0CE0720CC00001004E307207F
:107A400010B509F097FC002800D0012010BD0000FF
:107A50002DE9F04188B006004FF000044FF02040BF
:107A60001E4FDFF87C801F4D0794009012D007A8AE
:107A700000F0C6F8000625D4079886420FD0912062
:107A800028606F2038607946C8F80010912008B04F
:107A9000BDE8F081CDF81640ADF812400BE0CDF80E
:107AA0001640ADF81240012E05D03146684600F070
:107AB000D1F9000606D4162201A900984AF098F8D8
:107AC000000601D52868E2E7074884702C603C6016
:107AD0007946C8F800100020D9E7000024C007202C
:107AE00028C0072020C00720600000102DE9F047C3
:107AF0008A4601461C481D4FDFF8748082781D4E6F
:107B000000244FF0050C42B11B4DC368D5F812504C
:107B100023F07042AA4209D38470C6F800C03C60CA
:107B20007946C8F800100520BDE8F08702F1640C22
:107B3000AC4501D8642500E0AD1A81462A461846B6
:107B40004AF028F8000601D53068EDE7CAF8005081
:107B5000D9F80C102944C9F80C1034603C607946FF
:107B6000C8F800100020DFE76000001024C00720E4
:107B700028C0072020C00720DACD07202DE9FC41CE
:107B8000044600254FF02040009549F0FBFF461EBB
:107B900001A96846266000F0AFF9144F000606D42C
:107BA00016221349009849F0F5FF000602D53868FF
:107BB000BDE8FC810E4A0099D38921F07040184439
:107BC0002368181A2C382060B04203D8080102D16B
:107BD000D08900B92660074885703D600648056079
:107BE0007846064908600020E2E7000020C0072030
:107BF000DACD07206000001024C0072028C007202D
:107C00007CB500240646009401A96846019400F062
:107C100073F90C4D000606D416220B49009849F062
:107C2000B9FF000601D528687CBD0198306007487F
:107C300084702C600648046078460649086000207D
:107C40007CBD000020C00720DACD072060000010B6
:107C500024C0072028C0072038B50146684600F038
:107C6000F9F8144C000606D416221349009849F07E
:107C700091FF000601D5206838BD0F490F4A104B0F
:107C8000D1F8125000200DB9C98959B10D49CD68FC
:107C90001635CD6001258D70206010607846186023
:107CA000002038BD812121601060784618600846A8
:107CB00038BD000020C00720DACD072024C00720EF
:107CC00028C00720600000102DE9F0439DB000247B
:107CD0000E4627461B94FFF7BFFF214D000635D403
:107CE000DFF88080DFF880901BA902A8FFF7FEFE76
:107CF00005281BD0318802AA20461B9B01F038FBC7
:107D000031881B9A1144318008B10446ECE714B164
:107D100020464BF05DFE91202860DC21C8F8001061
:107D20007946C9F800101DB0BDE8F083012000902D
:107D300001900E4B32882146A3F1100000F018FA92
:107D400014B120464BF044FE286808B12868EAE7E1
:107D50002F60C8F800707946C9F800100020E2E7EB
:107D600020C0072024C0072028C00720EACD072014
:107D70002DE9F043804689B01F46154689464FF0ED
:107D8000204049F0FFFE461E07A9684600F0B4F8FF
:107D90002C4C00064BD40098162240F0204001A93C
:107DA000009049F0F7FE000641D40E22414601A89A
:107DB000FEF714FAADF814700098ADF8125020F0E8
:107DC000704116312944CDF8161021F07041711A16
:107DD0001D4E1E4F491E2C35A94209D2912020600C
:107DE0006E20306078463860912009B0BDE8F0839D
:107DF000162201A949F0FCFE000618D40098BDF82F
:107E000012204946163049F0F3FE00060FD4DDF883
:107E10001600002540F020400090CDF81650ADF837
:107E20001250162201A949F0E3FE000601D5206890
:107E3000DBE70748857025603560784638600020AC
:107E4000D3E7000020C0072024C0072028C0072057
:107E5000600000102DE9F34F4FF0204487B08B46AF
:107E6000204649F08FFE471E00251F4EDFF87C801C
:107E7000DFF87C904FF0010ABBF1000F20D000BF6B
:107E800024F07040B8421BD216226946204649F0C1
:107E900081FE000603D5306809B0BDE8F08FDDF83B
:107EA000120040B1D34513D0DDF812000AF1010AE7
:107EB00040F02044E4E7BDF80E0008B1D34507D0F8
:107EC00081203060C8F800507946C9F80010E3E717
:107ED000079804600748C4603560C8F800507946C8
:107EE000C9F800100020D7E720C0072024C00720D1
:107EF00028C00720600000102DE9F34F83464FF0A3
:107F0000204587B0284649F03DFE461E204FDFF849
:107F10008490DFF884A001244FF0000825F0704021
:107F2000B04211D216226946284649F033FE0006B7
:107F300003D5386809B0BDE8F08FDDF8120058B1FC
:107F4000DDF81200000F1CD081203860C9F80080D5
:107F50007946CAF80010EDE7BDF80E0000B9641EBE
:107F6000CBF8005008980D490460DBF80000C860A9
:107F7000C7F80080C9F800807946CAF800100020D0
:107F8000D8E7DDF81200641C40F02045C6E7000089
:107F900020C0072024C0072028C007206000001050
:107FA0002DE9F0410025154F2E4600BF05EB450099
:107FB00000EBC50007EB4004D4F8120060B1204686
:107FC0000E21FEF733F9D4F8120018B14BF000FD82
:107FD000C4F812602682E6816D1C15F0FF05E5D01D
:107FE00007480670467007480660074806607846EE
:107FF000064908600020BDE8F0810000C4CD0720DC
:108000006000001020C0072024C0072028C00720DF
:108010002DE9FF4F394C89460146354FDFF8D480B2
:10802000354E0025A06883B09B464FF0910A012988
:1080300001D0D0B103E010B14BF0CAFCA5605B46A3
:10804000A188059AA06801F093F9A28802EB0B01C0
:108050008AB2A28068B1DFF8A8A00146A0609AF8B1
:108060000000C00615D5062014E0C6F800A0662062
:1080700007E0A06810B14BF0ABFCA560C6F800A00B
:10808000DC2038607946C8F80010912007B0BDE8C0
:10809000F08F0120CDE9009002AB194800F068F89C
:1080A00030B1A06810B14BF093FCA5603068EDE7EB
:1080B000B9F1000F14D09AF800108A060BD521F000
:1080C00020018AF80010A388BDF808200C48A16898
:1080D00000F0B6F818B1A06810B14BF079FCA560BB
:1080E00035603D607946C8F800100020CEE70000FA
:1080F00024C0072028C0072020C0072060000010EF
:10810000B6CD0720F0B5154C164E174F6478DFF842
:108110005CC004EB440505EBC405114C04EB4504BD
:108120000025D4F812E0BEF1000F0ED00460D4F8A0
:1081300012000860208A1080E089188035603D6058
:108140007846CCF800000020F0BD812030603D6012
:108150007846CCF800008120F0BD000060000010DF
:10816000C4CD072020C0072024C0072028C0072036
:10817000FEB504781A46DDE9083714F0030C134DF8
:10818000134E144C0AD0BCF1020F0BD0912020608A
:108190007A202860784630609120FEBD009736F046
:1081A000A7FF08E087780097CDE901234378B0F86E
:1081B00005200AF0D1F8000601D52068FEBD002098
:1081C00020602860784630600020FEBD24C0072073
:1081D00028C0072020C007202DE9F0418046014635
:1081E0000E221248FDF7FAFF11480024114E848038
:1081F0000E48114F114D807850B198F8000080065C
:108200000ED5FFF7CDFE00060AD52868BDE8F0813F
:108210009120286013203060784638609120F5E77F
:108220002C603460784638600020EFE7B6CD072038
:108230006000001024C0072028C0072020C00720AD
:108240002DE9F05F194C8A4601462078914600EBF3
:10825000400202EBC000164A9B4602EB4000154D5F
:10826000D0F81230144E154F43B191202860DC2015
:108270003060784638609120BDE8F09F90460E222D
:10828000FDF7ACFF207800EB400202EBC00208EBE8
:108290004200C0F812A0A0F81090A0F80EB0002084
:1082A00028603060784638600020E5E76000001004
:1082B000C4CD072020C0072024C0072028C00720E5
:1082C00030B587B00D4601A9034601220091114641
:1082D000022046F0ABFF0E4C000602D5206807B026
:1082E00030BD0598069A400705D504232946019814
:1082F00001F020FFF3E728460199FDF76FFF00200A
:108300002060044908607846034908600020E6E7D9
:1083100020C0072024C0072028C007202DE9F041F5
:1083200005468EB007A80C46012200902B46114648
:10833000022046F07BFF604E00067BD403A90C9818
:108340000094CDE9010101222B461146022047F09D
:1083500053F800066ED40B98400709D520460399C0
:108360001EF038FA20B920460C9A0799FDF736FF1F
:108370003B2D13D12078F4280BD006DC092808D037
:108380000A2806D0F32809D103E0F52801D0F62801
:1083900004D120460C9A0799FDF720FF0B98474F10
:1083A000DFF81C81C0062AD5A07800F00F01000973
:1083B00000EB800001EB400000F5FA60ADF8000032
:1083C000607800F00F01000900EB800001EB400035
:1083D0008DF80200207800F00F01000900EB80000A
:1083E00001EB40008DF80300684639F01FF9D8B35F
:1083F0002078A0BB607890BBA07880BB4CE00B9845
:10840000400732D5042301A920460C9A01F092FEC0
:1084100000060FD4042302A90C9A089801F08AFEE2
:10842000000607D4042369460C9A099801F082FEDD
:10843000000603D530680EB0BDE8F081DDE901012A
:10844000884202D30099884204D920460C9A0799A1
:10845000FDF7C4FE492D1FD1019801281CD12046EB
:108460000C9A0799FDF7BAFE16E00B9800071AD58B
:1084700000250EE00899605D495D884203D30999A3
:10848000495D884204D920460C9A0799FDF7A6FE5B
:108490006D1C0C98A842EDD80020306038607946F9
:1084A000C8F80010C7E7862030601220386079468F
:1084B000C8F800108620BEE720C0072024C007208F
:1084C00028C0072070B506468AB001A80D460122D3
:1084D000009033461146022046F0A8FE114C0006DB
:1084E00005D407A93046FFF719FF000602D520681A
:1084F0000AB070BD0598400706D5069B29461A4666
:1085000007A801F017FEF3E707A92846069AFDF72A
:1085100065FE002020600449086078460349086031
:108520000020E5E720C0072024C0072028C007203E
:10853000044900200860044908607846034908603F
:108540000020704720C0072024C0072028C0072033
:10855000411E1E2901D30020704701208840024996
:108560000968084070470000140000102DE9F0432E
:10857000411E8BB00A461E294BD2012404FA00F199
:1085800041F65063194244D0274D39B904FA02F13B
:108590006A680A436A602A6811432960DFF88C9090
:1085A000D9F80870461E6868B440044238D10DF10D
:1085B000200807AA082140468DE807000123721C05
:1085C00019460A2046F018FF18BB0798082820D142
:1085D00003A813F08FFAE0B9711C03AAC9B21448BA
:1085E0008DE8060150F836306038124950F83620D0
:1085F00045F6415004F04EFA0028286801D0204387
:1086000000E0A0432860D9F808000B49C01B88424D
:1086100003D300200BB0BDE8F08368682043686096
:1086200028682040F6E70000140000100000094010
:10863000485C0500776BD00580969800411E1E2986
:1086400006D2012101FA00F241F650631A4201D12B
:1086500000207047401E8140024842688A434260C1
:10866000012070471400001010B501242046FFF7C8
:10867000E5FF641C1E2CF9DD10BD00002DE9F04F54
:10868000834685B00D464FF0C04049F07BFAA0F11B
:10869000010904A9684600F011FB3B4C000667D4B1
:1086A000092201A9009849F075FA000660D4DFF8A4
:1086B000DCA0019850B140F0C0400090092201A90F
:1086C000CAF8040049F066FA000651D4BDF8080063
:1086D0002F4E304FA0F57061FF3910D09DF80C106F
:1086E0004FF00008A9421AD088B1862020600920E6
:1086F000306078463860862005B0BDE8F08F912064
:10870000206013203060784638609120F4E7012023
:108710008DF80C50ADF80800CDF8048002E0401C44
:10872000ADF80800BDF808000099401E093100FBB3
:10873000051020F07041294409310090494507D9BE
:1087400089202060C6F80080784638608920D3E709
:108750002A46594649F04CFA000609D4DAF80400D2
:108760005546092201A9009049F042FA000601D5B8
:108770002068C1E785F80080C4F80080C6F8008052
:10878000784638600020B7E720C007205800001066
:1087900024C0072028C007202DE9F04186B005003D
:1087A0004FF000044FF0C0401C4FDFF874801D4EA6
:1087B0000494009012D004A800F014F9000622D40A
:1087C000049885420BD0912030606F203860794644
:1087D000C8F80010912006B0BDE8F0810125ADF881
:1087E000084001948DF80C40012D05D029466846BB
:1087F00000F014FA000606D4092201A9009849F0F5
:10880000F7F9000601D53068E5E7074804703460E1
:108810003C607946C8F800100020DCE724C007203F
:1088200028C0072020C00720580000102DE9FF4174
:1088300004460146684600F041FA1E4D000633D456
:108840001D4E1E4F2068002440B1092201A9009846
:1088500049F0A0F9000627D4019838B12C603460A3
:1088600078463860002004B0BDE8F08100989DF89B
:108870000C2020F07041BDF80830093102FB0311D3
:108880000191092201A949F0B3F900060CD401981D
:10889000ADF8084040F0C040CDE90004092201A92C
:1088A00049F0A6F9000601D52868DCE70448047001
:1088B000D4E7000020C0072024C0072028C00720DC
:1088C000580000102DE9FC4105464FF0C04049F02A
:1088D00059F9441E01A968462C6000F0EFF9164EC4
:1088E000000606D409221549009849F053F90006FC
:1088F00002D53068BDE8FC811048009A037A878869
:1089000022F0704103FB07112B68591A12392960B4
:10891000A14205D8110104D1017A8088414300D1D8
:108920002C600749002008703060064908607846CE
:10893000054908600020DDE720C00720280400105A
:108940005800001024C0072028C007202DE9F04758
:108950001F4B8146002418781E4E1F4F1F4D8A461C
:10896000052268B11E49D1F800C05FEA1C700DD025
:10897000812028603460784638608120BDE8F08727
:108980002A603460784638600520F7E7586820F0A0
:108990007048E04501D31C70F2E788460A7A4946E0
:1089A000994649F0F7F8000601D52868E6E798F8F7
:1089B0000820CAF8002098F80810D9F804201144BB
:1089C000C9F804102C603460784638600020D5E780
:1089D0005800001024C0072028C0072020C007200E
:1089E000280400107CB5054601A9684600F066F928
:1089F000104C000606D409220F49009849F0CAF825
:108A0000000601D520687CBD0B480C4A0021036894
:108A100023B9808810B10120507000E05170019896
:108A20002860117021600648016078460549086099
:108A300000207CBD20C00720280400105800001032
:108A400024C0072028C0072038B50146684600F03A
:108A5000E5F8154C000606D409221449009849F09F
:108A600099F8000601D5206838BD1048104A114B0E
:108A7000056800216DB100250F484570456809352E
:108A8000456001250570216011607846186000205E
:108A900038BD808808B10125EEE781202060116093
:108AA00078461860812038BD20C0072028040010B7
:108AB00024C0072028C00720580000102DE9F043EB
:108AC00000248FB0984691462546124ECF080E944A
:108AD00011E06B46012138460E9A29F055FD00063B
:108AE00003D530680FB0BDE8F0836D1C4D4502D34F
:108AF000B8F1000F05D00EA96846FFF727FF002840
:108B0000E7D03460044804607846044908600020D7
:108B1000E8E7000020C0072024C0072028C0072065
:108B200010B5FFF791FF0106064801D5006810BD9A
:108B30000021016004480160784604490860002073
:108B400010BD000020C0072024C0072028C0072037
:108B50002DE9F0438FB02C4F002406460E94388840
:108B600015468946401E2AF0BBFA80463046FFF77C
:108B70006BFF264E000645D42549FA89254F087A11
:108B800002FB08F209EBC00CDFF88C8094450AD98F
:108B900091203060132038607946C8F80010912089
:108BA0000FB0BDE8F083AA0703D58988012236F00B
:108BB000C3F94FEAD9090EA96846FFF7C7FE002896
:108BC0004FEA85700ED0002805DAE80703D036F0AA
:108BD0009BF936F0C9F934603C607946C8F800105A
:108BE0000020DDE7002803DA0121684636F068F945
:108BF000012DE0D16B46012148460E9A29F0C4FCB4
:108C00000006D8D53068CBE73204001020C007201A
:108C10002804001024C0072028C007202DE9F34FA6
:108C20004FF0C04483B08B46204648F0ABFF471E50
:108C300000251E4EDFF87880DFF878904FF0010AAB
:108C4000BBF1000F1ED000BF24F07040B84219D213
:108C500009226946204648F09DFF000603D530688A
:108C600005B0BDE8F08F009838B1D34512D0009818
:108C70000AF1010A40F0C044E6E7BDF8040008B17B
:108C8000D34507D081203060C8F800507946C9F834
:108C90000010E5E703980460074844603560C8F8B1
:108CA00000507946C9F800100020D9E720C00720FD
:108CB00024C0072028C00720580000102DE9F34FDA
:108CC00007464FF0C04485B0204648F05BFF461E83
:108CD000DFF88480DFF884A0DFF884B001254FF04E
:108CE0000009009424F07040B0420FD2092201A97B
:108CF000204648F04FFF000604D5D8F8000007B022
:108D0000BDE8F08F019850B1000F1ED08120C8F847
:108D10000000CAF800907946CBF80010EFE7BDF8E4
:108D2000080008B13C6002E000986D1E38600698AB
:108D300005600C4839684160C8F80090CAF8009096
:108D40007946CBF800100020D9E70198009440F054
:108D5000C0446D1CC6E7000020C0072024C00720C7
:108D600028C00720580000102DE9F04180468AB045
:108D70000D7802A80F4601220090002443461146B8
:108D8000022046F053FA104E000611D408AA2846D5
:108D90002146079B01F0B0FD000609D4CDE900741F
:108DA000012243461146022046F0FEFC000603D590
:108DB00030680AB0BDE8F081346004480460784649
:108DC000034908600020F4E720C0072024C00720E2
:108DD00028C007201CB50024CDE900140346012259
:108DE0001146022046F0E0FC0106064801D5006865
:108DF0001CBD0460044804607846044908600020F3
:108E00001CBD000020C0072024C0072028C0072068
:108E10002DE9F74F92B0144610A819F093FC2F4D8E
:108E2000000649D49DF84000DFF8B480DFF8B49024
:108E30008827B0B10607304648F0A4FE2A4A401EF3
:108E40004FF0000A51680B195B1D98420ED22F603B
:108E5000C8F800A07946C9F80010882015B0BDE810
:108E6000F08F2F600A21C8F80010F3E746EA0107E7
:108E70008DF800401298ADF8010093466E462246E8
:108E8000F01C1399FDF7AAF93019FF21C470017184
:108E9000221D711C781C48F0ABFE00060CD4092082
:108EA000B0EB177F01D1621D00E001226946384610
:108EB00048F09EFE000601D52868CFE7DBF80410D5
:108EC0002144091DCBF80410C5F800A0C8F800A083
:108ED0007946C9F800100020C0E7000020C0072034
:108EE00024C0072028C00720300000102DE9F047DB
:108EF0008A46064641880088141D091A124FDFF879
:108F00004C80DFF84C90A14209D2862038600921BC
:108F1000C8F800107946C9F80010BDE8F0877168FC
:108F20000D18281D6A801946FDF758F9A5F800A00C
:108F300030882044308000203860C8F8000079462E
:108F4000C9F80010E9E7000020C0072024C007206E
:108F500028C007200170427070470000F0B589B04A
:108F600006460024ADF800401420ADF8020003A826
:108F70000D4601901F46042102A820F066FC02461F
:108F800002AB01216846FFF7B1FF3A46042102A86F
:108F900020F05BFC024602AB02216846FFF7A6FF09
:108FA000BDF80020A9B23046019BFFF79FFF05489E
:108FB00004600548046078460449086009B0002050
:108FC000F0BD000020C0072024C0072028C00720D3
:108FD0000448016F11B1491C01677047022101204B
:108FE00043F004BC04C307202DE9F0439DB0814643
:108FF000DDE924780024ADF804406420ADF80600D3
:10900000164603A80A4602901D4604211CA820F01B
:109010001CFC02461CAB032101A8FFF767FFAAB2A4
:109020003B46042101A8FFF761FF424604211CA82A
:1090300020F00BFC02461CAB052101A8FFF756FFF0
:10904000BDF80420B1B24846029BFFF74FFF054828
:109050000460054804607846044908601DB000209B
:10906000BDE8F08320C0072024C0072028C00720C7
:109070002DE9FF4F8BB04FF0000B0746ADF804B061
:109080004068424EDFF80881424D1C468A46C8B10E
:1090900005A950463DF006FF00063BD49DF815207B
:1090A00021460D9802F05AFEADF80400021E09D0C8
:1090B000798838880B1A111D8B4207D286202860C8
:1090C000162042E088202860584659E079680C183C
:1090D0009DF8150004F104090C284ED2DFE800F0D9
:1090E0004D0606060B1406060606060648460D99AA
:1090F000FDF774F805E001AA49460D9801F08CFCD3
:1091000000BBBDF8040026E004A950463DF03AFF3C
:10911000000603D528680FB0BDE8F08F9DF8101049
:1091200089F8001001AB09F1010248460D9901F0E0
:109130000DFC38B9BDF80400401C80B2ADF8040045
:10914000082808D986202860092030607946C8F8A8
:1091500000108620DFE76080A4F800A0BDF80400BE
:109160003988001D08443880C5F800B0C6F800B042
:109170007946C8F800100020CDE788202860092033
:1091800030607946C8F800108820C4E724C0072062
:1091900028C0072020C007202DE9FE430F46804647
:1091A000ADF8082002AA6946184601F035FC0F4DBB
:1091B0000F4E104C40B18620206009202860784670
:1091C00030608620BDE8FE836B46BDF80820394636
:1091D0004046FFF78BFE000601D52068F2E700202D
:1091E00020602860784630600020EBE724C007202C
:1091F00028C0072020C00720416851B1084A926862
:109200000368D21A01EB4103C3EBC111B2EBC10FEA
:1092100001D200207047002141600120704700000A
:109220000000094041600249896801607047000000
:10923000000009402DE9FC5F0F46044600884A49BA
:10924000DDE917B6401A80B25FEA000822D0DFF8E5
:109250001C914146B9F80E00B0FBF6F26846521C6C
:10926000FCF7B2FF019D002D7BD04FF00A0ABBF145
:10927000010F12D0BBF1020F26D0B9F80E102068F2
:10928000B1FBF6F2401B0244BA424CD2B1FBF6F1FC
:10929000084449E00120BDE8FC9FB9F80E00C8F57C
:1092A000A572B0FBF6F1491B891C914256D8B0FB60
:1092B000F6F0401B85B2202229462068FCF7AFFF5C
:1092C00020682844206047E0B9F80E202168B2FBEE
:1092D000F6F3481B381A834201DAB2FBF6F080B28B
:1092E00085423BDA401B86B201EB5600411B05E08C
:1092F0002268521E2260127800F8012D8142F7D3B5
:1093000020682022091AFCF78AFF2068A6EB560184
:10931000284400EB56000D4620222060FCF77FFF1A
:109320002068284415E03846411B05E02268521E9B
:109330002260127800F8012D8142F7D320682022A4
:10934000091AFCF76CFFB9F80E002168B0FBF6F0C3
:1093500008442060B84201D280F800A02068401C78
:109360002060002097E700006CCC0720320400103A
:109370002DE9F0411F469046002400B10C46E61945
:10938000711C4BF0B3F8050009D028193A46414644
:10939000FCF724FF0020A8552846BDE8F0810020F6
:1093A000FBE70000F8B51B4E02271B4C0025684662
:1093B00002F0C8F90006306816D405280DD09DF8D3
:1093C0000000A071FDF796FCB52815D0B6280CD08A
:1093D000B72819D0FDF79CFB0AE035600F480560FF
:1093E00078460F4908600020F8BDA079FE2801D01A
:1093F000257009E0277007E0A079FE2808D02570C5
:1094000094F81D08FDF744FC9DF80000E070CEE7DD
:109410002770F5E720C00720ACD5072024C007201F
:1094200028C007202DE9F0410D480E4D0E4E407822
:109430000E4F002408B1022804D1012002F09CF94B
:10944000052806D02C603460784638600020BDE8DE
:10945000F081052028603460784638600520F6E702
:10946000ACD5072020C0072024C0072028C0072033
:1094700070B5114C0025607898B1012811D1A07801
:10948000012610B102280CD105E02671FEF73CF947
:1094900038B1A67004E02671A570FEF7B3F900B1EB
:1094A000257106482571056005480560784605491F
:1094B0000860002070BD0000ACD5072020C0072048
:1094C00024C0072028C0072010B51348002440F20C
:1094D000FF71047104704470847044820482C181FD
:1094E000A0F82848A0F826487F21A0F824180B48A7
:1094F0000F2144808480018034F0F8FE0106084882
:1095000001D5006810BD046006480460784606492D
:109510000860002010BD0000ACD5072004E3072040
:1095200020C0072024C0072028C007202DE9F041D3
:1095300009480A4E0A4F00790A4D002430B9FFF756
:1095400031FF000602D52868BDE8F0812C60346048
:10955000784638600020F7E7ACD5072024C0072004
:1095600028C0072020C007200D4810B581780D4C79
:1095700001290BD10221817034F0D2FE000603D400
:10958000FFF776FF000601D5206810BD002020609F
:1095900005490860784605490860002010BD0000B4
:1095A000ACD5072020C0072024C0072028C00720F2
:1095B00070B5164C012529462571A8204BF0A4F959
:1095C000C4F80A00411C0AD0B4F82428A221104093
:1095D00004EBC00080F82A180220A07065700020FB
:1095E0002071D4F80A400A490A4A0B4B641C05D082
:1095F0000860106078461860002070BD05240C607B
:10960000106078461860204670BD0000ACD5072079
:1096100020C0072024C0072028C007200D4810B50F
:1096200081780D4C01290BD10221817034F0A0FF0B
:10963000000603D4FFF71CFF000601D5206810BD0B
:109640000020206005490860784605490860002030
:1096500010BD0000ACD5072020C0072024C0072083
:1096600028C007200549052008600549002008603A
:1096700078460449086005207047000020C0072094
:1096800024C0072028C00720064A39B1012904D187
:10969000B2F811100180D17C81707047D1890180AE
:1096A000117CF9E7A803001021B1012901D1034978
:1096B000887070470149C91EFAE70000B90300101D
:1096C00010B50021064A08462BF0EAF80548018843
:1096D00041F002010180BDE8104001202BF0A6BE40
:1096E000C574050018C0072070B586B0054600880F
:1096F00069463DF0D7FBBDF804000F4CC00511D5FD
:1097000028463CF0DBFB0D4E000601D5022005E0AB
:1097100028463DF083FE000604D50320B070206883
:1097200006B070BD002020600549086078460549F4
:1097300008600020F4E7000020C00720B9030010F3
:1097400024C0072028C007202DE9F8430420FEF795
:10975000FFFE174F174C184D184E07F103084FF036
:10976000A60920B11648007818B1052016E004209B
:1097700014E0684619F0ECF99DF8000008B10620E5
:109780000CE0012015F034FB38B100202060286087
:10979000784630600020BDE8F8830720B87088F86C
:1097A0000200C4F80090286078463060A620F2E7F6
:1097B000B603001020C0072024C0072028C00720BF
:1097C0009CC207202DE9F34F62480024ADF5257DAA
:1097D00000788B46800725464FF001070AD440F2F7
:1097E0004D40ADF80000ADF802708DF804506846A9
:1097F0003DF014FE1B2181A8FCF718FD1B218FA84A
:10980000FCF714FD54480DF50F79B0F87E01B8B996
:10981000524B40F2FD364122991C30463DF0B6FCD9
:10982000010640F2B34005D5ADF83C62ADF83E020A
:10983000022405E0494900230C2244313DF0A6FCF6
:1098400040F2C5469DA930463DF028FDBDF87402A2
:1098500040B9ADF80060ADF802708DF8045068466C
:109860003DF0DCFDADF804624FF484680DF5017A3B
:1098700001269DA940463DF011FDBDF87402A8B92E
:109880009DAB01229FA940F2EA303DF07FFC9DF89C
:109890007C0210B18DF8045001E08DF80470ADF831
:1098A0000080ADF8027068463DF0B8FD9DAB012226
:1098B0009FA940F2EA303DF069FC0022A0A99EA8D1
:1098C00018F05CFB264F000621D538680DF5277D82
:1098D000BDE8F08F9DA93DF0E1FCBDF874020028C1
:1098E0009E9808D001882AF81610761CF6B29E9829
:1098F000801D9E900CE09DF88012014489784907F4
:10990000F5D5008829F81400641CE4B2EFE79E98AE
:1099100000880028DED1314681A84BF0C9FABBF19E
:10992000000F0DD00122314681A800F067F8002118
:109930000CA028F067FE002221468FA800F05EF8F8
:10994000A59804803D60094805607846084908608C
:109950000020BBE721C5072020F207209EF3072047
:1099600020C00720202020202000000024C0072045
:1099700028C0072002480021A0F81110C1747047C8
:10998000A80300103EB50546184CA0F580602138AC
:1099900013D040F2FF31684611F080FC02AA6946FC
:1099A00028463DF0EFFC000614D40198011D028802
:1099B000A2F580634D3B08D105E000210C4A084622
:1099C0002AF06EFF08E00A7832B1006811F0E6FC78
:1099D000000601D520683EBD0020206005490860D2
:1099E00078460549086000203EBD000020C00720E1
:1099F0004489050024C0072028C007202DE9F05F16
:109A0000DFF89CA0DFF89CB00E00054617464FF02B
:109A100000083AD0DFF89090012EC9F8005009D024
:109A2000C7B10021214A08462AF03AFF2888FFF7EB
:109A3000A9FF14E042B100211D4A08462AF030FF78
:109A40002888FFF79FFF20E000211A4A08462AF0E5
:109A500027FF1AE00021184A08462AF021FF0124B6
:109A600011E000BF05EB4401C9F8001027B135F83B
:109A70001400FFF787FF04E00021104A08462AF08F
:109A80000FFF641CE4B2B442ECD3CAF80080CBF8F8
:109A9000008079460A4801600020BDE8F09F000080
:109AA00020C0072024C0072030C507202E730500E2
:109AB00018730500367405004473050065730500CE
:109AC00028C007202DE9FF470024ADF800400E20F4
:109AD00015F08EF9364E374F374D002861D0FFF71D
:109AE00033FE00065DD40E2003F0B8FF3348DFF8E4
:109AF000D0A0007880071BD58DF8044003AB01226D
:109B000001A940F24D403DF041FB000649D49DF8CB
:109B10000400E0B301216846FFF754FEBAF80010D4
:109B200041F00201AAF8001001202BF07FFC03E0B5
:109B300000216846FFF746FEBDF8000038BB02A9C9
:109B40008D20FEF7EBFB000603D5286804B0BDE8C6
:109B5000F0879DF80800DFF86C804FF001090128BC
:109B600002D002281DD118E00021174A08462AF029
:109B700097FEBAF8001041F00201AAF80010012087
:109B80002BF054FC88F80190104A926800E008E03D
:109B9000C8F8302088F8029003E000F019F888F83F
:109BA00002902C603460784638600020CEE70000D8
:109BB00024C0072028C0072020C0072021C5072077
:109BC00018C00720A8030010E1720500000009403A
:109BD00010B50D2040F02CFD12F0D6FA000609D485
:109BE00040F2FD303DF01CFBBDE8104040F2B340B8
:109BF0003DF016BB0D2003F045FF00210A20FFF7C2
:109C000053FD0121BDE810400A20FFF74DBD0000C3
:109C10002DE9F0471D46294F294CDFF8A88013464F
:109C20000E464FF00009012807D02089884227D02E
:109C300004F11101092088701AE022482681401C95
:109C40002062A4F80A902A461946FCF7C7FAB8F829
:109C50000320291F40468A420DD8B0F80110B142B6
:109C600021D100BF08F10100FFF73EFD00061AD523
:109C70003868BDE8F087206A28442062618112E0DC
:109C80002A461946206AFCF7A9FA206A284420626D
:109C90006089284481B26181B1F5807F03D8B8F82A
:109CA00003208A42DED0C7F800900749C1F800902F
:109CB0007846064908600020DBE7000020C0072046
:109CC000A8030010A8F5072024C0072028C00720FB
:109CD0002DE9FC4799468A46082A22D80AB3002172
:109CE000CDE90011012100236FF00108841814F858
:109CF000016C06F00F04092C10DCA1FB045CE70FDB
:109D000003FB04C401FB0744DDE900C71CEB0505A8
:109D10006741CDE900573509092D05DD4046BDE80D
:109D2000FC874FF0FF30FAE70A27A1FB074C03FB43
:109D300007C3002601FB0633A4FB0517EE1703FB40
:109D4000057504FB0655DDE9007679186E41CDE90D
:109D500000160A26A4FB0617002503FB067304FB66
:109D60000533521EC2D14FEAC90101208840DDE906
:109D70000023401EC117801A994101D2E81ECEE788
:109D80004A4669465046FCF729FA0020C7E708B55D
:109D9000027802F00F03120902EB820203EB420287
:109DA0008DF80220427802F00F03120902EB8202C2
:109DB00003EB42028DF80120807800F00F020009C9
:109DC00000EB800002EB40008DF80000684600F0D8
:109DD00033F808BD0278407802F00F03120902EB55
:109DE000820203EB420200F00F03000900EB800047
:109DF000D2B203EB4000C0B2C2EB021200EB820011
:109E00000880704770B515467BB15C1E08D4094EBA
:109E100064220023FCF772F9B25C2A55641EF7D560
:109E2000084305D06FF0010070BD4FF0FF3070BDEA
:109E3000002070BD4E5B050010B5027840F26D1336
:109E40005A430A8043780C4C34F813301A440A8081
:109E500083781A4493B20B800278940705D1407836
:109E6000022802D803EB920003E0012000EB9200ED
:109E70001844088010BD0000CC5B050008B50288BE
:109E8000B2F5FA6F0ED3C2788DF8022082788DF881
:109E900001200078A0F5FA608DF800006846FFF711
:109EA000CBFF08BD0020088008BD000010B5040EDF
:109EB000C0F30743A0F5FA60C2B20448045D0C7019
:109EC000C35C4B70805C887010BD00004E5B050069
:109ED00000B90120044BC1EB0111584300EB810094
:109EE00002490844106070478051010000F26B384D
:109EF00018B50C46694600F02BF89DF8021006488C
:109F0000415C21709DF80110415C61709DF800106A
:109F1000405CA07018BD00004E5B05001CB50C46EF
:109F200001A900F015F89DF8040000909DF8053097
:109F30009DF8062002A1204648F0B4F91CBD00009F
:109F4000253032752E253032752E253032750000C1
:109F500030B500B90120401E80B240F2B553B0FBCD
:109F6000F3F2B0FBF3F403FB14009206401C120E54
:109F700080B24FF4B77398420BD9521CD2B2A0F5FD
:109F8000B77003E0521CD2B2A0F26D1080B29842BA
:109F9000F8D2202801D2012318E01F3880B293079D
:109FA00001D01C2300E01D23984201D802230DE0BC
:109FB000C01A80B20023074D03E0001B5B1C80B277
:109FC000DBB2EC5C8442F8D3DB1CDBB20A704B7072
:109FD000887030BDC25B050018B50C466946FFF7B6
:109FE000B7FF9DF80200E0709DF80100A0709DF899
:109FF000000000F5FA60208018BD3C22B0FBF2F3AF
:10A000000B70B0FBF2F302FB130048700020887065
:10A010007047C0F30722C0B2C0EB001002EB800013
:10A0200008807047044AC3B2C0F30720D35C0B70AA
:10A03000105C4870704700004E5B05003C2310B573
:10A04000B0FBF3F2B0FBF3F403FB1400034BD2B20A
:10A050009A5C0A70185C487010BD00004E5B0500E9
:10A0600030B50C460E49884202D34942084400E00C
:10A0700000200C49B0FBF1F2B0FBF1F301FB13003F
:10A080003C21B0FBF1F092B285B221461046FFF7B9
:10A09000A3FF211D2846BDE83040FFF7AEBF0000FA
:10A0A00000F26B38805101000A4B10B5984202D380
:10A0B0005B42184400E00020074BB0FBF3F40C8037
:10A0C000B0FBF3F103FB11003C21B0FBF1F0108079
:10A0D00010BD000000F26B388051010070B5002403
:10A0E000064604250220FCF7F3FCC0F38910044463
:10A0F0006D1EF7D14FF4A5704443230B0A480B495A
:10A100000B4A3360DC2B07DA8223036011200860DE
:10A1100078461060184670BD002303600B607846D7
:10A120001060184670BD000020C0072024C0072022
:10A1300028C0072010B5FFF7CBFD1549154A164B6F
:10A1400010F1030F1CD010F1020F11D0B0F1FF3F3E
:10A1500006D000200860106078461860002010BD0E
:10A16000882008600920106078461860882010BD9B
:10A17000862008602020106078461860862010BD78
:10A18000892008600420106078461860892010BD7E
:10A1900020C0072024C0072028C007202DE9F04F49
:10A1A00088460021204D214E214F82464FF08609DE
:10A1B000B3EB420F16D3012020E000BFA2EB000B4F
:10A1C0001AF80B4004F00F04092C0BDCA3EB400E33
:10A1D0000EEB080C30348CF801401AF80B402409BF
:10A1E000092C07DDC5F8009031607846386086207C
:10A1F000BDE8F08F303408F80E40401C9042DDD9A5
:10A20000012000EB4200302205E000BFA3EB000C70
:10A21000401C08F80C209842F8D929603160784633
:10A2200038600020E4E7000020C0072024C0072099
:10A2300028C0072010B14FF0FF3070470248406D32
:10A2400040F3C020401C704700C0092008B501221F
:10A250006946034847F09EFC9DF8000008BD0000D9
:10A2600028000020502000F0AFF84FF46175C8219D
:10A27000284600F039FA0E4CA1684CF25030A26822
:10A28000521A8242FBD3C821284600F02DFAA0685A
:10A290000849A268121A8A42FBD307480168074A94
:10A2A00001F4E06111430160BFF34F8FFEE700004E
:10A2B00000000940400D03000CED00E00400FA0529
:10A2C00010B5FFF7C3FF502805D0522808D05328F7
:10A2D00006D1552000E04420BDE8104000F074B8DD
:10A2E00010BD00002DE9F047354C4FF4FA69608845
:10A2F000484501D2401C6080324E706D4FF480376B
:10A3000000054FF4FA784FF000052ED4A580207890
:10A3100010B96078401C6070608840451AD9607838
:10A32000012817D141F0EAFEA0B941F0DBFE10B1DF
:10A3300001280FD107E0B7636088B0F57A7F09D1B3
:10A3400001F022FA06E0608840F2DC51884201D92F
:10A35000FFF788FF6078022803D16570012028F09C
:10A3600085FE01202070BDE8F087022028F07EFEE7
:10A37000A088484501D2401CA08061884FF4E17359
:10A38000414502D880B298420DD16078012801D1B0
:10A39000414502D8A088984203D141F0AFFE00B9F0
:10A3A000F763657009E06178012906D1B0F5967F01
:10A3B00003D141F0A3FE00B9B76365802570D2E7F1
:10A3C0004801001000C0092001B501226946024879
:10A3D00047F00EFC08BD0000280000200B488068F4
:10A3E0000B49CA68801A0A6902EB4203C3EBC21226
:10A3F000B0EBC20F08D3074802224260C26B02F0E2
:10A40000FD02C2630020086170470000000009409F
:10A4100078010010008000402DE9F843012027F06A
:10A4200015FE0227304EDFF8C480DFF8C490314CAF
:10A43000002578B3D8F8000082284BD1D9F8001055
:10A4400048460A2902D000680E2843D16946612097
:10A45000FEF738F89DF8000080073BD500F060F863
:10A4600060BB254988686268801AA26802EB4203D3
:10A47000C3EBC212B0EBC20F2CD32068C2070AD0C4
:10A480007760F26B02F0FD02F263256111280DD2B4
:10A49000FA200DE013E011284FF0FA0101D2480034
:10A4A00001E04FF4FF7000F0BFF804E042F21070DA
:10A4B000A060886860602068401C20600AE0206816
:10A4C00040B125606560A5607760F06B00F0FD002D
:10A4D000F0632561C8F80050C9F800507846074974
:10A4E00008600020BDE8F8830080004020C00720FD
:10A4F00024C00720780100100000094028C0072070
:10A5000008B569466120FDF7DDFF9DF80000C00732
:10A5100004D0FA2140F2262000F086F808BD0000A1
:10A5200030B50F4881680F48114BC26800698C1A1A
:10A5300000EB4001C1EBC01500200B490B4AB4EB06
:10A54000C50F06D205240C601060784618602046BE
:10A5500030BD0860106078461860002030BD0000F3
:10A56000000009407801001020C0072024C0072007
:10A5700028C007200B4900200867C86010224A61E4
:10A580008861C022CA6308498A680849C1E9032072
:10A5900007490860074908607846074908600020B5
:10A5A0007047000000800040000009407801001062
:10A5B00020C0072024C0072028C0072038B56946DE
:10A5C0006120FDF77FFF9DF80000144C40071CD56B
:10A5D0003221080100F088F8000614D4322140F23C
:10A5E000EF3000F081F800060DD4322140F2AE4089
:10A5F00000F07AF8000606D4322140F2E65000F06E
:10A6000073F8000601D5206838BD00202060044999
:10A610000860784603490860002038BD20C0072044
:10A6200024C0072028C007202DE9F04341F28832DA
:10A630000023264C264D274E904208D8642800D28D
:10A6400028B942F21072914201D8052907D286201A
:10A6500020602B60784630608620BDE8F083DFF80C
:10A660007890D9F80820DFF87480D8F80C70D21BE5
:10A67000D8F8107007EB470CCCEBC717B2EBC70F3D
:10A6800006D2052020602B60784630600520E4E784
:10A69000134A02275760D2F83CC00CF0FD0CC2F8F8
:10A6A0003CC040B1DFF83CC0BCFBF0F04010D061D2
:10A6B000576001205060D9F80800C8E90301236001
:10A6C0002B60784630600020C7E7000020C00720DC
:10A6D00024C0072028C0072000000940780100108E
:10A6E0000080004080A8120170B50F4C00250E4676
:10A6F0002561FFF799FF0D49000601D5086870BD77
:10A700000B4B06EB4602E068C2EBC6129E68361A97
:10A71000B6EBC20FFAD3074802224260C26B02F0C6
:10A72000FD02C2632561E9E77801001020C007201F
:10A73000000009400080004010B5044600BF04201E
:10A740003FF0D8FE00F0800010B10748006810BD4F
:10A7500000BF00BF04490020086004490860784633
:10A76000034908600020F2E720C0072024C007202A
:10A7700028C0072070B52E4B0A4600BF12F8014BC7
:10A780001C5D3F2CFAD9521A941CE51704EB957402
:10A79000A41004EB4404521E21E000BF11F8015B39
:10A7A00011F8016B5D5D9E5DAD0045EA161500F880
:10A7B000015B11F8015C11F8026B5D5D9E5D2D017E
:10A7C00045EA960500F8015B11F8015C11F8026C8E
:10A7D000121F5D5D9E5D45EA861500F8015B042A47
:10A7E000DCDC012A08DD0D784E785D5D9E5DAD00F4
:10A7F00045EA161500F8015B022A08DD4D788E78CF
:10A800005D5D9E5D2D0145EA960500F8015B032A1A
:10A8100007DDCD7889785D5D595C45EA811100F8E6
:10A82000011B00210170504200F00300201A70BD8E
:10A83000806F0500F0B5002304462E4D971E27E0DB
:10A84000CE5C05EB9606367804F8016BCE5CB60755
:10A850004FEA966CCE18DB1C96F801E04CEA1E1C01
:10A8600015F80CC004F801CB96F801C096F802E088
:10A870004FEA0C7C4FEA9C6C4CEA9E1C15F80CC00D
:10A8800004F802CBB67806F03F06AE5D04F8016C22
:10A89000BB42D5DB934227DACE5C521E05EB96060F
:10A8A000367804F8016B3D2693420AD1C95C01F069
:10A8B000030105EB0111097804F8011B04F8016B91
:10A8C00010E0CA5C194492074B78920E42EA1312C8
:10A8D000AA5C04F8012B497801F00F0115F821104A
:10A8E00004F8011B04F8016B002104F8011B201A75
:10A8F000F0BD00008070050010B5FFF783FA104925
:10A90000104A114B10F1020F11D0B0F1FF3F06D0E9
:10A9100000200860106078461860002010BD882074
:10A9200008600920106078461860882010BD8920D2
:10A9300008600420106078461860892010BD00006F
:10A9400020C0072024C0072028C007202DE9FC5F75
:10A950000026CDE9006693468246994601251A886D
:10A960006846FBF73BFC00209AF800400AE00A2307
:10A97000A5FB0327002106FB037305FB0136401CE2
:10A980001546C0B28442F2D8DDE900012A463346BA
:10A99000FBF7B4FB1646984607460D460BE00A2225
:10A9A000002330464146FBF7A9FB1A4305D1641E3C
:10A9B00006468846E4B2002CF1D18AF80040002017
:10A9C0000AE00A23A7FB031C002205FB03C307FBC5
:10A9D0000235401C0F46C0B28442F2D8B91945EB8B
:10A9E0000805CDE900150821A9F800104A46594686
:10A9F000684600F011F80549002008600449086025
:10AA00007846044908600020BDE8FC9F20C007206C
:10AA100024C0072028C007202DE9F0410B461188EB
:10AA200000271A4C1A4D1B4E8446082902D809B13A
:10AA3000002012E0862020601520286078463060D3
:10AA40008620BDE8F08100BF1CF800E0BEF1000FD9
:10AA500008D000271180401C80B28842F4D31088AF
:10AA600028B106E0002FF6D110800127F3E701207E
:10AA7000108082B261461846FBF7B0FB00202060D0
:10AA80002860784630600020DBE7000020C0072007
:10AA900024C0072028C007202DE9F04190B0224EA5
:10AAA00040216846FBF7C2FB20226946304647F04A
:10AAB00071F81E4D000629D4202269461C48FBF778
:10AAC00005FC38B3002441F20C1741F2542800BFB2
:10AAD00007EB441040F0E0402022694647F05AF866
:10AAE000000613D408EB841040F0E0404022694691
:10AAF00047F07EF8000609D4641C082CE8DB3046D9
:10AB000020220B4947F074F8000603D5286810B0DE
:10AB1000BDE8F081002028600649086078460649B3
:10AB200008600020F3E700000C11007020C007202F
:10AB3000E170050024C0072028C007203EB500258D
:10AB40008DF8045001A902A841F014F8114C000638
:10AB500015D49DF80800012813D11CF0DDFE01205A
:10AB6000034600220146009026F0B6FA000606D4FD
:10AB700001A840F0FBFBFFF78FFF000601D520681E
:10AB80003EBD256004480560784604490860002001
:10AB90003EBD000020C0072024C0072028C0072099
:10ABA0002DE9F04104000E464FF0FF370DD0084666
:10ABB00047F0D0FB050008D0606808B148F008FFF6
:10ABC000C4E900650020BDE8F0813846FBE72DE9C7
:10ABD000F0410D0004464FF0FF3721D02968C1B184
:10ABE0002068C8B1084447F0B5FB060018D0D4E986
:10ABF0000021FBF7F3FAD5E9002120683044FBF788
:10AC0000EDFA606848F0E4FE206829680844C4E969
:10AC100000060020BDE8F0812046FFF7C1FF08B123
:10AC20003846F7E7D5E900216068FBF7D7FAF0E787
:10AC30002DE9F047814679B10D46164600F077F8C8
:10AC400004004FF000072DD0E900FFF7A9FF30B155
:10AC5000204600F060F825E00020BDE8F0870021E4
:10AC60004FF0010C606810E08023002216F801808C
:10AC700018EA030F02D080F800C000E007705B08FC
:10AC8000401C521C082AF1DB491CA942ECDB4CB1E8
:10AC900021464846FFF79BFF0546204600F03BF85B
:10ACA0002846DAE74FF0FF30D7E72DE9F04180463C
:10ACB00079B10D46164600F03AF804004FF000074F
:10ACC00026D02946FFF76CFF30B1204600F023F86C
:10ACD0001EE00020BDE8F081681E012202FA00F0AB
:10ACE0000023616807E0064201D00A7000E00F709F
:10ACF0004008491C5B1CAB42F5DB4CB12146404689
:10AD0000FFF765FF0546204600F005F82846E1E715
:10AD10004FF0FF30DEE710B5040007D0606848F060
:10AD200057FE2046BDE8104048F052BE10BD10B599
:10AD3000082047F00FFB002802D00021016041608D
:10AD400010BD2DE9F041046805467CB1E01DC11736
:10AD500000EB5170C01047F0FDFA002807D0E11752
:10AD600004EB5171CE10002369680EE00020BDE8AD
:10AD7000F081002215465206170E11F8012B6D1CAA
:10AD80003A43082DF7DBC2545B1CB342F1DB620788
:10AD9000EDD00022134604F0070405E05206150E1C
:10ADA00011F8012B2A435B1C9C42F7DC8255DEE73D
:10ADB0002DE9FF4F81B09A46DDE90E8791468B461B
:10ADC0001588002419E0391B491E2AFA01F000F009
:10ADD00001008DF8000000260BE000BF9DF8003058
:10ADE0002A46594601983FF02DFC761C6D1CF6B2A0
:10ADF000ADB24645F2D3641CE4B2BC42E3D3A9F839
:10AE0000005005B0BDE8F08F2DE9FF4F8DB08246B0
:10AE100000260A46ADF8286008A909A817F0AEF880
:10AE20003D4C000656D409983C4F3D4D00286DD04E
:10AE30009DF820004FF0880903285AD20DF12C0B01
:10AE4000099860E09DF8202010448078000757D5CD
:10AE5000404661F30F000F9A0799032362F30F0135
:10AE60000791109961F31F408046BAF802000AA9C1
:10AE70008DE80B08DDE906215346404614F04AF8F8
:10AE800010B9BDF8280098BB206820B128681628A2
:10AE900009D0286838B19DF82010099808448078B6
:10AEA000C0072DD11AE01A98D8B150460FF044FDD2
:10AEB00000060FD4BAF802000AABCDE90003032262
:10AEC000CDE9022BDDE906215346404614F022F875
:10AED000000615D5206811B0BDE8F08FBDF8280038
:10AEE00038B1206820602868286078463860F1E72B
:10AEF00006E0C4F800902E60784638608820EAE7C3
:10AF00000998801D0990018800299BD126602E6038
:10AF1000784638600020DEE720C0072028C00720E0
:10AF200024C0072000220A8043880088834201D978
:10AF3000181A0880044802600448026078460449F0
:10AF4000086000207047000020C0072024C00720B0
:10AF500028C00720F0B5428806880B4B971B0022BB
:10AF60000A4C0B4D8F4206DA882018602260784622
:10AF700028608820F0BD314401801A602260784644
:10AF800028600020F0BD000020C0072024C007205A
:10AF900028C0072002460020012907D0022907D037
:10AFA000032908D0042900D1106870471078704731
:10AFB000108880B27047106820F07F40704730B52D
:10AFC00042180023521E07E00478157800F8015B50
:10AFD0005B1C02F80149DBB2B3EB510FF4D330BD77
:10AFE00070B50520FBF75AFD1149104B8A6DCD6DE8
:10AFF00053F822402C1B0444CC6543F82200521C19
:10B0000002F007008865E0100A49C0F389100A4A77
:10B0100041431144094AC91201FB0021084A49125F
:10B0200001FB002002498031086070BDBCE60720AA
:10B0300004C307206F9A0F006EE1C6865F54134960
:10B04000EA319FF070B50320FBF742FD1E493E2513
:10B050004B8924390968B5EB216F01DD0E1600E03C
:10B060003E26194AA43A946BA61B3E36B34207D338
:10B07000B5EB216F01DD0B1600E03E23E31A3E33F2
:10B080009BB242F2454463434FF4FA6403F2D52382
:10B09000B3FBF4F342F66424A4EBA1410F334B431A
:10B0A0000A49897A1E2901D9562100E05A214B43C9
:10B0B0004043000BB3FBF0F040F23541D0678842CB
:10B0C00000D9D16770BD0000A8C30720DCE60720C7
:10B0D0002DE9F14F7E4C00277E4D2079B8464FF088
:10B0E000005A40F23B1944F6206B4FF08056072877
:10B0F00008D2DFE800F0045B73919FC9E800207874
:10B1000008B10227D9E0607810BB18F02BFDC0B25F
:10B11000122803D2686900F4003002E0686B00F086
:10B12000020010B16C48007890B918F01BFDC0B255
:10B13000122803D2686900F4802002E0686B00F0F6
:10B14000100010B16548007810B9686D000601D490
:10B150000127B2E041F07EFD6148416A21F0407173
:10B160004162416E21F0407141F000714166C5F8C5
:10B170009C60D5F8800040F08050C5F88000E078F1
:10B1800010B1C5F8986001E0C5F89C607320E080BC
:10B19000C5F898A041F006FCE06052484168491C9F
:10B1A00041604169491C4161012085E0002041F076
:10B1B0004DFBE060D5F89400C00002D5C5F89C6056
:10B1C00001E0C5F8986041F035FB002875D0686D46
:10B1D000000642D4A4F8068002206DE0002041F071
:10B1E00035FBE060D5F89400C00002D5C5F89C603E
:10B1F00001E0C5F8986041F01DFB90B3E088411C68
:10B20000E180A17809B1F52100E04946884254D98E
:10B210000320C4F80CB04FE0C5F89CA041F0C2FB7D
:10B22000E060A07808B1F52000E048466430E08096
:10B23000042041E0002041F009FBE060D5F89400D3
:10B24000C00002D5C5F89C6001E0C5F8986041F0E7
:10B25000F1FA30B1686D000604D4E088411EE18047
:10B2600009D32AE0A07808B1F52000E04846E1883B
:10B270006438884204DA41F0ABFB84F8048067E765
:10B28000A4F80680052017E0002041F0DFFAE06016
:10B29000D5F89400C00002D5C5F89C6001E0C5F85F
:10B2A000986041F0C7FA40B1E088411CE1800F2866
:10B2B00003D90620C4F80CB020710098E168016041
:10B2C0003846BDE8F88F84F8048041F081FB18E728
:10B2D0009C01001000C0092006C3072005C30720F9
:10B2E00000C0024098E607202DE9F0470025884677
:10B2F000174601462C462E46EFF3108000F0010958
:10B3000072B62846214A012902D002290BD017E043
:10B310001F499070486008601031486008600D4611
:10B320001B4C1A4E0CE01A49D0702031486008605E
:10B33000103148600860154E0D46A1F11004761CCE
:10B340003078F0B1E968414506D0A86848F040FB84
:10B35000404646F0FFFFA860E068B84206D0A0680B
:10B3600048F036FB384646F0F5FFA060C5F80C8083
:10B370000120E7603070B9F1000F00D162B6BDE87E
:10B38000F087404646F0E6FFA860EBE7F6010010C4
:10B3900044EC072030B593B08F21109117491191DB
:10B3A00011AB10AA012147F09DFC119800246B46B7
:10B3B0000168426891420DD04168C268491C8A42C6
:10B3C00000D8891AD0E90152525D1A554160641CB7
:10B3D000402CEDD30A4D002C02DCA878002808D0C0
:10B3E00022461946109846F041FA402C03D000201E
:10B3F000A87013B030BD0120FAE7000044EC07202C
:10B40000F601001030B597B00E2104911049029159
:10B4100005AC02AB04AA022147F064FC2146049863
:10B4200045F0D8FE10E0029B1A68D968521C914280
:10B4300000D8521A5968914208D09D6814F8011B2F
:10B440001B68E95402990A60401EECD217B030BD67
:10B4500054EC072070B5074C0A20214645F0BAFE8F
:10B46000054603E014F8010B45F036F86D1EF9D2DD
:10B4700070BD000084EC0720012070470120704758
:10B4800001207047084A0948116801700B0A43708F
:10B490000B0C8370090EC1701179017151794171E2
:10B4A0009179817101207047FD0100101C0200108C
:10B4B00007490020887007494860086010314860DB
:10B4C00008601031486008601031486008607047BB
:10B4D000F601001044EC072001207047012070475E
:10B4E00001207047012070470748C178026861F366
:10B4F0001F6206490A6002790A7142794A718079AD
:10B5000088710120704700001C020010FD0100102E
:10B5100070B518F027FBC0B21A4C122803D260692C
:10B5200000F4003002E0606B00F00200164D08B13C
:10B53000A87888B918F016FBC0B2122803D2606947
:10B5400000F4802002E0606B00F0100008B1687821
:10B5500010B90E48007848B11BF0E4FE20B9012074
:10B560001BF0FCFE0120E871012070BDE87938B1C4
:10B570001BF0D8FE20B90020E87101201BF0DEFE90
:10B58000002070BD00C0092004C307209D010010E9
:10B590006A4900B50A686A488F2A75D00FDC872A85
:10B5A00073D005DCDAB1822A20D0862A15D156E084
:10B5B000882A18D0892A3DD08A2A0ED1B5E0962A49
:10B5C0006FD006DC912A0CD0922A35D0932A04D170
:10B5D00036E0A22A6FD0A52A6ED0086800BD0020F0
:10B5E00000BD006800BD4FF2036000BD0068142874
:10B5F0001ED008DCA0F10A0006286ED2DFE800F0B9
:10B600000C120E910C0C1A280AD01B280AD01D28E7
:10B610000AD0232861D109E0672000BDD12000BDF8
:10B62000682000BD692000BDE62000BD772000BD78
:10B63000C82000BD7F2000BD5DF804EB0DF0B6BB57
:10B640000068012809D0062805D0802805D0812867
:10B6500003D0A02000BDA92000BDBA2000BD006815
:10B6600030281BD008DC102810D0112810D0122848
:10B6700010D0152806D10FE0312813D0332814D06C
:10B68000342815D0132000BD2AE016E09120FAE7F7
:10B690009220F8E79320F6E71420F4E74FF20160D8
:10B6A000F1E728E04FF20460EDE74FF20860EAE7C7
:10B6B0004FF20960E7E731E039E0006804280DD077
:10B6C000052804D0062806D007280ED101E01F2047
:10B6D000D9E77620D7E7ED20D5E722E09C20D2E716
:10B6E0000068032805D0072801D06620CBE71A2080
:10B6F000C9E7AA20C7E70068801E07280BD2DFE849
:10B7000000F008080A0608040400AD20BBE7DC20AE
:10B71000B9E7AC20B7E74FF20560B4E7006804284A
:10B7200001D0BE20AFE73F20ADE78820ABE700683F
:10B7300080B20AF0D9FFEE20A5E7000020C0072064
:10B7400024C0072001460248006800F0C3B800008A
:10B7500098010010034603480A461946006800F0A5
:10B76000EFB800009801001001460248006800F0A0
:10B7700029B900009801001001460248006800F055
:10B780005FB900009801001010B50821002035F0C5
:10B7900053FD012000F082F90106064801D500683A
:10B7A00010BD00210160044801607846034908602B
:10B7B000002010BD20C0072024C0072028C007207B
:10B7C0000148006870470000980100102DE9F0431F
:10B7D00087B05FEA000805D0B8F1010F02D101205F
:10B7E00045F044FC01242D4D0DF10C09274605AE12
:10B7F000CDF80090CDE901760223224601210920EF
:10B8000043F0FAFD20B1FFF7BFFF07B0BDE8F083BA
:10B81000012C04D0022C09D0042C33D10CE09DF86B
:10B820000C10002035F008FD0224E1E79DF80C1013
:10B83000022035F001FD25E004A8CDE90007012331
:10B84000042219460296092043F0D6FD18B1FFF7ED
:10B850009BFF000614D4B8F1000F13D09DF8100020
:10B8600020B1042804D0FFF78FFF07E0012003E098
:10B87000012045F0FBFB042000F010F9000601D583
:10B880002868C2E7641C042CB2D90020286004494F
:10B8900008607846034908600020B6E720C007200A
:10B8A00024C0072028C0072006490968016006490E
:10B8B00000200860054908607846054908600020B6
:10B8C000704700009801001020C0072024C0072006
:10B8D00028C007202DE9F0410024164D164E174FC1
:10B8E0004FF0050801280CD002280BD0042815D0F1
:10B8F0008220286014203060784638608220BDE8BD
:10B90000F081002035F022FD401C0BD0FAF793FDAA
:10B910002C603460784638600020F0E7084645F037
:10B9200087FCF1E7C5F80080346078463860052070
:10B93000E5E7000020C0072024C0072028C007201A
:10B940002DE9F04786271C4C1C4D1D4E0B464FF031
:10B950001508012809D0022808D04FF082090428D0
:10B9600009D0C4F80090142021E0002035F016FD25
:10B97000401C12D009E00121184645F0D5FE10F117
:10B98000020F11D0B0F1FF3F07D0002020602860E7
:10B99000784630600020BDE8F0872760C5F8008059
:10B9A000784630608620F6E7C4F8009013202860BF
:10B9B000784630608220EEE720C0072024C00720B0
:10B9C00028C007202DE9F3411A4C9DF804101A4DA8
:10B9D0001A4E01280CD002280BD0822704280BD045
:10B9E000276014202860784630608220BDE8FC8102
:10B9F000002035F0E2FC0AE00122114601A845F0E2
:10BA000093FE10F1020F11D0B0F1FF3F06D00020DD
:10BA100020602860784630600020E7E786202060BC
:10BA200015202860784630608620DFE727601320E5
:10BA3000D8E7000020C0072024C0072028C0072026
:10BA400070B5134C134D144E01280BD002280AD0A8
:10BA500004280BD0822020601420286078463060B3
:10BA6000822070BD002035F077FB02E0084645F0EB
:10BA70006DF8002130B105202060296078463060E3
:10BA8000052070BD2160296078463060002070BDBF
:10BA900020C0072024C0072028C0072010B50C496B
:10BAA0000C4A0D4B012809D0042807D082200860D9
:10BAB0001420106078461860822010BD074C20606A
:10BAC00000200860106078461860002010BD00005B
:10BAD00020C0072024C0072028C00720980100109C
:10BAE00030B502464FF6FF731846084C08E000BF19
:10BAF00012F8015B85EA1025655D85EA002080B2B9
:10BB0000491E89B2F4D2584030BD000008690500D2
:10BB100070B50023084D0AE0CE5C04885B1C86EA01
:10BB200014269BB235F8166086EA04240480521E5F
:10BB300092B2F1D270BD0000186A0500024610B53D
:10BB4000FF20002907D0044B541814F8014C44403E
:10BB5000491E185DF8D110BD186C050070B50C4673
:10BB6000054616F05BFF0F4E000604D4204616F083
:10BB70007FFE000601D5306870BD2968206800226C
:10BB8000814203D3081A2860226002E0401A206034
:10BB90002A60326004480260784604490860002048
:10BBA00070BD000020C0072024C0072028C0072047
:10BBB0002DE9FF5FDFF88480DFF88490214C1E467A
:10BBC00093460D0082464FF0000701D0042D09D99D
:10BBD00088202060C8F800707946C9F8001004B0C9
:10BBE000BDE8F09F0020C6E900006A465946284695
:10BBF00017F0F4F800060FD4BAF1000F0ED102AA24
:10BC00005946284617F0F9F8000605D402A96846F7
:10BC100027F02AFC000601D52068E0E70098306094
:10BC2000BDF80400B0809DF80600B0712760C8F828
:10BC300000707946C9F800100020D0E724C0072022
:10BC400028C0072020C007202DE9FF47DFF88080AB
:10BC5000DFF88090204C16460D0082464FF000071A
:10BC600001D0042D09D988202060C8F800707946D9
:10BC7000C9F8001004B0BDE8F0870020C6E9000054
:10BC80006946284617F0DAF800060ED4BAF1000F1C
:10BC90000DD102A9284617F0C8F8000605D402A95C
:10BCA000684627F0E1FB000601D52068E2E700982E
:10BCB0003060BDF80400B0809DF80600B0712760C8
:10BCC000C8F800707946C9F800100020D2E70000DB
:10BCD00024C0072028C0072020C007202DE9F041FC
:10BCE0000D8812680646A2FB050C002707FB05C558
:10BCF0003C4602FB0455098842F210728A1847F14B
:10BD0000000123B14B084FEA320738185D410B465A
:10BD10002946FAF7F3F90D4A0D4B0E4D31B9DFF80C
:10BD200038C00227BCEB000C8F4108D2892010607C
:10BD300003201860784628608920BDE8F0813060D3
:10BD400014601C60784628600020F6E720C00720B9
:10BD500024C0072028C00720FFE30B54034630B45B
:10BD600000200C2A08D2DFE802F0070609090F0FAD
:10BD7000060606060609084630BC704730BC184661
:10BD800040F0A2B80820F7E70829FBD2F3E700004B
:10BD90003EB5684617F0CAF8274C000639D402A809
:10BDA00017F016F9000634D49DF800000025082885
:10BDB00009D009280DD02560204805607846204923
:10BDC000086000203EBD684617F0B8F8000620D491
:10BDD0000CE001A816F0EAFD00061AD49DF8040054
:10BDE000012818D05FF013008DF8000068463FF07E
:10BDF00045FA00060DD48DF8045001A83EF034FE3B
:10BE0000000606D48DF8045001A83EF0C9FE0006D5
:10BE100003D520683EBD0220E6E7BDF80800800794
:10BE200001D4084A00E0084A0021084628F038FDFD
:10BE3000012029F0FBFA3EBD20C0072024C00720C6
:10BE400028C00720C5740500E67405002DE9F04FF1
:10BE5000ADF50D7D0D46044612F0B2F8ADF80C02BA
:10BE6000AD1EAEB204F13301B4F83180A6F1310257
:10BE7000881EFAF7B3F93246214683A8FFF748FE39
:10BE8000BDF80C023125DFF89490254F4FF0010AE0
:10BE9000404535D020E0601983460188ADF82C126A
:10BEA000B0F80280BDF82C0285A98B903AF0FAFF19
:10BEB000BDF81802C0051FD5ADF802808B98ADF80B
:10BEC00000000BF10401424601A8FAF787F9684621
:10BED00039F0F4FF000602D589F802A007E06846B1
:10BEE0003BF09CFA000607D5032189F80210386858
:10BEF0000DF50D7DBDE8F08F05EB0800001D85B246
:10BF0000B542C8D30C203EF03BFB00203860054909
:10BF100008607846044908600020E9E7B60300108D
:10BF200020C0072024C0072028C007202DE9FE4399
:10BF3000884600241F461C80694602A8FFF70EFEB3
:10BF4000154E000612D4029808B90098E0B9019481
:10BF5000012500946946284616F058FD000605D4D0
:10BF6000694601A836F02EFF000602D53068BDE80C
:10BF7000FE836D1CEDB2052DECD9019810B95FEA76
:10BF8000184001D0012038803460044804607846AD
:10BF9000034908600020EAE720C0072024C00720EA
:10BFA00028C007202DE9FC4100251D801F4688463A
:10BFB00001A8009516F01AFD154E000612D401A92D
:10BFC000684636F0FFFE00060CD4012401A9204685
:10BFD00016F01CFD000605D401A9684636F0F2FEF5
:10BFE000000602D53068BDE8FC81641CE4B2052C73
:10BFF000ECD9009810B95FEA184001D001203880D0
:10C000003560044805607846034908600020EAE787
:10C0100020C0072024C0072028C007202DE9FC41AC
:10C020000746002090460E46ADF8000004460EE09C
:10C03000351B402D00D9402539192A460D481BF0E3
:10C0400091FBAAB20B496846FFF762FD2C44B4424B
:10C05000EED33919424601A81BF084FBBDF800005D
:10C06000BDF80410884202D10120BDE8FC81002007
:10C07000FBE70000F8C807200099002018800A6933
:10C080000AB9896909B10121198004490860044984
:10C0900008607846034908600020704720C00720E8
:10C0A00024C0072028C00720009800211980828A18
:10C0B0000AB9C28A2AB102690AB9806908B10120A5
:10C0C000188004480160044801607846034908600C
:10C0D0000020704720C0072024C0072028C0072068
:10C0E0002DE9F0478CB000273E4609A816F01EFF48
:10C0F000824D00067ED49DF82400DFF80482DFF82C
:10C1000004920024022803D0192801D01A2872D1E1
:10C1100002A93520FCF702F90006EBD49DF80A00CD
:10C1200000F00F01000900EB800001EB400000F57A
:10C13000FA60ADF81C009DF8090000F00F0100093D
:10C1400000EB800001EB40008DF81E009DF8080018
:10C1500000F00F01000900EB800001EB40008DF8BA
:10C160001F000BA907A8FDF789FE02A93620FCF7DE
:10C17000D5F800063ED49DF80A0000F00F01000932
:10C1800000EB800001EB400000F5FA60ADF81C0008
:10C190009DF8090000F00F01000900EB800001EBA1
:10C1A00040008DF81E009DF8080000F00F01000906
:10C1B00000EB800001EB40008DF81F000AA907A8E2
:10C1C000FDF75CFE03A816F0CDFA000612D406A80F
:10C1D00035F0F0FA00060DD4BDF82C000DF1080A78
:10C1E000B0B1BDF80C10814212D39DF81800172889
:10C1F0000ED201E075E057E00127CDE900A4352318
:10C200003A4639460294022043F0CEFA000668D43A
:10C21000BDF8280098B1BDF80C1081420FD39DF8ED
:10C22000180060B10126CDE900A43623324631461C
:10C230000220029443F0B8FA000652D4A7BB56EA93
:10C24000070052D008A93420FCF768F8000648D44B
:10C250009DF8200001281DD0022804D0032844D1D5
:10C2600029497D20087008A95320FCF757F80006DB
:10C2700037D49DF8200010F002008DF8200004D083
:10C28000012029F0D3F800062BD400211F4A0846CC
:10C2900028F006FB06A835F08DFA000621D49DF89B
:10C2A000180016B1401E01E01FE0401C8DF8180078
:10C2B00006A835F06BFB9DF82000022801D003286A
:10C2C00013D10EB1124A00E0124A0021084628F0AC
:10C2D000E7FA9DF8200040B1012029F0A7F80006F8
:10C2E00003D528680CB0BDE8F0872C60C8F8004082
:10C2F0007946C9F800100020F4E7000020C00720AC
:10C3000024C0072028C007209CC20720A789050059
:10C31000BD890500E9890500F8B500241E460F46D1
:10C3200025461C80684616F093FA0A49000601D596
:10C330000868F8BD0098204301D1380C01D00120D5
:10C3400030800D600448056078460449086000208C
:10C35000F8BD000020C0072024C0072028C0072007
:10C360002DE9FE434FF00008ADF800801D460C4655
:10C37000A3F8008001A800F089FE274E000632D401
:10C380009DF8040048B3A0B21C2812D2DFE800F0E8
:10C39000110E0E0E0E0E0E0E0E0E0E0E0E0E0E0EBA
:10C3A0000E0E0E0E0E0E0E0E0E0E0E0EC4B2C7B2F6
:10C3B00011E001242A276946204616F0D5FA000626
:10C3C00011D4BDF80000401E0004000CADF80000C0
:10C3D00003D1641CE4B2BC42EDD902A96920FCF788
:10C3E00071F8000602D53068BDE8FE83BDF8000094
:10C3F00030B99DF80800400602D5A5F8008001E09C
:10C4000001202880C6F800800449C1F800807846E1
:10C41000034908600020E7E720C0072024C0072068
:10C4200028C007207CB5154C00258DF800502068E9
:10C43000134E70B132F02AFD30682168C0B240EA74
:10C4400001400190042201A9172044F0B3F827F01D
:10C4500031F932F01BFD69468A20FBF75FFF27F0B8
:10C4600029F99DF8000008B120687CBD2560356081
:10C4700078460449086000207CBD000020C00720E9
:10C4800024C0072028C0072070B592B000250422E0
:10C490004FF4876110A81BF053F91098B0F5F42FF2
:10C4A00001D30B48109000246E460BE04022214639
:10C4B00068461BF045F900217058091D05444029C4
:10C4C000FAD3403410988442F0D312B0284670BD9D
:10C4D000FF9F070038B51C46000C69463AF0DEFEA7
:10C4E00001060C4801D5006838BD016841B9BDF8A6
:10C4F000001029B10849B1F8CE1109B101212180FC
:10C500000021016005480160784605490860002067
:10C5100038BD000020C0072020F2072024C00720DB
:10C5200028C007202DE9F04F764C074606468BB011
:10C530000020A070E070884620711AF093F8DFF8B0
:10C54000C8A1DFF8C8914FF4807B0125192231463C
:10C5500068461BF007F9022216213046FFF75EFD00
:10C5600000287DD0DDF80E10022206F11900FFF739
:10C5700055FD002874D09DF8000006282CD2DFE875
:10C5800000F02B03032B2B1CDAF87420DDF80A30A3
:10C59000521C93421FD2DAF87410DDF80A30C91A1F
:10C5A000DDF80E30491C994215D3DDF80A10DDF88C
:10C5B0000E30194491420ED80EE0DDF80E10B1F5A0
:10C5C000F42F00D9A570DDF81210C1F30B41A1F5CD
:10C5D0008072113A00D0A570012803D0022801D042
:10C5E000052845D19DF808005A46400706F2194132
:10C5F00007D547481BF0B6F84449454804F090FB7E
:10C6000002E042481BF0AEF800200990B9F804108F
:10C61000ADF82410099A019992B24846914200D08F
:10C62000A57000210991017B8DF82410099ABDF8AD
:10C630000110D2B2914200D0A5709DF800100229DD
:10C6400016D1016B0991DDF81210099A914200D0C0
:10C65000A5700021099199F834008DF8240000E0BC
:10C6600032E009999DF80300C9B2884200D0A57054
:10C670009DF81800401EFE2800D2A570BDF80100EC
:10C68000A0F57F41FF3901D0562802D19DF8030063
:10C6900060B968461AF0AAF940B9BDF801005028FF
:10C6A00003D19DF80000052800D0A570DDF80E002C
:10C6B0001B36064468461AF099F930B1E07880B12B
:10C6C000217988420DD012E0A5709DF8180010B9AC
:10C6D0002079401C2071E078401CC0B2E0700C282A
:10C6E00001D3A57003E0A07800283FF42FAFB8F184
:10C6F000000F02D0F11BC8F80010A0780BB0BDE805
:10C70000F08F0000DCC00720EC6D0500F8CA0720A0
:10C71000F8C90720002204E0835C0BB100207047B9
:10C72000521C8A42F8D30120704700002DE9F047DF
:10C7300082460AA8154690E884020E461C4608A9BF
:10C740001846DDF824803DF00DFC88F80000FF2835
:10C7500069D0215C464A01EB410012F820004128D3
:10C7600047D024DC232844D010DC162841D006DC36
:10C770000E283ED011283CD0152874D139E0182855
:10C7800037D01D2835D01E286DD132E0312830D069
:10C7900006DC26282DD029282BD02D2863D128E08F
:10C7A000352826D0392824D03D285CD121E0A8287E
:10C7B0001FD010DC81281CD006DC442819D0482862
:10C7C00017D04B284FD114E0842812D0A12810D0C4
:10C7D000A52848D10DE0B4280BD006DCAB2808D042
:10C7E000AE2806D0B1283ED103E0B72801D0BA2840
:10C7F00039D19DF82000205C00EBC00028448279EC
:10C80000920630D501EBC1012944C278CB789A4217
:10C8100029D103790A79934225D24079497918447C
:10C820001144884210D21EE03988B9F800008142D4
:10C8300007D210A10AF10700F9F703FD3888401C60
:10C8400038803088401C30809DF82000205C00EB50
:10C85000C000284401794079084431888842E3D8EF
:10C860000120BDE8F087FF2188F800100020F8E7DC
:10C87000E8BB0500200000002DE9F84F894604467A
:10C880000020ADF8000091B21D466A46484639F0D6
:10C890009FFDA4F10E00254E254FDFF89880052856
:10C8A00003D80A20FBF754FEA8B14FF0A50A4FF4B5
:10C8B000837B102C19D00F2C17D0BDF8000028B1A5
:10C8C00081B248463FF079FA1FFA80F90F2C10D058
:10C8D000102C1DD015E091203060B12038607946D1
:10C8E000C8F800109120BDE8F88FBDF8000098B19D
:10C8F000E6E7A9F1010018280ED8287840F00800D2
:10C9000028700020306038607946C8F80010EAE7E7
:10C91000A9F11A000528F0D9C6F800A0C7F800B0A0
:10C920007946C8F80010A520DDE7000020C00720E8
:10C9300024C0072028C0072000B58FB0694600201A
:10C9400035F062F825216846FFF7F8F89DF82510C4
:10C95000884202D101200FB000BD0020FBE700009B
:10C96000F0B587B000268DF80C600420FBF7FEFDC3
:10C9700004460A20FBF7FAFD20444FF48265264F57
:10C98000B5EB400F30D00021244A084627F088FF3D
:10C9900001246D08E8070ED02046FBF7E7FD50B9EB
:10C9A0000A2206A9204647F0DBF9034600211C4A6B
:10C9B000084627F075FF641CE4B21E2CE9D303A9D6
:10C9C0005320FBF7ABFC00061AD49DF80C0010F0C6
:10C9D00002008DF80C0007D01248018841F00201D6
:10C9E0000180012028F022FD012105AA04A88DE87C
:10C9F00007000B460422092042F0FEFC000602D587
:10CA0000386807B0F0BD3E600748066078460749C1
:10CA100008600020F5E7000020C007201E71050017
:10CA20002875050018C0072024C0072028C007204B
:10CA30002DE9F843002481460480684615F018FF6C
:10CA4000114E00060CD4114FDFF844800098A0B1BD
:10CA5000062500946946284615F0D8FF000602D541
:10CA60003068BDE8F883009818B10121A9F80010DA
:10CA700003E06D1CEDB20B2DECD334603C607946C5
:10CA8000C8F800100020ECE720C0072024C00720D1
:10CA900028C007202DE9FF4F91B00546DDE91FA40E
:10CAA00008212046DDF8789019F094FE00287DD00A
:10CAB00000216846625C00EB4103120900F8112076
:10CAC000625C491C02F00F025A700829F2D39DF8EB
:10CAD0000F80DFF878B102460E2100BF5BF82830E6
:10CAE0004F1C5E5CDB5D891E975D12F803C002F887
:10CAF00006C0D754F2D5002100EB410210F81130E6
:10CB0000527842EA03126254491C0829F4D30822DD
:10CB10000020161A3319215C13F8016D370147EA1A
:10CB2000161626540E0146EA1111401C1970B0EB7E
:10CB3000520FEED307210AF1060019F04BFE002830
:10CB40007ED014216846F9F771FB30208DF8000083
:10CB5000DAF80610CDF80110BAF80A10ADF8051091
:10CB60009AF80C008DF80700B9F1070F1AD968463A
:10CB7000F9F71CFC064607A944F09EFEB9F10C0F1C
:10CB800001D2079804E009F0070007A951F8200036
:10CB90002F497040B0FBF1F201FB12022DA1684653
:10CBA00045F080FB08226946002000E048E0131AA7
:10CBB0000B440E5C13F8017D0F54401C1E70B0EB4B
:10CBC000520FF2D30FAB06AA2146684646F032FE5A
:10CBD0000F98002834D005AA294609F0CDFD90BB56
:10CBE0006846F9F7E3FB05992A46A0FB01010023FB
:10CBF000F9F784FA1146DDE9122047F04FFC0446AC
:10CC0000DDE90510A0FB01012A460023F9F776FAB9
:10CC10001100059118D0129A149847F03FFCA0FB20
:10CC200004010023129AF9F769FA104619462A46B8
:10CC30000023F9F763FA06980592904204D1012087
:10CC400015B0BDE8F08FFFE70020F9E744C00720EA
:10CC5000FFE0F50525303864000000002DE9FC41B7
:10CC60008046032034F024FD2D4E2E4F2E4C0025FF
:10CC700030B9B8F1000F03D0042019F0BEFD80B325
:10CC800069465320FBF74AFB9DF80000002100F0A5
:10CC900002008DF80000254A084627F001FE002119
:10CCA000234A084627F0FCFD9DF8000010B1012042
:10CCB00028F0BCFB1F4975200870684616F036F94D
:10CCC00000061CD468463EF0F1FA000617D401A80D
:10CCD00015F03EFF000612D49DF8040010B1192093
:10CCE00001E016E01A208DF8000068463EF0C6FA12
:10CCF000000604D404203DF0FDFB000602D52068A8
:10CD0000BDE8FC8182202060356078463860822052
:10CD1000F6E725603560784638600020F0E70000CF
:10CD200024C0072028C0072020C00720E375050085
:10CD3000047605009CC207200099002018800A692B
:10CD40001AB9896909B9012119800449086004499F
:10CD500008607846034908600020704720C007201B
:10CD600024C0072028C007202DE9FE4398460A9DCD
:10CD70009146074601290DD1684616F049F9424C03
:10CD8000000604D401A816F0D1F8000605D52068E5
:10CD9000002800D00120BDE8FE8340F212410026A9
:10CDA0003A4CA7F212408F4260D01EDC40F2FA31BA
:10CDB000A7F2FA308F4227D00EDC062F56D004DCC3
:10CDC000042F53D0052FE5D150E0072F4ED0A7F503
:10CDD0004070F138DED11AE012380628DAD2DFE8E6
:10CDE00000F016134503454ED4E723283ED028DC37
:10CDF0000D283BD004DC042809D00628CAD106E05F
:10CE0000122804D01428C5D1A0780228C2D002ABC1
:10CE10004246494638463AF0B9F90028BAD01C488B
:10CE200000682128B6D19DF8000030B3012011F030
:10CE3000DFFF10B3607880071FD516480078E0B197
:10CE4000A8E74A2812D004DC37280FD04228A1D105
:10CE5000DDE7922801D093289CD19DF800006178ED
:10CE600040420840800795D4002094E79DF80000D8
:10CE700061784042084080078CD42E80F4E701207E
:10CE800011F0B6FFDBE7000020C0072020C5072017
:10CE900024C007209CC207202DE9F04F87B0002452
:10CEA00088B203941D4FDFF878801E4E9B468A4659
:10CEB0001C808146052829D895B20A2D26D8052D33
:10CEC0001AD905AA012104A88DE807006A1E0223C9
:10CED0000C2042F091FA00060AD49DF81010894502
:10CEE00014D103A94FEA050015F090FD000605D501
:10CEF000306807B0BDE8F08F03A9F5E7039810B9D3
:10CF00005FEA1A4002D00120ABF8000034603C60B8
:10CF10007946C8F800100020EBE7000024C0072085
:10CF200028C0072020C00720F8B500251C460E4663
:10CF30001D80684615F05AFD0106094801D50068B4
:10CF4000F8BD009909B9310C01D00121218005609B
:10CF5000044805607846044908600020F8BD0000D8
:10CF600020C0072024C0072028C007207CB50E461B
:10CF700000251C461D8001A96846FEF7EFFD01064D
:10CF8000094801D500687CBD019929B9009909B902
:10CF9000310C01D0012121800560044805607846EC
:10CFA0000349086000207CBD20C0072024C0072062
:10CFB00028C007202DE9F8430E4613490024134FDB
:10CFC00009693480DFF84880D1F80220114D02430E
:10CFD00003D0D1F8661169B960B169467620FBF7D4
:10CFE0009DF9000602D52868BDE8F8839DF8000089
:10CFF000000701D4012030802C603C607946C8F8DD
:10D0000000100020F0E7000020C5072024C0072002
:10D0100028C0072020C007201FB5684614F0FAFE7C
:10D0200004B010BD38B50546684615F07FFF144CB6
:10D03000000618D49DF80010062916D008DC012936
:10D0400013D0032911D004290FD0052906D10CE0F3
:10D0500007290AD0132908D0152906D0284615F02B
:10D0600077FD000603D5206838BD01202870002018
:10D07000206004490860784603490860002038BDF4
:10D0800020C0072024C0072028C0072038B5054647
:10D09000684615F053FF144C000618D49DF8001094
:10D0A000072916D006DC0DD2DFE801F00C130C13B3
:10D0B000131313000E290CD013290AD0152908D0F8
:10D0C0001B2906D0284615F043FD000603D520682D
:10D0D00038BD01202870002020600449086078468F
:10D0E00003490860002038BD20C0072024C0072065
:10D0F00028C007202DE9FE434FF00008CDF800803E
:10D100001D460C46A3F8008001A8FFF7BFFF1F4E85
:10D11000000623D49DF80400D0B1A0B2012810D09D
:10D1200002280ED003280CD004280AD0012404279A
:10D130006946204615F019FE00060FD4009838B94C
:10D1400002E0C4B2C7B201E0641CE4B2BC42EFD951
:10D1500002A96920FBF7B6F9000602D53068BDE8E0
:10D16000FE83009830B99DF80800400602D5A5F866
:10D17000008001E001202880C6F800800449C1F841
:10D1800000807846034908600020E8E720C00720B7
:10D1900024C0072028C007202DE9F04788B00024CC
:10D1A0008DF80040CDE90444CDE902448DF81840E3
:10D1B000884681468DF804409246148069461220C4
:10D1C000FBF7ACF8504D00067ED406A96920FBF7AA
:10D1D000A5F8000678D401A97620FBF79FF8000691
:10D1E00072D44A4E4A4FB9F1050F37D2DFE809F041
:10D1F00003101A262E009DF8000000F001019DF892
:10D20000180000F00202114346D1400775D543E0F3
:10D210009DF80000C00770D014E000BF9DF8040026
:10D22000800708E09DF80000C00766D012E000BF4C
:10D230009DF80400400700285FDA15E09DF818000B
:10D2400080075AD5B8F1000FE8D11DE09DF818000D
:10D25000400752D5B8F1000FEAD115E0B9F1000F3F
:10D260001AD0B8F1000F0FD002AB42464946002059
:10D27000FEF79EFC000635D4B8F1050F28D9DDE98C
:10D280000201084339D023E002AA49460020FEF7F4
:10D29000DBFC000626D41BE00020CDE902000120C3
:10D2A0008046014604AA0020FEF7CEFC000619D4F1
:10D2B000DDE90220DDE90431D2184841CDE9022040
:10D2C00008F10100C0B200E00CE080460428E8D973
:10D2D000DDE9020108430DD169466920FBF71EF81C
:10D2E000000603D5286808B0BDE8F0879DF8000067
:10D2F000800602D40121AAF800102C603460784620
:10D3000038600020EFE7000020C0072024C007207D
:10D3100028C007202DE9FE4F00241F460E46254653
:10D32000A1461C80684615F0F3FBDFF874A00006E8
:10D3300012D49DF80000DFF86CB028BBB0B2012811
:10D340000ED002280CD001264FF0020801A9304669
:10D3500015F0F0FC000607D5DAF80000BDE8FE8FF6
:10D36000C6B200F0FF0809E09DF80800019C60F3D8
:10D37000070554EA050003D1761CF6B24645E5D907
:10D380002C4302D00120388001E0A7F80090CAF8B1
:10D390000090CBF800907946034801600020DDE75B
:10D3A00020C0072024C0072028C007202DE9FC4703
:10D3B000002400941E4688461C8001A8FFF766FEE4
:10D3C000194F000618D49DF80400F0B11FFA88F038
:10D3D0008046012806D0022804D0032802D0B8F1E4
:10D3E000040F10D101254FF010096A462946404626
:10D3F00015F04EFD000602D53868BDE8FC870098A0
:10D4000028B96D1CEDB24D45EFD9009848B1012007
:10D4100030803C600548046078460549086000207B
:10D42000EBE73480F5E7000020C0072024C0072088
:10D4300028C007202DE9FF5F00240E4698462546A8
:10D44000A3461C8069464B20FAF768FF2E4F000662
:10D4500040D49DF80000C00749D003A8FFF716FE8E
:10D46000000637D49DF80C0070B3B0B201281AD072
:10D47000022818D0032816D0042814D001264FF013
:10D48000040901208246014601AA304615F00CFD30
:10D4900000061FD49DF80800019C60F3070554EABC
:10D4A00005000AD103E0C6B200F0FF090AE00AF164
:10D4B0000100C0B282460628E5D954EA050003D12E
:10D4C000761CF6B24E45DCD969466920FAF7FAFFB8
:10D4D000000603D5386804B0BDE8F09F2C4303D1A3
:10D4E0009DF80000C0070CD00121A8F80010C7F873
:10D4F00000B00649C1F800B0784605490860002030
:10D50000E9E7A8F800B0F2E720C0072024C0072010
:10D5100028C007202DE9FE434FF00008ADF8008039
:10D520001D460C46A3F8008001A8FFF7AFFD1E4E74
:10D53000000620D49DF80400B8B1A0B201280DD097
:10D5400002280BD0012402276946204615F0C4FCAE
:10D55000000610D4BDF8000038B902E0C4B2C7B26A
:10D5600001E0641CE4B2BC42EED902A96920FAF7DA
:10D57000A9FF000602D53068BDE8FE83BDF80000B3
:10D5800030B99DF80800400602D5A5F8008001E0FA
:10D5900001202880C6F800800449C1F80080784640
:10D5A000034908600020E7E720C0072024C00720C7
:10D5B00028C007202DE9FF41002598460E462C463D
:10D5C00002A8FFF763FD254F00062ED49DF8080042
:10D5D00028B33004000C04D0012816D002281ED134
:10D5E00013E001266946304615F088FC00061CD47D
:10D5F0009DF80400009D60F3070455EA04000ED175
:10D60000761CF6B2022EEDD909E0694615F076FCDB
:10D6100000060AD49DF80400009D60F3070403A9E6
:10D620006920FAF74FFF000603D5386804B0BDE85B
:10D63000F0810020254306D19DF80C10890602D503
:10D64000A8F8000002E00122A8F800203860044990
:10D6500008607846034908600020E7E720C00720FB
:10D6600024C0072028C007202DE9FC471D46884616
:10D6700001A80A9E15F04CFA1B4F000622D49DF813
:10D680000400DFF86890DFF868A0002408B12C805F
:10D6900021E0012028801FFA88F14FEA1840012973
:10D6A00002D0652903D006E0317BC90702D1F16AB7
:10D6B00009B900B92C8096F86000694636F00CFE76
:10D6C000000602D53868BDE8FC87BDF80000A0F56B
:10D6D00080615139DBD03C60C9F800407946CAF816
:10D6E00000100020EFE7000020C0072024C0072022
:10D6F00028C007202DE9F04786B000251F468A463E
:10D700001D8004A815F004FA2B4C00063ED49DF8A9
:10D710001000DFF8A880DFF8A89008B13D8043E052
:10D720001FFA8AF6701E06280AD38820206012216C
:10D73000C8F800107946C9F8001006B0BDE8F087B7
:10D740006946304615F09CF800061FD401A815F074
:10D75000F7F900061AD49DF800009DF8041008435C
:10D7600022D0F0B203A936F0B7FD00060ED4BDF802
:10D770000C00B0F58A6F0BD0A0F58061513907D04D
:10D7800002A9304615F0CFF8000606D52068D4E788
:10D79000F0B202A936F0CAFDF6E7029810B95FEAC6
:10D7A0001A4001D0012038802560C8F80050794621
:10D7B000C9F800100020C0E720C0072024C00720BF
:10D7C00028C007207CB50025ADF80050684615F04C
:10D7D000DDFB104C000604D401A814F0C3FF0006C2
:10D7E00001D520687CBDBDF80010BDF804003AF0FA
:10D7F00061FC0949094A38B19120206088200860FD
:10D800007846106091207CBD25600D6078461060E0
:10D8100000207CBD20C0072024C0072028C007208E
:10D820007CB5044600680D460346114903E01E78A6
:10D830000A2E18D05B1E8B42F9D80E49C989B1FB5C
:10D84000F2F2C11A6846F8F7BFFCDDE90001401E9C
:10D85000884207D12068A84204D20A2101702068BA
:10D86000401C20607CBDAB42E7D25B1CE5E70000BA
:10D870006CCC0720320400101CB50446684614F036
:10D8800071FF50B901A9BDF80000FCF761FB9DF8DC
:10D890000400A04201D301201CBD00201CBD0000DB
:10D8A0002DE9F0410026354631465A4C28E000BFAC
:10D8B00004EBC303571CA4F82678D3F82A78D3F8CE
:10D8C0002EC8FBB2A32B02D0A42B04D006E03B0E43
:10D8D000DB0715D002E03B0E9B0711D47EB3D4F8D2
:10D8E0000A30934201D1C4F80A10914206D0084090
:10D8F00004EBC002C2F82A78C2F82EC8491C89B2CB
:10D90000B4F82408B4F8282800EA0207B4F8262856
:10D9100000EA0203FF1A0742CAD15EB1A4F82658F2
:10D92000A4F82818B4F824280A4000EA0501511A7E
:10D93000014205D1002060822082BDE8F08118E01C
:10D94000208A354D00266082608A46F075FFB4F863
:10D950002418014004EBC10000F62A0076B1228AA7
:10D9600081888A42E9D0628A91420BD1C088608264
:10D97000EAE7012695B2521C91B2C1E781880126DF
:10D980002182F3E72B88B5F802C0B4F81A7803EACD
:10D990000C0305EB8303DF802B88B5F802C0B4F8D5
:10D9A000187803EA0C0305EB83031F816B885B1C6B
:10D9B0006B80A4F81818C188A4F81A18828010E0A7
:10D9C000C1F30A012144638A0A7DE1891940214497
:10D9D0000A75B4F81818491CA4F81818618A491C6B
:10D9E0006182B4F81A28B4F81818521A5205E7D10F
:10D9F000618AC1806888401E80B2688029880140A1
:10DA000005EB8100C188A4F81A180089A4F8180849
:10DA10009AE70000ACD5072004E3072038B5044698
:10DA2000684615F06DF8000602D50648006838BD56
:10DA30009DF80000A0438DF8000068463DF020F9F5
:10DA400038BD000020C00720012181400248027932
:10DA50008A43027170470000A80300100121814031
:10DA6000024842888A4342807047000034C0072041
:10DA7000012181400248C2788A43C2707047000089
:10DA80004C03001001218140024882888A43828031
:10DA90007047000034C007202DE9FC410746694665
:10DAA0006020FAF70FFD1B4D000617D41A4C002614
:10DAB00001A8A66024F0D2FB00060FD4019861688B
:10DAC000884213D27FB96168091A0020A1603FF033
:10DAD000C5FA082004F0D0F8000602D52868BDE891
:10DAE000FC8125F0CBFA9DF8001008E06168421A2D
:10DAF0009DF800108A4205D26268801A091A002037
:10DB00003FF0ACFA2E60054806607846044908608C
:10DB10000020E4E720C0072094C1072024C007208C
:10DB200028C007200168084A491E0160914200D9B7
:10DB300002600649002008600549086078460549EA
:10DB40000860002070470000FFE0F50520C00720B6
:10DB500024C0072028C007200168084A491C01602A
:10DB6000914201D901210160054900200860054961
:10DB7000086078460449086000207047FFE0F5051A
:10DB800020C0072024C0072028C00720F0B510B10E
:10DB90006FF0010300E00223002001240CE000F0FC
:10DBA00001070E5C7F4200FB03F504EB470705FB12
:10DBB00007650D54401CC0B29042F0D3F0BD000088
:10DBC00010B501460222084843F0E4FF0106074869
:10DBD00001D5006810BD002101600548016078464C
:10DBE00004490860002010BDF014007020C0072018
:10DBF00024C0072028C0072001B502226946084832
:10DC000043F0F6FF0106074801D5006808BD002172
:10DC1000016005480160784604490860002008BD9D
:10DC2000F014007020C0072024C0072028C007205F
:10DC30000178242903D0FC2903D1242100E0FC2110
:10DC4000017070472DE9F04F87B08946044693462E
:10DC5000002506A95F20FAF735FCDFF810810006E1
:10DC600008D49DF81800206004A95E20FAF72AFC69
:10DC7000000604D5D8F8000007B0BDE8F08F3C4896
:10DC80009DF810104078814201D98DF810009DF860
:10DC900010100126401AC7B2DFF8D8A07F1C51E04F
:10DCA0008222CDE900920123CDF808B03246194610
:10DCB000062041F0A1FBD8BB01224846DBF800104A
:10DCC00042F0AAFA99F8000099F801100A2802D047
:10DCD0000B2808D020E00846FAF7B6FEE0B926493E
:10DCE0002068898807E041B10846F9F7B5FF98B97F
:10DCF00022492068098A084420E00020ADF8140079
:10DD000002900390ADF80400009005AB01AA03A9AE
:10DD100002A8FAF7F7F960B125F0CCF92168BAF852
:10DD200006200144022000EB420008440125206047
:10DD300006E0BDF8040018B1216808440025206001
:10DD4000761CF6B2BE42ABD32DB1BAF806002168FC
:10DD5000081A401E20600020C8F80000084908602A
:10DD6000784608490860002086E7000020C00720A8
:10DD700094C107203204001028040010DACD0720D7
:10DD800024C0072028C007202DE9F0470646144686
:10DD90000D464FF4806044F0DDFA234FDFF88C909D
:10DDA000DFF88CA001000BD0DFF888C00020002233
:10DDB000206023685FEAC3780CD08CEA53030AE042
:10DDC000882038601021C9F800107946CAF8001080
:10DDD000BDE8F0875B08521C2360082AE9DB41F8A4
:10DDE0002030401CFF28E2DD4FF0FF3008E02068C3
:10DDF00016F8012B4240D2B251F8222082EA1020BC
:10DE00006D1E2060ADB2F2D211B1084645F0E0FDC2
:10DE10002068C043206000203860C9F800007946BF
:10DE2000CAF80010D4E7000020C0072024C0072053
:10DE300028C007202083B8ED2DE9FF4F8DB006469E
:10DE40000020DDE91A421F4680460B90079083466A
:10DE500003460A900F98491EC355306800EB010A2B
:10DE60002079012148B3A07908B13FB146E00020F4
:10DE7000206020716071E0714FB33FE01078E3796A
:10DE8000184410700020E07161712068F8B12046DC
:10DE900018F01DFE58B11AE0514620461C9AFFF7B3
:10DEA000BFFC206805702068401C206001E02068ED
:10DEB000202531688842EFD309E00020206060719E
:10DEC000E7B930682060607F692800D06171A08A5E
:10DED000652813D0A07D742833D0607F6D2810D0C2
:10DEE0004D280ED069280CD0204618F0F0FD28B936
:10DEF0002346514630461C9A0DF05AFEA07D7428E8
:10DF00001FD0A07D0A2822D0627F692A00D0C7B125
:10DF1000617911B1A18A65292FD0662839D0692A83
:10DF20007ED0B9464D46208AA84200D805466D2AC3
:10DF300077D04D2A76D0217E302974D0702972D0C6
:10DF4000B6E0FC4900200860FB4908601AE00020A8
:10DF50000A2206E03168401C80B20A703168491C10
:10DF60003160218A8142F5D8F24900200860F249E7
:10DF700008607846F149086007E0EE48002101603A
:10DF8000ED4801607946ED48016011B00020BDE820
:10DF9000F08F0F9800782D2808D1022F04D37F1E10
:10DFA0000F98BFB2401C0F9001200B90A07CB8428C
:10DFB00003D34FF00009804603E0391A80461FFA68
:10DFC00081F9E57D302D35D0732D03D07A2D01D028
:10DFD000404653E0012F03D10F990978302903D02F
:10DFE000B84205D9394604E04FF00109002116E096
:10DFF00001460B460CE000BFDDF83CC009EB010810
:10E00000C4441CF801CCBCF1300F03D1491E89B2C5
:10E010000029F1D1591A7B1A411A9FB289B203E043
:10E0200034E04BE053E040E08846732D08D1B8F16E
:10E03000000F03D009F1010108440AE04D4609E050
:10E04000B8F1000F01D0012100E00021494401EBAB
:10E05000080085B2B9F1000F7FF465AF6D1CADB259
:10E0600061E700BF0F9909EB0003194411F8011C87
:10E07000302905D1012803D0401E80B20028F1D1FB
:10E08000A8EB0001791A8FB28046D9E7AC481C99F9
:10E09000238AC089B0FBF1F1994203D21C99B0FBED
:10E0A000F1F02082258AA9463DE7637E702B06D0D9
:10E0B00069B1A84210D9401B80B207900CE0A84279
:10E0C0000AD9401BC0F34F01401A079102E0A84251
:10E0D00002D9401B80B20A9020206076207E7028F2
:10E0E00001D120202076692A09D0A06838B1E168E2
:10E0F000884204D2091A01EB0B001FFA80FB079833
:10E1000041190A98692A014401EB0B0080B2099079
:10E110000AD0E06A40B1216B884205D8091A0998F3
:10E120000844401C80B20990A07E722808D00020CC
:10E1300060622085A08A63280CD065281BD080E00F
:10E14000218D099808442085606A0028F2D1306842
:10E150006062EFE7306851461C9A10F097FB09990E
:10E1600088426ED2306851461C9A10F08FFB31689D
:10E1700000EB010A65E0306810F8011C0A2901D1A2
:10E18000401E306083466F4A06E000BF1BF8011C4A
:10E19000202903D1ABF1010B9345F7D80999A0EBE6
:10E1A0000B028A4208DB401A3060A17D73294FD0F0
:10E1B000216A89BB206248E0A17D732902D0216ACF
:10E1C00001B92062306851461C9A10F073FE014676
:10E1D000206A814202D3C6F800B032E0A17D7329E3
:10E1E00002D008B930682062306851461C9A10F09D
:10E1F00061FE216A3368091A0998A3EB0B02801AA1
:10E20000814206DC514618461C9A10F053FE216AE2
:10E21000081A81B2002005E01AE0135C521A135468
:10E22000401C80B2226AABEB02038342F5DCABEB0D
:10E2300001003060206A401A2062206808B1401A4C
:10E240002060A07D732803D0206A08B9306820625E
:10E25000207908B930682060607F692821D0A068E3
:10E26000F8B1E16888421CD24FF0200BD4E90201DA
:10E27000884216D2514630461C9AFFF7D1FA3068D0
:10E2800050450ED2617911B180F800B002E0A1686A
:10E2900009780170A068401CA0603068401C3060A4
:10E2A000E4E700204FF0200B009015E05146304687
:10E2B0001C9AFFF7B5FA3068504511D2617911B157
:10E2C00080F800B001E0217E01700098401C80B20F
:10E2D00000903068401C3060079900988842E5D370
:10E2E0000B9888B1306850450ED2617911B180F831
:10E2F00000B001E02D2101703068401C3060606A80
:10E3000010B1208D401C2085B9F1000F04D0A06809
:10E3100004900020009056E0514630461C9AFFF7CA
:10E320007FFA3068504550D2617969B180F800B009
:10E330000CE0000020C0072024C0072028C00720D0
:10E34000320400106CCC0720302101703068401C72
:10E350006D1EADB2306038E0BDB3514630461C9AF8
:10E36000FFF75EFA306850452FD2617F692904D0EB
:10E370006179C1B180F800B01BE0A168C9B1E26861
:10E38000914216D2617911B180F800B002E004998F
:10E39000097801700498401C0490E168814208D813
:10E3A000A068049005E00F99097801700F98401C4F
:10E3B0000F9000986D1E401C80B200903068ADB286
:10E3C000401C306000984845C6D3B8F1000F76D0A5
:10E3D0009DB1514630461C9AFFF722FA30685045ED
:10E3E0000BD2617911B180F800B001E02E210170EB
:10E3F0003068401C6D1EADB23060474520D2A8EB9E
:10E4000007074FF000094FF0300817E0514630463B
:10E410001C9AFFF705FA3168514511D2607910B1A5
:10E4200081F800B001E081F8008009F101001FFAD5
:10E4300080F96D1E3068ADB2401C30604F45E5DCA0
:10E440000F98F7F732FF1FFA80F8002719E05146BE
:10E4500030461C9AFFF7E4F9306850452AD26179BA
:10E4600011B180F800B005E00F99097801700F989C
:10E47000401C0F907F1C6D1E3068BFB2401CADB2B7
:10E480003060474516D2002DE1D118E051463046A4
:10E490001C9AFFF7C5F93068504510D2617909B16F
:10E4A000077001E080F800806D1E3068ADB2401C3E
:10E4B000306002E04FF030085F46002DE6D1607F0B
:10E4C0004D2818D000255F4612E0514630461C9A70
:10E4D000FFF7A6F9306850450DD2617909B1077090
:10E4E00001E0617E01706D1C3068ADB2401C30608F
:10E4F0000A988542E9D3E06AF0B1216B88421BD8C3
:10E500004FEA0B05D4E90B01884215D85146304635
:10E510001C9AFFF785F9306850450DD2617909B131
:10E52000057002E0E16A09780170E06A401CE0626F
:10E530003068401C3060E5E7607F4D287FF401AD16
:10E5400000255F4613E0514630461C9AFFF768F9F4
:10E5500030685045BFF4F5AC617909B1077001E04E
:10E56000617E01706D1C3068ADB2401C30600A984D
:10E570008542E8D3E5E400002DE9FF4FA5B09146C0
:10E58000329FDDE936643878349D4FF00108FF286A
:10E5900013D120780721305C00EBC000284440787C
:10E5A000B1EB101F02D30009387006E03946202075
:10E5B000F9F788FF08B187F80080787848B92078A3
:10E5C000305C00EBC00028444078C0F38000401C61
:10E5D0007870B87848B92078305C00EBC0002844E7
:10E5E0004078C0F3C000401CB870F87870B920784B
:10E5F000305C00EBC0002844C07900F00300411EED
:10E60000022901D8F87001E087F803803879FF28E3
:10E6100007D12078305C00EBC0002844C0790009A5
:10E620003871B7F805004FF0FF08FE280CD12078AC
:10E63000305C00EBC000284480780F2802D8A7F88F
:10E64000050001E0A7F80580F81DF7F72EFEADF8EC
:10E650003C0040F257203899ADF84400002081F882
:10E6600000801C90229014901790139016901E908A
:10E670002190189015901B9012901D902390207857
:10E68000305C00EBC0002844807910F0030006D015
:10E69000012806D0022832D0032805D131E03020ED
:10E6A00000E000208DF86C002078305C00EBC000AA
:10E6B00028448079400602D572208DF858002078D1
:10E6C000305C00EBC0002844C079C0F381017020A9
:10E6D000022918D0032918D08DF8500020784FF067
:10E6E0006D08305C00EBC00028448079C0F38100E5
:10E6F00001280DD002280ED0032813D149E07A203A
:10E70000D0E77320CEE78DF850008DF85400E5E790
:10E710008DF8508040E000208DF850005FF0300010
:10E720008DF854002078305C00EBC00028448079DC
:10E73000C00602D563208DF870002078305C00EBB5
:10E74000C00028448079800602D565208DF85C00E1
:10E750002078305C00EBC00028448079000602D5A8
:10E760005A208DF874002078305C00EBC0002844FB
:10E770004078C00702D053208DF88C002178339860
:10E78000715C008801EBC10129440979884219D3E1
:10E7900022E04D208DF850000020C1E7BDF83C007C
:10E7A000BDF84410884208D24BA1F81DF7F749FD87
:10E7B000BDF83C00401CADF83C003398339900880C
:10E7C000401C088021783398715C008801EBC101FE
:10E7D000294409798842E1D32078305C00EBC000FD
:10E7E00028448079800625D500208DF850808DF84A
:10E7F000540013E0BDF83C00BDF84410884208D234
:10E8000035A1F81DF7F71DFDBDF83C00401CADF823
:10E810003C00339833990088401C08802078305C95
:10E8200000EBC00028440179407901443398008806
:10E830008142DFD82078305C00EBC0004119087AB3
:10E84000B8B149788A074FF0200102D58DF84C0005
:10E8500001E08DF848007C280BD18DF84810207815
:10E86000305C00EBC0002844007A8DF849008DF838
:10E870004A003599BF205E2902D05F2903D004E009
:10E880008DF8880001E08DF88400BDF84410BDF8D3
:10E890003C00814201D9091A00E000210904090C59
:10E8A0000E911BD02699DDF898C04FEA194B359B85
:10E8B0004FEA114A1FFA89F91FFA8CFC0DF1700E0C
:10E8C0000DF148080AF0FF0109F0FF02CDF864C01D
:10E8D000C42B03D203E00000200000001AE25FEA2C
:10E8E000830CFC44DCF806C0E7440000840300000D
:10E8F00084030000840300008403000084030000FC
:10E9000084030000840300008403000084030000EB
:10E910001003000010030000840300004C060000F8
:10E9200092060000DE0500001406000084030000CB
:10E9300084030000D20600008C0C0000400D000093
:10E94000CC0C0000020D00007C0D0000020D000048
:10E950007C0D000084030000620500001E0C000016
:10E9600098110000A0050000D80A000084030000F0
:10E97000840300008403000084030000D20600002A
:10E980006804000068040000D80A00008403000046
:10E9900084030000D2060000C4100000C410000070
:10E9A00010110000D80A0000C4100000C4100000BC
:10E9B00010110000D80A0000C4100000C4100000AC
:10E9C00010110000D80A0000C4100000C41000009C
:10E9D00010110000D80A0000C4100000C41000008C
:10E9E00010110000D80A0000C4100000C41000007C
:10E9F00010110000D80A0000440A0000800A00003C
:10EA0000CC0A00008403000084030000840300009B
:10EA1000D2060000EE040000EE040000D80A000058
:10EA20008403000084030000480300008403000006
:10EA3000840300008403000010030000840300002E
:10EA4000D203000084030000D2030000840300000E
:10EA5000840300002A0400008403000084030000F3
:10EA6000840300008403000084030000840300008A
:10EA7000840300008403000084030000840300007A
:10EA8000D20300008403000084030000840300001C
:10EA9000840300008403000084030000840300005A
:10EAA00084030000840300001003000084030000BE
:10EAB0001003000084030000D20300008403000060
:10EAC000840300008403000084030000840300002A
:10EAD0001003000084030000100300008403000002
:10EAE0008403000084030000560C0000840300002F
:10EAF00084030000D20600008403000084030000A9
:10EB0000D2060000521100005211000084030000E0
:10EB100084030000840300008403000084030000D9
:10EB200084030000840300008403000084030000C9
:10EB300084030000840300008403000084030000B9
:10EB400084030000840300008403000084030000A9
:10EB50008403000084030000840300008403000099
:10EB6000840300008403000084030000A604000066
:10EB7000A6040000D80A00008403000084030000FB
:10EB800084030000D2060000840300008403000018
:10EB9000D20600008403000084030000D2060000B7
:10EBA0003410000074100000840B000034100000CA
:10EBB00074100000840B000034100000741000007A
:10EBC000840B00003410000074100000840B00005F
:10EBD0003410000074100000840B00008403000057
:10EBE0008403000084030000840300008403000009
:10EBF0008403000084030000D20300000DF1180B11
:10EC0000C4461DAB16AA17A98BE80E10227814A9CA
:10EC100015ABB25C0DF14C0C02EBC2022A44384435
:10EC20005279CDE90421CDE902C3CDE900A9FBA2C7
:10EC3000199BF3E30DF11C0EC4461DAB16AA17A9D0
:10EC40008EE80E10227814A915ABB25C0DF14C0CB5
:10EC500002EBC2022A4438445279CDF808B0CDE91B
:10EC60000521CDE903C3CDE900A9F4A2199B7CE3FA
:10EC70000DF1840C1DAA16A9CDE90A12CDE90C8C60
:10EC800094F800C017AA14AB16F80CC038440CEB6B
:10EC9000CC0CAC449CF805C0CDF818C0CDF824E0ED
:10ECA000CDE9073215AB0DF14C0CCDE904C3199A2F
:10ECB000CDE9002ACDE9029B22ABE9A226E021782A
:10ECC000715C01EBC10129444979FF2900D1491C3C
:10ECD000434621AACDE90C320DF1740C0DF1580810
:10ECE000CDE90A8C17AB0DF1500CCDE9083ECDE90A
:10ECF000061C15AB0DF14C0CCDE904C31999CDE9F7
:10ED0000029BCDE9001A384422ABD5A2C01D0E9952
:10ED100043F0B4FA89E316ABCDE90838CDF81CE02E
:10ED2000CDF828B0237814AA17A9F35C0DF1540C80
:10ED300003EBC3032B4438445B79CDE90432CDF8AF
:10ED40000CC0069113ABCDF800A0CDE90193CEA283
:10ED5000199B8CE716ABCDE90838CDF81CE0CDF84F
:10ED600028B0237814AA17A9F35C0DF1540C03EB17
:10ED7000C3032B4438445B79CDE90432CDF80CC091
:10ED8000069113ABCDF800A0CDE90193CBA2199B5E
:10ED90006DE7217843460DF1580C715C384401EB66
:10EDA000C1016A5CCDE9093BCDE907EC294414AB0C
:10EDB0004979CDE90413052A17AA0DF1540CCDF8B1
:10EDC0000CC0069213ABCDF800A0CDE90193199BBE
:10EDD00001D0C8A24BE7D5A249E7217843460DF1FF
:10EDE000580C715CF04601EBC1016A5C052A17D032
:10EDF000CDE9093BCDE9078C294414AB4979CDE92C
:10EE0000041317AA0DF1540C0692CDF80CC013ABE5
:10EE1000CDF800A0CDE901933844D2A2199B26E792
:10EE2000CDE9093BCDE9078C294417AB14AA4979F0
:10EE3000CDE905230DF1540CCDF800A0CDE903C1B7
:10EE400013ABCDE901933844D4A2199B0FE716AB5D
:10EE5000CDE90838CDF81CE0CDF828B0237814AA05
:10EE600017A9F35C0DF1540C03EBC3032B44384496
:10EE70005B79CDE90432CDF80CC0069113ABCDF827
:10EE800000A0CDE90193D3A2199BF0E616ABCDE922
:10EE90000838CDF81CE0CDF828B0237814AA17A9BB
:10EEA000F35C0DF1540C03EBC3032B4438445B7942
:10EEB000CDE90432CDF80CC0069113ABCDF800A01B
:10EEC000CDE90193D1A2199BD1E60DF1140BC446F3
:10EED00016AB17AA14A98BE80E1021780DF14C0C73
:10EEE00015AB715C384401EBC10129444A79CDF876
:10EEF00008C0CDE90332CDE900A9D1A2199B90E366
:10EF00000DF1180BC44616AB17AA14A98BE80E1006
:10EF100022781BA915ABB25C0DF14C0C02EBC202BE
:10EF20002A4438445279CDE90421CDE902C3CDE920
:10EF300000A9CFA2199B3AE330218DF86C100DF196
:10EF40001C0BC4461DAB16AA17A98BE80E1023781C
:10EF50001BA914AAF35C0DF1540C03EBC3032B445F
:10EF600038445B79CDE904310692CDF80CC013AB7F
:10EF7000CDF800A0CDE90193C5A2199BF5E10DF1F3
:10EF80001C0BC4461DAB16AA17A98BE80E102378DC
:10EF90001BAA14A9F35C0DF1540C03EBC3032B441F
:10EFA00038445B79CDE90432CDF80CC0069113AB3F
:10EFB000CDF800A0CDE90193BEA2199BD5E1BE20FA
:10EFC0008DF87800DDE938010DF1040C11AB0FAAC2
:10EFD0008CE80F002078009033462A463846339953
:10EFE000FDF7A4FBC0B123781DA81BAAF35C03EBBB
:10EFF000C3032B445B79CDE906200593CDF820802F
:10F000001EAA13ABCDF808B0CDE90332CDE900A9B3
:10F01000BDF83C00384467E169E10000252525641E
:10F020002F25642F25647C2573257325646425733F
:10F0300025732573257325737C0000002525256421
:10F040002F25642F25642F25647C25732573256463
:10F0500064257325732573257325737C00000000D8
:10F060002573252525642F25642F25642F25647C91
:10F0700025732573256473257325732573257325DF
:10F080007325737C25730000252525642F25642FA7
:10F0900025647C2573257325647325732573257377
:10F0A000257325737C26252532303030302F3131C1
:10F0B00031372F302F25647C31747C002525256461
:10F0C0002F25642F25647C25732573256473257390
:10F0D00025732573257325737C2625253230303022
:10F0E000302F31303035332F302F25647C31747C14
:10F0F00000000000252525642F25642F25647C252C
:10F100007325732564732573257325732573257300
:10F110007C26252532303030302F31303037342FB7
:10F12000302F25647C31747C000000002525256487
:10F130002F25642F25647C2573257325647325731F
:10F1400025732573257325737C26252532303030B1
:10F15000302F31303037332F302F25647C31747CA1
:10F1600000000000252525642F25642F25647C25BB
:10F170007325732564732573257325732573257390
:10F180007C26252532303030302F31303031332F4E
:10F19000302F25647C31747C000000002525256417
:10F1A0002F25642F25647C257325732564732573AF
:10F1B00025732573257325737C2625253230303041
:10F1C000302F31303031352F302F25647C31747C35
:10F1D00000000000252525642F25642F25647C254B
:10F1E0007325732564732573257325732573257320
:10F1F0007C26252532303030302F313037322F31D8
:10F2000030312F25647C31747C0000002525256475
:10F210002F25642F25647C2573257325647325733E
:10F2200025732573257325737C26252532303030D0
:10F23000302F313037322F312F25647C31747C00F0
:10F24000252525642F25642F25647C2573257325AA
:10F25000647325732573257325737C262525323029
:10F260003030302F313032337C31747C000000007C
:10F27000252525642F25642F25647C25732573257A
:10F28000642E3366257325732573257325737C00DF
:10F29000252525642F25642F25647C25732573255A
:10F2A000642E3266257325732573257325732573A4
:10F2B0007C000000252525642F25642F25647C25EE
:10F2C00073257325642E3266257325732573257384
:10F2D000257325737C26252532303030302F313090
:10F2E00032337C31747C0000F5A2199B99E117AB95
:10F2F00008931DA916AACDF82C80CDE90921227802
:10F3000015AB14A8B25C1BA902EBC2022A445279C5
:10F31000CDE90610CDE90432CDE900A913ABCDE962
:10F3200002B3BDF83C00EFA23844199B3AE300BF9A
:10F330008DF8601016ABCDE9073818A9CDE9091B87
:10F3400094F8008017AB0DF1500C16F8088013AA42
:10F3500008EBC808A844384498F80580CDE9053E74
:10F3600015AB8DE80E11E9A2199B87E38DF860209B
:10F3700018AACDE908820DF1580CCDF81CC0CDF8C3
:10F3800028B094F800C017A914AA16F80CC013AB43
:10F390000CEBCC0CAC4438449CF805C0CDE90421FE
:10F3A000CDF818E0CDF80CC015AACDF800A0CDE935
:10F3B0000132E4A2199B61E3BE208DF878008DF83C
:10F3C00060105AE0272B31D05FF0BE008DF8780036
:10F3D000DDE938010DF1040C11AB0FAA8CE80F0028
:10F3E0002078009033462A4638463399FDF79EF937
:10F3F000F0B122781EAB1BA9B25C02EBC2022A4418
:10F400005279CDE90618CDE90432CDE900A913AB54
:10F41000CDE902B3BDF83C00384400E0C7E0199BD9
:10F42000D6A2C01D0E9942F029FF2BE32D20CDE777
:10F4300016A917AACDE9082114AB0793CDF82880A7
:10F4400021781BA815AA715C13AB01EBC1012944FB
:10F450004979CDF808B0CDE90510CDE90332CDE901
:10F4600000A9BDF83C00CDA23844199B06E300BFBB
:10F47000BE208DF860108DF87800DDE938010DF1BF
:10F48000040A11AB0FAA8AE80F00207800903346D7
:10F490002A4638463399FDF749F9C0B122781EABA8
:10F4A0001BA8B25C02EBC2022A4452790493CDF845
:10F4B0001C80CDE9052018ABCDE9003913AACDE9B0
:10F4C00002B2BDF83C00BEA23844199BA9E716A9B8
:10F4D00017AA14ABCDE908210793CDF8288021782D
:10F4E00015AA1BA8715C13AB01EBC1012944497932
:10F4F0000393CDE90421069018AA8DE8040ABDF80B
:10F500003C00B8A23844199BB8E20DF1180BC44670
:10F510001DAB16AA17A98BE80E10227814A915ABFB
:10F52000B25C0DF14C0C02EBC2022A443844527911
:10F53000CDE90421CDE902C3CDE900A9B3A2199B0D
:10F5400035E00DF1140BC44616AB17AA14A98BE8CD
:10F550000E1021780DF14C0C15AB715C384401EBA9
:10F56000C10129444A79CDF808C0CDE90332CDE97B
:10F5700000A9AFA2199B54E00DF1180BC4461DABB6
:10F5800016AA17A98BE80E10227814A915ABB25C45
:10F590000DF14C0C02EBC2022A4438445279CDE9F9
:10F5A0000421CDE902C3CDE900A9199BABA2C01D7E
:10F5B0000E9942F063FE65E20DF1140BC44616ABE2
:10F5C00017AA14A98BE80E1021780DF14C0C15AB7D
:10F5D000715C384401EBC10129444A79CDF808C077
:10F5E000CDE90332CDE900A9A4A2199B19E00DF1E0
:10F5F000140BC44616AB17AA14A98BE80E10217879
:10F600000DF14C0C15AB715C384401EBC101294480
:10F610004A79CDF808C0CDE90332CDE900A9199B9C
:10F62000A2A2C01D0E9942F029FE2BE20DF11C0B87
:10F63000C4461DAB16AA17A98BE80E1023781BAA87
:10F6400014A9F35C0DF1540C03EBC3032B443844B1
:10F650005B79CDE90432CDF80CC0069113ABCDF83F
:10F6600000A0CDE9019358E1BE208DF87800DDE9D6
:10F6700038010DF1040B11AB0FAA8BE80F002078B5
:10F68000009033462A4638463399FDF74FF8A8B123
:10F6900023781BA91DA8F35C1EAA03EBC3032B440C
:10F6A0005B79CDE90431CDE90608CDE900A913ABBA
:10F6B000CDE90232BDF83C0038440FE111E1000011
:10F6C000252525642F25642F25642F25647C25732B
:10F6D000257325642E326625736D65257325737C2D
:10F6E00000000000252525642F25642F25642F2583
:10F6F000647C2573257325642E3266257325732556
:10F70000732573257325737C00000000252525646F
:10F710002F252525737C2573257325647325732573
:10F72000732573257325737C2625253230303030C0
:10F730002F31303037352F252525732F25647C3127
:10F74000747C0000252525642F25647C2573257392
:10F75000256473257325732573257325737C2625EE
:10F760002532303030302F31303037352F252525B8
:10F77000732F25647C31747C0000000025252564EE
:10F780002F25642F25642F25647C2573257325641C
:10F790002E326625736D6525737C00002525256452
:10F7A0002F25642F25642F25647C257325732564FC
:10F7B0002E3266257325732573257325737C00000F
:10F7C000252525642F252525732F25642F25647C69
:10F7D0002573257325642E326625736D6525737C2C
:10F7E00000000000252525642F252525732F25647D
:10F7F0002F25647C2573257325642E326625732599
:10F80000732573257325737C00000000252525646E
:10F810002F25642F25647C2573257325642E32667D
:10F8200030257325732573257325737C0000000034
:10F83000252525642F25642F25647C2573257325B4
:10F84000647325732573257325737C252531393918
:10F8500039392F317C310A7C0000000025252564D0
:10F860002F25642F25647C257325732564732573E8
:10F8700025732573257325737C00000025252564D9
:10F880002F25642F25647C257325732564732573C8
:10F890002573257325737C26252532303030302F93
:10F8A00031303036317C31747C00000025252564F0
:10F8B0002F25642F25647C25732573256473257398
:10F8C0002573257325737C26252532303030302F63
:10F8D00031303036327C31747C00000082A2199BBA
:10F8E0009FE51DA916AA17ABCDE908210793CDF80E
:10F8F000288022781BA914A8B25C15AB02EBC202C7
:10F900002A445279CDE904210690CDE900A9BDF839
:10F910003C0013AACDE9022338447FA2199BADE035
:10F920008DF8601018ABCDF82C90CDF82080CDE983
:10F93000093B17AB0DF1500C16AACDE904C3CDE974
:10F9400006E2217815AB0DF14C0C715C384401EBEB
:10F95000C10129444A79CDE9009CCDE902321FE07A
:10F960008DF8602028990DF1600C8AB2CDE90AB2B9
:10F97000CDE9088C0DF15C0C14AB16A9CDE9043C63
:10F98000CDE906E1217815AB0DF14C0C715C3844E2
:10F9900001EBC10129444A79CDE900ACCDE902323D
:10F9A000199B6AA2C01D0E9942F068FC6AE000BF74
:10F9B0000DF18C0CCDE90A8ACDF824C016A9CDF83A
:10F9C00030B0CDE907E117AB0DF1500CCDE905C31F
:10F9D00021780DF14C0C15AB715C384401EBC10181
:10F9E0002944C01D4A7951468DE80212CDE90332FF
:10F9F00064A2199B0E9942F041FC43E00DF1580CB2
:10FA000008A94346CDF81CC081E8080A94F800C054
:10FA100017AB14A916F80CC015AA0CEBCC0CAC440F
:10FA200038449CF805C0CDE9053ECDF800A0CDE9ED
:10FA300003C113ABCDE9013260A2199B1EE00DF1A9
:10FA40001C0BC4461DAB16AA71468BE80E1023781A
:10FA500014AA17A9F35C0DF1540C03EBC3032B4458
:10FA600038445B79CDE90432CDF80CC0069113AB74
:10FA7000CDF800A0CDE90193199B5DA2C01D0E99A0
:10FA800042F0FCFB9DF84C0010B99DF8480080B195
:10FA9000339833990088401C80B208802178715CCB
:10FAA00001EBC1012944097A7C2902D13399401C18
:10FAB00008802078305C00EBC000284481798906FA
:10FAC00005D433994079098808443399088050490E
:10FAD000002008604F49086078464F49086029B007
:10FAE0000020BDE8F08F0000252525642F25642F18
:10FAF00025647C2573257325642E326625736D6518
:10FB0000257325737C26252532303030302F313057
:10FB10003036327C31747C00252525642F25642FF6
:10FB200025647C2573257325642E32662573257321
:10FB300025732573257325737C26252532303030B7
:10FB4000302F31303036327C31747C0025252564ED
:10FB50002F25647C257325732564732573257325F0
:10FB600073257325737C26252532303030302F31B4
:10FB7000303037352F252525732F25642F25647CBC
:10FB800031747C00252525642F25642F25647C2570
:10FB90007325732564732573257325732573257366
:10FBA00025737C26252532303030302F31303034EB
:10FBB000342F25642F25647C31747C002525256431
:10FBC0002F25647C25732573256473257325732580
:10FBD00073257325737C26252532303030302F3144
:10FBE000303034342F25642F25647C31747C000040
:10FBF000252525642F25642F25647C2573257325F1
:10FC000064672573257325732573257325737C001D
:10FC100020C0072024C0072028C0072070B50E4848
:10FC200000250F4E45600D482C460570204600F01B
:10FC30001DF8000601D5306870BD641CE4B2022CCA
:10FC4000F4D33CF0CDFA35600648056078460649A5
:10FC50000860002070BD0000A4C107203C01001016
:10FC600020C0072024C0072028C007202DE9F14F1D
:10FC7000ADF5276D00200090DDF8700A40F2E462D7
:10FC8000C0EB8010C0EBC00141F6451000EB8100D5
:10FC900040F0805008A941F07DFF000605D5D54809
:10FCA00000680DF6742DBDE8F08F0020CDF85C0AD9
:10FCB000CDF8540ACDF8580ACDF8480ACDF84C0AC8
:10FCC000C4210DF65422CDF8500A1154401CC0B284
:10FCD00092460A28F9D3C84A00210DF6482808ACF4
:10FCE0005FF0000000EBC003E55C8D420ED12344C1
:10FCF0005D795DB1DB784BB11AF80150AB4205D8A4
:10FD000018F80150AB4201D908F8013000EB40036C
:10FD100012F82330072B00D10290401CC0B2C42837
:10FD2000E0D3491CC9B20A29DAD300214FF00109F6
:10FD300001EB410012F82070BC2F08D101EBC10586
:10FD4000635D012B03D125440023EB706B7102EB43
:10FD500080004368002B0CDA01EBC1002044457998
:10FD60003DB918254571862F03D101250095002541
:10FD7000C57001EBC105605D09FA00F61E420AD1AB
:10FD80000020CC460CFA00F6334203D1401CC0B22E
:10FD90000A28F7D36055002B18DA05EB040C9CF801
:10FDA00003301BB11AF80060B3420FD918F80030C5
:10FDB0005B1CDEB208F800601AF800309E4201D9E0
:10FDC00008F8003018F800008CF80300862F0FD1D7
:10FDD000009868B1002000900298072300EBC00053
:10FDE00023542B192044DB780833C37080F8059026
:10FDF000491CC9B2C4299BD30DF2DB700026CDF893
:10FE0000400AC4210DF5E160F6F710FA00210D4615
:10FE100001EBC100225CB2423ED120444279DAB308
:10FE2000C078C8B31AF80620904235D80DF5E16EB7
:10FE30000EF805108DF8605A27E000BF0EEB0003A6
:10FE4000039313F8013C009303EBC3031EF8002057
:10FE500003EB040802EBC203234498F8037093F801
:10FE600003C0674515D3774604D198F804C01B79C1
:10FE70009C450ED9039BDDF800C003F8012C07F860
:10FE800000C0A0F101008DF8600A9DF8600A00280A
:10FE9000D4D105F10105EDB201F10101C9B2C429C6
:10FEA000B6D34FF0000E70468DF860EA5FE020B3E5
:10FEB0000DF5E1610A18095C12F8012C01EBC10192
:10FEC00002EBC20222442144D278C978521C8A42F1
:10FED00049D200BF0DF5E163195C01EBC10121447A
:10FEE000C97840B11A1812F8012C02EBC202224460
:10FEF000D278891AC9B2002219E09DF8081701EBDF
:10FF0000C1012144C9780129E4D12CE0A5EB020C00
:10FF10000DF5E1630CEB03088C44634418F8017C95
:10FF200003F8027CFF23521C08F8013CD2B22B1AC2
:10FF30009342EBDC2A1A8A420EDAD2B2A1F101080E
:10FF40000DF5E167FF2305E000EB020C521C07F8FA
:10FF50000C30D2B24245F7DB6A18521E0844401EEC
:10FF6000D5B28DF8600AC0B2401C8DF8600AC0B2EC
:10FF7000A8429CD3ADF868EA4FF41A710DF2CC7028
:10FF8000F6F754F9FF20FE218DF8D8078DF8D40735
:10FF9000ADF8D917002D31D000218DF8601A8DF8F9
:10FFA000640AFDE30DF5E16818F80020FF2A26D069
:10FFB000DDF80437002161F30F0361F31F43CDF82F
:10FFC00004375B4661F30F0361F31F439B4602EB6B
:10FFD000C2031F194146BF793F0603D45F4669F348
:10FFE0001F47BB4602EB4207034A12F82720C42AE8
:10FFF00006D206E020C00720E8BB0500F8E3F8E3DE
:020000040001F9
:1000000087E397007F447F68BF440000100300002F
:100010002403000024030000240300002403000044
:100020002403000024030000240300002403000034
:10003000440300004C0300005C0300006403000064
:100040006C030000740300007C03000084030000C4
:100050008C030000940300009C030000A803000030
:10006000B80300008C030000C80300008C030000EC
:10007000D0030000E0030000E8030000F0030000EC
:10008000B80300008C030000F80300000004000027
:1000900008040000100400008C0300002404000089
:1000A0002C0400004004000050040000580400002C
:1000B0008C0300006C04000074040000AC04000019
:1000C0000C050000980500007C040000B40400004A
:1000D0002C050000A005000084040000CC040000F2
:1000E00034050000A805000094040000DC040000B2
:1000F00050050000B00500009C040000EC04000066
:100100006C050000B8050000A4040000FC04000019
:1001100088050000C0050000C8050000D0050000EB
:10012000EC050000080800001C0800008C0300001B
:10013000240800002C0800008C0300003E0800008A
:1001400050080000580800006C08000090080000EB
:10015000A4080000AC080000C0080000C8080000A7
:10016000DC080000E4080000F808000000090000B6
:10017000140900001C0900003009000038090000C3
:100180004C090000540900006809000070090000D3
:10019000840900008C090000A0090000A8090000E3
:1001A000BC090000C4090000D4090000E8090000EF
:1001B000F0090000F8090000000A0000080A000029
:1001C000100A0000240A0000380A0000400A00005B
:1001D000540A00005C0A0000700A0000780A00005F
:1001E0008C0A0000940A0000A80A0000B00A00006F
:1001F000C40A0000CC0A0000E00A0000E80A00007F
:10020000FC0A0000040B00002C0B0000FC050000A1
:100210008C03000010060000180600008C0300008C
:100220002C060000340B0000480B00000C0B0000F3
:10023000140B00001C0B0000240B0000040B00003A
:100240000C0B0000140B00001C0B0000240B000022
:10025000040B00000C0B0000140B00001C0B000032
:10026000240B0000040B00000C0B0000140B00001A
:100270001C0B0000240B0000040B00000C0B000002
:10028000140B00001C0B0000240B0000580B000096
:100290008C0300006A0B00005403000034060000C9
:1002A0008C03000048060000500600008C0300008C
:1002B000640600006C0600008C030000800600004D
:1002C000880600009C060000C0060000D006000062
:1002D000D806000008070000240700002C070000D3
:1002E000500700006C070000740700009C07000026
:1002F000B8070000C0070000E8070000940B0000EA
:100300009C0B00009C0B00009C0B00009C0B000051
:100310009C0B0000A40B0000BC0B0000DDF80437B0
:1003200043F2154767F30F0342F23F777AE200BFCB
:10033000DDF8043743F2154767F30F034FF41D57F9
:1003400067F31F43CDF804375B4662F30F032EE0DB
:1003500042F219776AE200BF42F21B7766E200BF01
:1003600042F24B7762E200BF40F206475EE200BF16
:1003700042F21E775AE200BF40F2374756E200BF12
:1003800042F66837DEE300BF40F2FF374EE200BFBF
:1003900040F2AD474AE200BF42F66837DCE300BFF7
:1003A00040F2134742E200BF42F24C7704E09B4622
:1003B000ECE300BF42F24D77DDF8043767F30F033B
:1003C000B3E000BFDDF8043742F6683767F30F0388
:1003D0000327F5E342F24E77EEE700BFDDF804377E
:1003E0004FF4856767F30F03C1E000BF42F23C772B
:1003F000E2E700BF40F22947DEE700BF40F22E47A8
:10040000DAE700BF4FF48667D6E700BF40F2BC478B
:10041000DCE300BF40F2BE47D8E300BFDDF804379D
:1004200043F2154767F30F0342F24477C8E300BF76
:1004300042F24477CAE300BFDDF8043743F21547C0
:1004400067F30F0342F24677BAE300BFDDF80437E3
:1004500042F6683767F30F030427B1E342F24577AA
:10046000B4E300BFDDF8043743F2154767F30F0329
:100470004FF47F77A4E300BF4FF47F77A6E300BF7C
:1004800042F23C77AEE200BF42F23C771AE000BF96
:1004900042F23C7722E00227CDF80437B6E100BFF4
:1004A00042F23C7722E000BF42F23C7726E000BFF8
:1004B00042F23C772AE000BF40F2294792E200BFB7
:1004C00040F22947DDF8043767F30F03022767F38B
:1004D0001F43CDF8043799E140F22947DDF804378E
:1004E00067F30F030327A0E240F22947DDF8043742
:1004F00067F30F03042798E240F22947DDF8043739
:1005000067F30F03052790E240F22947DDF804372F
:1005100067F30F03062788E2DDF8043742F66837F1
:1005200067F30F03022767F31F43CDF804375B46D9
:1005300069F30F033BE700BF42F66837C2E700BF2D
:10054000DDF8043742F6683767F30F03022767F3D5
:100550001F430327CDF8043758E100BFDDF8043707
:1005600042F6683767F30F03022767F31F43042738
:10057000CDF804374AE100BFDDF8043742F66837AA
:1005800067F30F03022767F31F430527CDF80437EE
:100590003CE100BFDDF8043742F6683767F30F032C
:1005A00002277AE04FF486671CE200BF4FF48667AB
:1005B00088E700BF4FF4866790E700BF4FF4866777
:1005C00094E700BF4FF4866798E700BF4FF4866753
:1005D0009CE700BF42F2507710E000BFDDF804371F
:1005E00042F6683767F30F03022767F31F43642758
:1005F000CDF804370AE100BF42F25B77DDF804373B
:1006000067F30F036427DBE2DDF8043743F2154795
:1006100067F30F0340F20747D2E200BF40F20747FB
:10062000D4E200BFDDF8043743F2154767F30F0348
:1006300040F23947C4E200BF40F23947C6E200BF8A
:10064000DDF8043743F2154767F30F0340F2BF4765
:10065000B6E200BF40F2BF47B8E200BFDDF80437A2
:1006600043F2154767F30F034FF49867A8E200BF02
:100670004FF49867AAE200BFDDF8043743F215474C
:1006800067F30F0340F2C1479AE200BF40F2C1474F
:100690009CE200BF42F250771AE067F31F4306273F
:1006A000CDF80437B2E000BFDDF8043742F6683712
:1006B00067F30F03022767F31F43CDF8043764275E
:1006C0005B4667F30F039B4606271CE042F25B770D
:1006D000DDF8043767F30F036427DEE742F2507753
:1006E0001AE000BFDDF8043742F6683767F30F03FE
:1006F000022767F31F43CDF8043764275B4667F38F
:100700000F039B460727DDF8443A67F30F03CDF844
:10071000443A3BE242F25B77DDF8043767F30F03BC
:10072000642767F31F430727CDF804376EE000BF47
:1007300042F2507714E000BFDDF8043742F6683724
:1007400067F30F03022767F31F43CDF804376427CD
:100750005B4667F30F039B460827D4E742F25B77BB
:10076000DDF8043767F30F03642767F31F43082797
:10077000CDF804374AE000BF42F2507716E000BFE0
:10078000DDF8043742F6683767F30F03022767F393
:100790001F43CDF8043764275B4667F30F0300E07F
:1007A0008BE29B460927AEE742F25B77DDF8043720
:1007B00067F30F03642767F31F430927CDF8043756
:1007C00024E000BF42F2507716E000BFDDF80437A6
:1007D00042F6683767F30F03022767F31F43CDF82C
:1007E000043764275B4667F30F039B460A278AE7B3
:1007F0006CE207E242F25B77DDF8043767F30F0340
:10080000642767F31F430A27CDF804375B4667F375
:100810000F03CCE5DDF8043743F2154767F30F0308
:1008200042F6FF07CCE100BF42F24177CEE100BFC4
:1008300042F24277CAE100BFDDF8043743F21547C0
:1008400067F30F0342F60117BAE1E35C052B02D010
:1008500042F21D77BAE142F21F77B7E142F2137715
:10086000B4E100BFDDF8043743F2154767F30F0327
:1008700042F60317A4E100BFDDF8043742F2107717
:1008800067F30F03022767F31F43CDF804375B4676
:1008900069F30F0369F31F4389E500BFDDF80437EF
:1008A00043F2154767F30F0340F2FD3788E100BFBD
:1008B00040F2FD378AE100BFDDF8043743F2154707
:1008C00067F30F0342F602177AE100BF42F2167790
:1008D0007CE100BFDDF8043743F2154767F30F03EF
:1008E0004FF483676CE100BF4FF483676EE100BF94
:1008F000DDF8043743F2154767F30F0340F2F13791
:100900005EE100BF40F2F13760E100BFDDF804377F
:1009100043F2154767F30F034FF47C7750E100BFB4
:100920004FF47C7752E100BFDDF8043743F21547FE
:1009300067F30F0340F25D4742E100BF40F25D47BD
:1009400044E100BFDDF8043743F2154767F30F03B6
:1009500040F20C4734E100BF40F20C4736E100BFE3
:10096000DDF8043743F2154767F30F0340F2F5371C
:1009700026E100BF40F2F53728E100BFDDF804377B
:1009800043F2154767F30F0340F2FA3718E100BF4F
:1009900040F2FA371AE100BFDDF8043743F2154799
:1009A00067F30F0340F21F470AE100BF40F21F4701
:1009B0000CE100BFDDF8043743F2154767F30F037E
:1009C00040F2A347FCE000BF40F2A347FEE000BFB7
:1009D000DDF8043740F2544767F30F035BE500BFCF
:1009E00040F22147DDF8043767F30F0369F31F4333
:1009F00051E500BF40F2214764E500BF40F22147C6
:100A00006CE500BF40F2214770E500BF40F221478E
:100A100074E500BF40F2214778E500BFDDF80437F8
:100A200040F2214767F30F03072767F31F4332E5BF
:100A3000DDF8043743F2154767F30F0340F20E4722
:100A4000BEE000BF40F20E47C0E000BFDDF8043753
:100A500043F2154767F30F0340F21247B0E000BFBF
:100A600040F21247B2E000BFDDF8043743F2154709
:100A700067F30F0340F22447A2E000BF40F224478F
:100A8000A4E000BFDDF8043743F2154767F30F0316
:100A900040F20D4794E000BF40F20D4796E000BFE2
:100AA000DDF8043743F2154767F30F0340F21147AF
:100AB00086E000BF40F2114788E000BFDDF8043750
:100AC00043F2154767F30F034FF4826778E000BFE6
:100AD0004FF482677AE000BFDDF8043743F2154730
:100AE00067F30F0340F235476AE000BF40F2354735
:100AF0006CE000BFDDF8043743F2154767F30F03DE
:100B00004FF47D775CE000BF4FF47D771AE000BFC3
:100B100043F698275AE000BF43F6992756E000BFF6
:100B200043F69A2752E000BF43F69B274EE000BFF2
:100B300043F69C274AE000BF42F6041746E000BF98
:100B400042F66937DDF8043767F30F0369F31F4393
:100B50001AE000BF42F66937DDF8043767F30F0388
:100B600002272DE0DDF8043743F2154767F30F0342
:100B700042F2597724E0E35C052B02D042F25A7727
:100B800024E042F2597721E0CDF804379DF8643A29
:100B9000FF2B20D098421ED1FF208DF8640A44E03C
:100BA00042F66A3712E000BF43F6E513D7180DE0AE
:100BB000DDF8043743F2154767F30F0340F2164799
:100BC00067F31F43E0E700BF40F21647DDF8043744
:100BD00067F30F03D8E70DF66420031FCDE9041374
:100BE000CDE90605011D03920DF2D4708DE81300C6
:100BF0005A46DDF8443ADDF80417DDF8700AFDF7CF
:100C0000BBFC12E000208DF8D4078DF8D8078DF8D2
:100C1000D5978DF8D697FF21ADF8D9178DF8D797CE
:100C20003AA1DDF8400AF5F70CFB9DF8600A411C7B
:100C3000A94212D03CD218F800204044FF2A407844
:100C400041D0FF2809D002EBC20100EBC0002144D3
:100C50002044C978C07881422AD0DDF8400AF5F7EF
:100C600024FB38B133460DF2CC712948DDF8702AE7
:100C70003FF092FA0020ADF8680A4FF41A710DF2B5
:100C8000CC70F5F7D3FA9DF8600A401CA84207D152
:100C900033460DF2CC711E48DDF8702A3FF07CFA25
:100CA000FF208DF8D4078DF8D807FE20ADF8D907BE
:100CB0009DF8600A401C8DF8600A9DF8600AA84201
:100CC000FFF470A910E0FF28C7D1F1E74FF41A71C3
:100CD0000DF2CC70F5F7AAFA33460DF2CC710C4840
:100CE000DDF8702A3FF058FA761CF6B20A2EFFF4AF
:100CF00088A8084900200860074908607846074925
:100D000008600DF6742D0020BDE8F08F0A00000089
:100D1000A8C1072020C0072024C0072028C0072022
:100D200070B50C4605460649064802F0ECF8224626
:100D30002946BDE870404FF48073024802F0B2B813
:100D4000086A0500E803001008B500208DF80000CF
:100D500001226946014840F04BFF08BDFC0C002011
:100D600070B50E4604460025F5F760FA3246214676
:100D7000044840F00FFF000601D5284670BD3046FC
:100D800070BD0000FC0C002008B500208DF80000AC
:100D900001226946024840F0FDFE9DF8000008BDB2
:100DA000FC0C002008B501208DF8000002466946C1
:100DB000014840F01DFF08BDFC0C002038B50020A4
:100DC0000A4C8DF8000001226946204640F0E2FE00
:100DD000000609D49DF800100122491C8DF800106E
:100DE0006946204640F004FF38BD0000FD0C00209D
:100DF00008B500208DF8000001226946084840F03F
:100E0000C9FE00060AD49DF800000122401C8DF89E
:100E1000000003486946401E40F0EAFE08BD00009D
:100E2000000D002070B505462E21F5F734FA0400B8
:100E300006D0F5F73AFA0246611C2046F5F7CEF9DE
:100E40002846BDE87040F5F730BA000008B5012229
:100E50006946054840F09EFE9DF800005A2801D0E2
:100E6000012008BD002008BD572C001008B55A20ED
:100E70008DF8000001226946024840F0B9FE3BF0BF
:100E800023FF08BD572C001010B5012021F090FD64
:100E9000114C000618D40121084621F0A1FF0006DC
:100EA00012D4052021F0B6FE00060DD40B4B1822FB
:100EB0006421002021F068FB000605D4002108A071
:100EC00021F0A0FB000601D5206810BDBDE8104050
:100ED000012021F019BA000020C00720F15D0500B3
:100EE000203420363032323432203030313733370C
:100EF0000A200A200A00000010B5002021F0B8FEE8
:100F0000214C000635D4002120A021F07BFB0006F7
:100F10002FD40121084621F063FF000629D40021C7
:100F20001BA021F06FFB000623D40221012021F039
:100F300057FF00061DD4002115A021F063FB000619
:100F400017D40121022021F04BFF000611D400210B
:100F50000FA021F057FB00060BD40221084621F018
:100F60003FFF000605D4002109A021F04BFB00063D
:100F700001D5206810BD002020600849086078462F
:100F800007490860002010BD20C00720200A00008B
:100F900031323520544543540A00000024C0072054
:100FA00028C0072070B58AB0064605A821F0E8FCE5
:100FB000174C00061FD4684621F0E2FC00061AD444
:100FC0000121ADF80210ADF80410ADF80A10ADF82B
:100FD0000610ADF8006004252946304622F0ACFC2E
:100FE000000608D4ED1C0F2DF6D3002105A821F032
:100FF00027FA000602D520680AB070BD00202060E4
:10100000044908607846044908600020F4E70000BD
:1010100020C0072024C0072028C0072010B5ACB08E
:1010200026A821F0ADFC234C00063CD421A821F0D9
:10103000A7FC000637D40220ADF88E00ADF886007C
:10104000ADF888000A20ADF88A00002121A821F01F
:10105000F7F9000627D418A31AA28221684641F0A6
:101060000DF919480A21C089420868463AF03BFF49
:101070000021684621F0C6FA0121084621F0B0FEA1
:10108000000610D4002111A021F0BCFA00060AD4F9
:10109000002126A821F0D4F9000604D4012021F073
:1010A00087FC000602D520682CB010BD21F0E6FFB9
:1010B000FAE7000020C0072080928E8B2031353067
:1010C0009400000025730A003204001084A5ACAE21
:1010D000ADE1E2E0A0E6A8AEADADA0EF20AFA5E7A0
:1010E000A0E2EC0A200A000070B500F09DF810495B
:1010F000104D114E114C087050B1114900EB800099
:1011000001EBC000C0688047000609D5206870BDAB
:10111000822020602120286078463060822070BDC7
:1011200000202060286078463060002070BD0000FC
:10113000E8C2072024C0072028C0072020C00720BD
:101140007CC6050070B5144A144D154E1278154C26
:101150005AB190B1144B02EB820203EBC202526A05
:101160009047000611D5206870BD822020602120A4
:10117000286078463060822070BD8620206009207B
:10118000286078463060862070BD0020206028608E
:1011900078463060002070BDE8C2072024C00720D8
:1011A00028C0072020C007207CC605000A48007818
:1011B00030B10A4900EB800001EBC00040680047F5
:1011C00007498220086007492120086078460649BF
:1011D0000860822070470000E8C207207CC6050036
:1011E00020C0072024C0072028C007200948007815
:1011F00028B1094900EB800051F830000047074949
:101200008220086006492120086078460549086068
:1012100082207047E8C207207CC6050020C0072056
:1012200024C0072028C0072070B5002400BF00BFDD
:1012300000BF00BF00BF00BF00BF00BF00BF00BFB6
:1012400000BF00BF00BF00BF00BF00BF00BF00BFA6
:1012500000BF00BF00BF00BF00BF00BF00BF00BF96
:1012600000BF00BF00BF00BF00BF00BF3A4E4FF439
:101270008025F5639F2037F03BFA002037F038FADD
:1012800060F30704002037F033FA60F30F240020E6
:1012900037F02EFA60F31744B56300BF00BF00BFFC
:1012A00000BF00BF00BF00BF00BF00BF00BF00BF46
:1012B00000BF00BF00BF00BF00BF00BF00BF00BF36
:1012C00000BF00BF00BF00BF00BF00BF00BF00BF26
:1012D00000BF00BF00BF00BF00BF2049601A8C42A2
:1012E00033D019DC1E4A4FF48031A4EB0200944243
:1012F0002BD009DCA4F1C204B4F5A11425D08C4292
:1013000023D01848204413E000F65A70B0F540404E
:101310001BD0884216D118E0134A811A90420FD090
:1013200008DCA0F56060A9380FD0A0F55F40FA385E
:1013300040B90AE00D48081809D00D49C84201D14A
:10134000022400E00024204670BD0324FBE70424AF
:1013500038F072FAF7E7000000C009201F321700CA
:101360001C70150025C0FEFFA0F3290000FFFEFF42
:101370000001F8FF0148007870470000E8C207202C
:101380000549822008600549222008607846044902
:10139000086082207047000020C0072024C007207A
:1013A00028C00720002070470549822008600549B1
:1013B00021200860784604490860822070470000B8
:1013C00020C0072024C0072028C00720054982200C
:1013D0000860054922200860784604490860822098
:1013E0007047000020C0072024C0072028C0072025
:1013F0002DE9F041144B154D154E1B78154C63B17A
:101400009AB1154F03EB830307EBC3035B6998475E
:10141000000612D52068BDE8F081822020602120DE
:101420002860784630608220F5E786202060092019
:101430002860784630608620EDE700202060286034
:10144000784630600020E6E7E8C2072024C0072085
:1014500028C0072020C007207CC605002DE9F041E8
:10146000144B154D154E1B78154C63B19AB1154FA1
:1014700003EB830307EBC3039B699847000612D570
:101480002068BDE8F0818220206022202860784614
:1014900030608220F5E786202060092028607846A9
:1014A00030608620EDE700202060286078463060BC
:1014B0000020E6E7E8C2072024C0072028C0072054
:1014C00020C007207CC605002DE9F041144B154DC6
:1014D000154E1B78154C63B19AB1154F03EB83037E
:1014E00007EBC303DB699847000612D52068BDE807
:1014F000F08182202060222028607846306082209F
:10150000F5E7862020600920286078463060862034
:10151000EDE7002020602860784630600020E6E794
:10152000E8C2072024C0072028C0072020C00720C9
:101530007CC60500F8B5184C184D194E2778194C83
:10154000DDF818C087B1BCF1000F15D0CDF800C090
:10155000DFF854C007EB87070CEBC7073F6AB847B3
:10156000000611D52068F8BD822020602220286066
:10157000784630608220F8BD8620206009202860EF
:10158000784630608620F8BD0020206028607846CC
:1015900030600020F8BD0000E8C2072024C007200A
:1015A00028C0072020C007207CC60500084908681D
:1015B00088600861C0070AD00648817C002906D1EE
:1015C0008069002803D00448C06F38F04FBC7047D2
:1015D00000400050DCE6072004C30720F0B578285F
:1015E00000D9782000EB4003C3EBC015104C114824
:1015F00001EB41062023C6EBC111521E0ED3E3615D
:1016000086688768BF1BB7EBC50FFAD3A3618668EE
:101610008768BF1BB7EBC10FFAD3EEE7064900207E
:101620000860064908607846054908600020F0BD5A
:1016300000C009200000094020C0072024C0072066
:1016400028C00720012264210846FFF7C7BF0A7897
:1016500002F5FA6202804A7882708978C170704718
:101660000A7802F5FA6202804A7882708A78C2703B
:10167000CA780271097941710021817170470A7835
:10168000A2F5FA6202708A784270CA7882700A798A
:10169000C2704979017170470149087070470000B4
:1016A000B0C607202DE9F041002680F85C60A0F864
:1016B0005A60A0F87462B0F87622044635460727CF
:1016C00000F15C084AB10021204613F01DFF28B349
:1016D0004046F4F7EAFDA0B914E0012503E04046D6
:1016E000F4F7E3FD06442A466D1CADB20121204605
:1016F00013F00AFF0028F2D13146404614F074FA84
:1017000030B12770B4F87602401CA4F876020EE0DF
:1017100009202070BDE8F04114F05CBE0748A4F831
:101720007652C56045610820207014F053FE404693
:10173000F4F7BBFDA4F85A00BDE8F08100C0072013
:101740002DE9F0410646B0F85A50114806F15C0701
:10175000104C86600020711981F85C0010E0207840
:101760000028387805D014F0FDFD207838B960687D
:1017700004E014F0E9FC6068401E606028B17F1C42
:101780006D1EADB2EBD2BDE8F08109203070FAE7F2
:1017900000C0072000C707202DE9FF5FDFF8708237
:1017A0009C4FDFF8749298F80000DFF870A20025D3
:1017B000002834D19A4C092604F15C0B21780C29BD
:1017C0002DD2DFE801F02C063A4B52638C92C7D140
:1017D000E1F903A811F004FC000604D402A811F0FA
:1017E000F7FB000603D5386804B0BDE8F09FBDF8EC
:1017F0000C0038B1BDF80800400703D498F8010088
:1018000003280CD0201DF7F7F7FC98F802204FF0C2
:10181000020650EA020103D0267088F80250EEE07A
:10182000606800907F48019015F024F80028F6D0F9
:101830006846F7F7E1FCE0BBE1E018F0F5FD0028B1
:10184000EDD109F0FFFD0028E9D118F035FF0020A7
:1018500009F04CFF03202070642113E0201DF7F7EE
:10186000CBFC0028DBD004208CE06D4AB4F8581083
:1018700000231632012015F00BFFD0B10520207097
:101880004EF66021201DF7F7CDFCB8E0012015F0E1
:10189000EFFEB8B1012015F02FFF06202070A4F84C
:1018A0007652002168463AF065F918B18DF800507B
:1018B00005E012E09DF8000008B11E2000E0E0689D
:1018C00020619CE0201DF7F797FC30B9012015F04E
:1018D00077FEFF2802D0022800D026708FE0504803
:1018E000FFF7E0FE47F23051CCE7012015F0C0FED3
:1018F0000028F2D0B4F85A00B4F81480404500D261
:101900008046B4F8741242465944012015F002FF93
:10191000A0B147F23051201DF7F784FCB4F85A000B
:10192000A0EB08000004000CA4F85A00B4F87412EC
:101930004144A4F8741262D1062023E0012015F07E
:1019400059FE18B1201DF7F757FC98B326703C21BB
:10195000216154E0012015F04DFE4EF66021201D5E
:10196000F7F760FC0B200DE0206940B1012015F075
:1019700019FE6421201DF7F755FC0A2002E01E2005
:101980002061052020703AE0201DF7F735FC88B172
:10199000206900EB4001C1EBC011032000EBC10145
:1019A000201DF7F73FFC0120207018F085FE012074
:1019B00009F09CFE23E0FFE74FEA040840F21622FC
:1019C0005946012015F078FE041E0BDDA8F85A00D8
:1019D0001348FFF7B5FE4EF6602108F10400F7F753
:1019E00021FCEBE7012015F043FE30B108F10400C3
:1019F000F7F702FC08B9002C01DA88F800603D60B6
:101A0000C9F800507946CAF800100020ECE6000042
:101A1000B0C6072020C0072024C0072028C0072008
:101A20005CFB0720C0D4010070B588B01A4E07AD2A
:101A300041200096CDE9010501220923114613201A
:101A40003DF0DAFC154C00060FD430463AF06EF942
:101A5000102003A9CDE9001001220A2302951146A6
:101A600013203DF0C9FC000602D5206808B070BD07
:101A70009DF80D009DF80C1000EB01200649163969
:101A8000A1F8580000202060054908607846054903
:101A900008600020EAE7000072FB072020C0072052
:101AA00024C0072028C00720014900200870704783
:101AB0005CFB07202DE9F04F89B04FF42171654898
:101AC000F4F7B4FBDFF8908100264FF0100A88F895
:101AD00000600DF10C0BCDE900BA08AF01220B2319
:101AE0000297114613203DF087FC5C4D000677D429
:101AF0009DF80D009DF80C10564C10EB0120E06095
:101B000002D14FF46160E060DFF84891412109F1B2
:101B10001609CDF80090CDE90117012209231146DD
:101B200013203DF069FC00066ED448463AF0FEF8FA
:101B30004846F4F7BAFB00287ED00120207084F8D4
:101B4000796207A9CDE900100246014604230297F5
:101B500013203DF051FC000656D49DF81C000028CF
:101B60006FD088F80100B946CDE900BA0122574686
:101B7000D8460A2311461320CDF808903DF03CFCCE
:101B8000000641D49DF80D009DF80C10002300EBD9
:101B90000120A4F858001A4601219DF81C0015F0F8
:101BA00047FDCDE900870122032311461320CDF81C
:101BB00008903DF021FC000626D4039888B19DF8DA
:101BC0000F109DF80E00CDE900019DF80D309DF835
:101BD0000C2023A103A840F065FB002203A902E02A
:101BE00012E000221146012015F076FD01201F4A67
:101BF000CDE90020024601462F23CDF808900220AF
